:100000000C94440F0C94650F0C94650F0C94650FC1
:100010000C94650F0C94650F0C94650F0C94650F90
:100020000C94650F0C94650F0C9444660C946166F7
:100030000C94650F0C94650F0C9422670C944F6719
:100040000C947C670C94A9670C94D6670C94036895
:100050000C9430680C945D680C948A680C94B768B2
:100060000C94650F0D94A6240D94DD240C94650F5B
:100070000C94650F0C94650F0C94650F0C94650F30
:100080000C94650F0C94650F0C94650F0C94650F20
:100090000C94650F0C94650F0C94650F0D94DA4F5A
:1000A0000D940C500D943E500D9470500D94A8007A
:1000B0000C94650F0C94650F0C94650F0C94A66A54
:1000C0000C94D36A0C94006B0C942D6B0C945A6BAB
:1000D0000C94876B0C94B46B0C94E16B0C940E6CC9
:1000E0000C943B6C0C94650F0D94CA230D94012461
:1000F0000C94650F0C94650F0C94650F0C94650FB0
:100100000C94650F0C94650F0D9482050C94650F8B
:100110000C94650F0C94650F0C94650F0D94124FA1
:100120000D94444F0D94764F0D94A84F0C94650F89
:100130000C94650F0C94E4680C9411690C943E695E
:100140000C946B690C9498690C94C5690C94F269D1
:100150000C941F6A0C944C6A0C94796A0C94650F89
:100160000D9438240D946F240C94650F0C94650F36
:100170000C94650F0C94650F0C94650F0C94650F2F
:100180000C94650F0C94650F0C94650F0C94650F1F
:100190000C94650F0C94650F0C94650F0C94650F0F
:1001A0000D9475000C94650F0C94650F0C94650FFD
:1001B0000C94686C0C94956C0C94C26C0C94EF6C61
:1001C0000C941C6D0C94496D0C94650F0C94650F88
:1001D0000C94650F0C94650F0C94650F0D94142509
:1001E0000D944B250C94650F0C94650F0C94650FC2
:1001F0000C94650F0C94E1780C949C791E10A1105E
:100200003010A1104210A11054106E10541088101C
:1002100088104F12631277129D12C3123E132B13D4
:100220003E1305130513DC18DC1814195119951920
:10023000D2187E1A9A1AD71A351A351A9A1A7E1AAD
:10024000951951191419DC18DC188F229922A32250
:10025000AD22B722C122CB22D022D522DF22DF223B
:10026000D022CB22B722AD22A32299228F22A72708
:10027000A727AE27AE27C127E427A727E427AE2765
:10028000AE27A727E427AE27AE27A727A7271D2835
:100290001D28252825283A2861281D286128252879
:1002A00025281D286128252825281D281D28712876
:1002B00012299A2812291229EB281229C328C328A7
:1002C000EB2812299A2812297128452950295F29DB
:1002D0007A299029B229F829012A1C2AD829D82953
:1002E000012AF82990297A295F2950294529585F40
:1002F000CF5FCF5FE85ECF5FCF5FCF5FCF5FCF5F76
:10030000CF5FCF5FCF5FCF5FCF5FCF5FCF5FCF5F7D
:10031000CF5FFD5ECF5FCF5FCF5FCF5FCF5FCF5F40
:10032000CF5F525FB05FCF5FCF5FBD5FCF5FCF5F0B
:10033000CF5FCF5FCF5FCF5F6B5FCF5FCF5FC95FB7
:10034000CF5FCC5FCF5FCF5FCF5FCF5FC65FCF5F49
:10035000CF5FCF5FCF5FCF5FCF5FCF5FCF5FCF5F2D
:10036000CF5FCF5FCF5FCF5FCF5FCF5FCF5FCF5F1D
:10037000CF5FCF5FCF5FCF5FCF5FCF5FCF5FCF5F0D
:10038000CF5FCF5FCF5FCF5FCF5FCF5FCF5FCF5FFD
:10039000CF5FCF5FCF5FCF5FCF5FCF5FCF5FCF5FED
:1003A000CF5F555FB573B873BB73BE73C173C4734E
:1003B000C773347B477B5A7B6D7B807B937BA67BAB
:1003C000AE80AE802B8070807080E37FE37F708092
:1003D000708070807080708070807080708070809D
:1003E000708070807080708070807080E37F70801B
:1003F0007080708070807080BA85FA86F58524865A
:10040000FA86FA86FA86FA86FA86FA86FA86FA86EC
:10041000FA86FA86FA86FA86FA86FA86FA86FA86DC
:10042000FA86FA86FA86FA86FA86FA86FA86FA86CC
:10043000FA86FA86FA86FA86FA86FA86FA86FA86BC
:10044000FA86FA86FA86FA86FA86FA86FA86FA86AC
:10045000FA86FA86FA86FA86FA869F86FA865E8693
:10046000FA86FA86BA86FA86FA86FA86FA86FA86CC
:10047000FA86FA86FA86FA86FA86FA866D86FA8609
:100480007B868390B38EEC8E368F9C8FE78FFC8FAC
:100490002E90509071903692C390CB90E890279117
:1004A0003A918491A691BD91D2913192319231923B
:1004B0003192319231923192319231923192E9916D
:1004C000F191FC9111921792D7AE07AFB3AEBFAEC8
:1004D00007AF07AF07AF07AF07AF07AF07AF07AF6C
:1004E00007AF07AF07AF07AF07AF07AFCBAE07AF99
:1004F00007AF07AF07AF07AF07AF07AF07AF07AF4C
:1005000007AF07AF07AF07AFD7AE07AFB3AEBFAE0A
:1005100007AF07AF07AF07AF07AF07AF07AF07AF2B
:1005200007AF07AF07AF07AF07AF07AFCBAE3EBA16
:1005300041BA92BA92BA92BA92BA92BA92BA92BAAC
:1005400092BA92BA92BA92BA92BA92BA92BA92BA4B
:1005500092BA92BA92BA92BA78BA92BA92BA92BA55
:1005600092BA92BA92BA5EBA92BA92BA92BA92BA5F
:1005700092BA44BA92BA92BA92BA92BA92BA92BA69
:1005800092BA92BA92BA92BA92BA92BA92BA92BA0B
:1005900092BA92BA92BA92BA78BA92BA92BA92BA15
:1005A00092BA92BA92BA5EBA92BA92BA92BA92BA1F
:1005B00092BA44BA3BBD38BD4DBD4DBD4DBD4DBDDC
:1005C0004DBD4DBD4DBD4DBD4DBD4DBD4DBD4DBDDB
:1005D0004DBD4DBD4DBD84BC57BC75BC4DBD4DBD65
:1005E000FBBC3EBC4DBD4DBD4DBD4DBD4DBD66BC06
:1005F0003EBD4DBD4DBD8EBC4DBD4DBD4DBD4DBD7A
:100600004DBD4DBD4DBD4DBD4DBD4DBD4DBD4DBD9A
:100610004DBD4DBD4DBD84BC57BC75BC4DBD4DBD24
:10062000FBBC3EBC4DBD4DBD4DBD4DBD4DBD66BCC5
:100630003EBD4DBD4DBD8EBC40C083C092C092C07A
:1006400092C092C092C092C092C092C092C092C01A
:1006500092C092C092C073BF92C02AC024C08CBF07
:100660003AC092C092C09CBF73BF92C092C04FC0AC
:1006700080BF34C088C030C092BF45C01EC097BF85
:1006800092C04AC06FBF8DC092C092C086BF92C058
:1006900092C092C092C092C092C02AC024C08CBFA7
:1006A0003AC092C092C09CBF73BF92C092C04FC06C
:1006B00080BF34C088C030C092BF45C01EC097BF45
:1006C00092C04AC06FBF8DC092C092C086BF4FBF5C
:1006D000B2C5A2C5A4C5A6C5A8C5AAC5ACC5AEC5A8
:1006E000CFC5BFC5C1C5C3C5C5C5C7C5C9C5CBC5B0
:1006F000DCC50AC6E4C50AC6E4C50AC6E4C50AC61E
:10070000E4C50AC6E4C50AC60AC60AC60AC60AC6B7
:100710000AC60AC6EBC5F2C5FEC5FEC53AD969D7F9
:1007200075D7C0D7F1D8D5D717D83BD864D8BFD89C
:10073000F1DFF1DF7BE0B3E193E2BBE3A5E493E516
:10074000A5E4DFE6DFE693E5A5E493E2B3E17BE031
:10075000F1DFF1DF15E915E956E9B4E9F3E941EA1A
:1007600076EAB5EA76EA03EB03EBB5EA76EAF3E973
:10077000B4E956E915E915E960EDCBED36EEEFEE9B
:100780009BEF8BF074F12BF274F12CF32CF32BF222
:1007900074F19BEFEFEE36EECBED60ED0D940D11A5
:1007A0000D944B100D9480110D9400120D94E811CE
:1007B0000D9466124E414E494E495459494E46CD0C
:1007C000CCCC3D0AD7233C17B7D13877CC2B329508
:1007D00095E6241FB14F0A000020410000C84200E6
:1007E000401C4620BCBE4CCA1B0E5AAEC59D74327E
:1007F00035304D4F686D0032354D4F686D003630E5
:10080000487A003530487A004E6F6E2D496E74007C
:1008100048692D4C4F004750530054696D650044A2
:10082000697374616E6365005075736820427574F6
:10083000746F6E00496D70657269616C004D65740E
:1008400072696300494E4300444543004F4E004FD8
:100850004646005B0956094C094509390932092603
:100860000915090709F408E108CC08BB08A8089A8B
:10087000088B08810877084349505326414356475F
:1008800000444356472641435647004349505326A8
:10089000444356472641435647003278444356471F
:1008A0002632784143564700434950532632784414
:1008B00043564726327841435647003278496D7097
:1008C0002E20434950532641435647003278496D04
:1008D000702E4349505326444356472641435647BA
:1008E00000327843495053263278444356472641D4
:1008F000435647003278496D702E204349505326A5
:1009000032784443564700506172616C6C656C20CC
:1009100043495053003278496D702E20434950535B
:100920002644435647003278496D702E2043495083
:100930005300347844435647004349505326327895
:100940004443564700327844435647004349505386
:1009500026444356470044435647004349505300FA
:100960002B126911A710E50F230F610E9F0DDD0CEF
:100970001B0C590BF80ADD0C9F0D230FE50FA71078
:1009800069112B128C12CA1108114610840FC20E65
:10099000000E3E0D7C0CBA0BF80A3E0D000E840FC3
:1009A00046100811CA118C1253616D706C652F735B
:1009B00065633A004552524F5220202020202000EB
:1009C000432D434950532C20522D434950532C2042
:1009D0000000000000000000000000000000000017
:1009E0000000000000000000000000000000000007
:1009F00000000000000000000000000000000000F7
:100A000000000000000000000000000000000000E6
:100A100000000000000000000000000000000000D6
:100A2000004C6F2D434950532C2048692D434950A9
:100A3000532C200000000000000000000000000017
:100A400000000000000000000000000000000000A6
:100A50000000000000000000000000000000000096
:100A60000000000000000000000000000000000086
:100A70000000000000000000000000000000000076
:100A80000000434950532C200000000000000000EB
:100A90000000000000000000000000000000000056
:100AA0000000000000000000000000000000000046
:100AB0000000000000000000000000000000000036
:100AC0000000000000000000000000000000000026
:100AD0000000000000000000000000000000000016
:100AE0000000004143564752506F6C2C2041435642
:100AF0004752526D732C2000414356474C506F6C47
:100B00002C20414356474C526D732C20414356478D
:100B100052506F6C2C204143564752526D732C201B
:100B200000000000000000000000000000000000C5
:100B300000000000000000000000000000000000B5
:100B400000000000000000000000000000000000A5
:100B5000000000000000000000522D4443564720D2
:100B60004F6E2C204C2D44435647204F6E2C204C6A
:100B70006F2D43495053204F6E2C2048692D434917
:100B80005053204F6E2C20522D44435647204F6621
:100B9000662C204C2D44435647204F66662C204C33
:100BA0006F2D43495053204F66662C2048692D43D2
:100BB000495053204F66662C2000522D444356471F
:100BC000204F66662C204C2D44435647204F6666C6
:100BD0002C204C6F2D43495053204F66662C2048E3
:100BE000692D43495053204F66662C20522D4443B3
:100BF0005647204F6E2C204C2D44435647204F6EB5
:100C00002C204C6F2D43495053204F6E2C204869A7
:100C10002D43495053204F6E2C2000432D43495003
:100C200053204F6E2C20522D43495053204F6E2C91
:100C300020432D43495053204F66662C20522D43AC
:100C4000495053204F66662C200000000000000031
:100C50000000000000000000000000000000000094
:100C60000000000000000000000000000000000084
:100C7000000000000000000000000000432D434978
:100C80005053204F66662C20522D43495053204F1D
:100C900066662C20432D43495053204F6E2C205222
:100CA0002D43495053204F6E2C20000000000000BF
:100CB0000000000000000000000000000000000034
:100CC0000000000000000000000000000000000024
:100CD00000000000000000000000000000522D4451
:100CE000435647204F6E2C204C6F2D4349505320C4
:100CF0004F6E2C2048692D43495053204F6E2C20B5
:100D0000522D44435647204F66662C204C6F2D438E
:100D1000495053204F66662C2048692D4349505353
:100D2000204F66662C20000000000000000000003C
:100D30000000000000000000000000000000522D34
:100D400044435647204F66662C204C6F2D43495034
:100D500053204F66662C2048692D43495053204F3D
:100D600066662C20522D44435647204F6E2C204C53
:100D70006F2D43495053204F6E2C2048692D434915
:100D80005053204F6E2C2000000000000000000097
:100D90000000000000000000000000000000004C07
:100DA0006F2D43495053204F6E2C2048692D4349E5
:100DB0005053204F6E2C204C6F2D43495053204FE1
:100DC00066662C2048692D43495053204F66662C97
:100DD00020000000000000000000000000000000F3
:100DE0000000000000000000000000000000000003
:100DF00000000000000000000000000000000000F3
:100E00004C6F2D43495053204F66662C2048692D66
:100E100043495053204F66662C204C6F2D43495058
:100E200053204F6E2C2048692D43495053204F6E5C
:100E30002C20000000000000000000000000000066
:100E400000000000000000000000000000000000A2
:100E50000000000000000000000000000000000092
:100E600000522D44435647204F6E2C204C2D4443B6
:100E70005647204F6E2C20462D44435647204F6E38
:100E80002C20422D44435647204F6E2C20522D4497
:100E9000435647204F66662C204C2D44435647202E
:100EA0004F66662C20462D44435647204F66662CDD
:100EB00020422D44435647204F66662C20000000F8
:100EC0000000522D44435647204F66662C204C2D7F
:100ED00044435647204F66662C20462D44435647D0
:100EE000204F66662C20422D44435647204F6666AD
:100EF0002C20522D44435647204F6E2C204C2D441D
:100F0000435647204F6E2C20462D44435647204FD2
:100F10006E2C20422D44435647204F6E2C2000005B
:100F2000000000522D44435647204F6E2C204C2D7C
:100F300044435647204F6E2C2043495053204F6E58
:100F40002C20522D44435647204F66662C204C2DB2
:100F500044435647204F66662C2043495053204F48
:100F600066662C2000000000000000000000000069
:100F70000000000000000000000000000000000071
:100F800000000000522D44435647204F66662C2037
:100F90004C2D44435647204F66662C2043495053FE
:100FA000204F66662C20522D44435647204F6E2C0E
:100FB000204C2D44435647204F6E2C20434950531C
:100FC000204F6E2C200000000000000000000000F8
:100FD0000000000000000000000000000000000011
:100FE0000000000000522D44435647204F6E2C2035
:100FF0004C2D44435647204F6E2C20522D444356CF
:1010000047204F66662C204C2D44435647204F66A0
:10101000662C20000000000000000000000000001E
:1010200000000000000000000000000000000000C0
:1010300000000000000000000000000000000000B0
:10104000000000000000522D44435647204F6666C2
:101050002C204C2D44435647204F66662C20522DA1
:1010600044435647204F6E2C204C2D444356472076
:101070004F6E2C2000000000000000000000000067
:101080000000000000000000000000000000000060
:101090000000000000000000000000000000000050
:1010A00000000000000000522D44435647204F6EC0
:1010B0002C2043495053204F6E2C20522D44435630
:1010C00047204F66662C2043495053204F66662CBC
:1010D00020000000000000000000000000000000F0
:1010E0000000000000000000000000000000000000
:1010F00000000000000000000000000000000000F0
:101100000000000000000000522D44435647204FCD
:1011100066662C2043495053204F66662C20522D82
:1011200044435647204F6E2C2043495053204F6E66
:101130002C20000000000000000000000000000063
:10114000000000000000000000000000000000009F
:10115000000000000000000000000000000000008F
:10116000000000000000000000522D4443564720BC
:101170004F6E2C20522D44435647204F66662C203C
:10118000000000000000000000000000000000005F
:10119000000000000000000000000000000000004F
:1011A000000000000000000000000000000000003F
:1011B000000000000000000000000000000000002F
:1011C00000000000000000000000522D444356477C
:1011D000204F66662C20522D44435647204F6E2CDC
:1011E00020000000000000000000000000000000DF
:1011F00000000000000000000000000000000000EF
:1012000000000000000000000000000000000000DE
:1012100000000000000000000000000000000000CE
:10122000000000000000000000000043495053206F
:101230004F6E2C2043495053204F66662C200000EF
:10124000000000000000000000000000000000009E
:10125000000000000000000000000000000000008E
:10126000000000000000000000000000000000007E
:10127000000000000000000000000000000000006E
:10128000000000000000000000000000434950532F
:10129000204F66662C2043495053204F6E2C20006F
:1012A000000000000000000000000000000000003E
:1012B000000000000000000000000000000000002E
:1012C000000000000000000000000000000000001E
:1012D000000000000000000000000000000000000E
:1012E0000000000000000000000000000044656CE9
:1012F00061792054696D653B0046696C65204E61DB
:101300006D653A2000436861696E6167652C200055
:10131000004C6F63616C54696D652C204C6F636188
:101320006C444D592C204C61742D4465672C204E23
:10133000532C204C6F6E2D4465672C2045572C2074
:10134000466978537461742C204E756D5361742C0A
:101350002050444F502C20416C745F4D2C2043682A
:101360006B2C20436F6D6D0000000000000000003A
:10137000000000000000000000000000000000006D
:1013800000000000000000000000000000004C6FA2
:1013900063616C54696D652C204C6F63616C444DC6
:1013A000592C204C61742D4465672C204C61742DA0
:1013B0004D696E2C204C61742D5365632C204E5367
:1013C0002C204C6F6E2D4465672C204C6F6E2D4D7C
:1013D000696E2C204C6F6E2D5365632C2045572C65
:1013E00020466978537461742C204E756D53617476
:1013F0002C2050444F502C20416C745F4D2C2043C6
:10140000686B2C20436F6D6D000000484558434FBA
:10141000524445522043414C4942482E54585400AE
:1014200000007777772E636174682D746563682E8A
:10143000636F6D0000000000004C494D4954454465
:10144000203930352D3835372D313035300000001A
:10145000434154484F44494320544543484E4F4C20
:101460004F47590000007B702C30302C662C007BDD
:10147000702C30302C657D007B702C30302C6F7DD3
:1014800000686369746F6F6C207061697220004539
:101490006E7465722050494E203A2000686369637B
:1014A0006F6E666967206E616D65200061742B62E6
:1014B00074642A007175697400736D6172745A00E6
:1014C00061742B72756E00456E74657220414356CF
:1014D00047202827462720666F722046726F6E7459
:1014E0002C2027422720666F72204261636B290AF5
:1014F0000D20616E6420737570706C79203332300A
:101500002B3634302073696E657761766520776994
:101510007468205065616B546F5065616B20766F05
:101520006C74616765206F6620302E385600456EFA
:101530007465722053434F504520766F6C74616719
:101540006520696E206D5620284E4E4E4E4E290065
:10155000456E746572204349505320766F6C7461F8
:10156000676520696E206D562A313020284E4E4E18
:101570004E4E2900456E74657220444356472076CE
:101580006F6C7461676520696E206D562A3130205A
:10159000284E4E4E4E4E2900CE15C715C315BF1509
:1015A000BB15B715A815A815432D53474E44205B0E
:1015B000352D3430565D00432D4200432D46004307
:1015C0002D5200432D4C00522D53474E4400432DC5
:1015D00053474E440020616E6420656E746572202E
:1015E000766F6C7461676520696E206D562A3130A4
:1015F00020284E4E4E4E4E2900506C65617365207A
:10160000636F6E6E65637420004572726F722C207A
:101610006D697373696E6720414443206E756D2058
:1016200028302D3729000A0D5363616C696E6743BA
:10163000616C6962204F66667365743A200045727A
:10164000726F722C20656E74657220766F6C746197
:10165000676520696E206D562A313020284E4E4E27
:101660004E4E29001217F316DD16D116AD169A1636
:10167000721643535B302F312F322F332F345D5B83
:1016800076767676765D202D204443205363616C18
:10169000696E672043616C6962004342202D2042DD
:1016A0006174746572792043616C696200435A5BAE
:1016B000302F312F322F332F345D202D2044432003
:1016C0005A65726F4F66667365742043616C696218
:1016D0000056202D20566E756D626572004C5B6958
:1016E0006E785D5B4F4E2F4F46465D202D204C653A
:1016F000647300416E6E202D205265616420414468
:10170000433120666F72206E6E207365636F6E6466
:10171000730041202D205265616420414443310013
:101720004552524F52004F4B0043415448205445BC
:10173000434820484558434F524445522056303183
:101740002E303900010002000300040005000600ED
:101750000A000C000F0014001E003C007800B400CA
:10176000F0002C01680100000000120002000100DE
:10177000B80B0F27010064006801100E010010274C
:101780001027102710271027102701000100010043
:101790000100F8010100010002000100F401000055
:1017A00000000100000000000A00F1D80000010064
:1017B0000100C8000000640064006400640064006C
:1017C0006400000000000000000050FE0000000067
:1017D0000000000001000000000001000000000007
:1017E0000A00000001000100020058020000FA0097
:1017F000FA00FA00FA00780078000000000000000B
:1018000001000000010001000000000001000100D3
:101810000080001900800019008000190080001964
:101820000080001900800019008000190080001954
:1018300000000100FF03E600E6007018621854186B
:101840004D18244A42494E2C39342C3100244A5335
:1018500041564500244A4153432C47504753412C9D
:101860003100244A4153432C4750524D432C310000
:10187000244A4153432C47504747412C31002450C0
:101880004D544B3636372A33350024504D544B33A4
:1018900031342C302C312C302C312C312C302C305C
:1018A0002C302C302C302C302C302C302C302C3058
:1018B0002C302C302C302C302A323900756E6C6F65
:1018C00067206C62616E64747261636B73746174BF
:1018D00061006C6F67206C62616E64747261636B2F
:1018E0007374617461206F6E74696D6520313000AE
:1018F000756E6C6F6720707372706F7361006C6FC0
:101900006720707372706F7361206F6E74696D659C
:1019100020313000646174756D207573657200202C
:10192000302E3020302E3020302E3020302E30001F
:1019300075736572646174756D2000646174756D92
:1019400020776773383400756E6C6F67206770613D
:101950006C6D006C6F67206770616C6D206F6E74CA
:10196000696D6520313000D019C119B219A3199BD6
:101970001982197519245047524D432C2C2C393695
:101980002C00245047524D432C412C2C3130302C0C
:101990002C2C2C2C2C2C2C2C2C2C00245047524D35
:1019A000434500245047524D4F2C5047524D542C24
:1019B0003000245047524D4F2C5047524D462C3149
:1019C00000245047524D4F2C47504753562C30005F
:1019D000245047524D4F2C2C3400311A221A131A1E
:1019E000041AF519E619445A203D200000000000B1
:1019F00000000000004459203D20000000000000CD
:101A0000000000004458203D2000000000000000BD
:101A1000000000466C6174203D20000000000000C2
:101A200000004D616A6F7241203D200000000000FF
:101A3000005354505220444154554D2E5458540094
:101A40007D1B701B631B561B491B3C1B2F1B221B42
:101A5000151B081BFB1AEE1AE11AD41AC71ABA1A78
:101A6000AD1AA01A931A861A791A6C1A414356476E
:101A70003220524D53203D200041435647312052E1
:101A80004D53203D200042415454202043616C209E
:101A90003D200041432020205343616C203D200025
:101AA00041432020205A43616C203D2000414443A3
:101AB00037205653636C203D200041444337205A61
:101AC00043616C203D200041444336205653636CF3
:101AD000203D200041444336205A43616C203D2084
:101AE0000041444335205653636C203D200041445F
:101AF0004335205A43616C203D200041444334204B
:101B00005653636C203D200041444334205A4361C6
:101B10006C203D200041444333205653636C203DEC
:101B2000200041444333205A43616C203D20004152
:101B3000444332205653636C203D200041444332DD
:101B4000205A43616C203D200041444331205653CC
:101B5000636C203D200041444331205A43616C2096
:101B60003D200041444330205653636C203D20000B
:101B700041444330205A43616C203D200046696C4B
:101B80006520496E646578203D20002B1E151EFFE0
:101B90001DE91DD31DBD1DA71D911D7B1D651D4F7D
:101BA0001D391D231D0D1DF71CE11CCB1CB51C9FF1
:101BB0001C891C731C5D1C471C311C1B1C051CEF65
:101BC0001BD91B454E44000000000000000000002F
:101BD0000000000000000000004443564720446518
:101BE000666563742056616C203D2000000000444F
:101BF0004356472044656665637420456E203D204A
:101C0000000000000053796E632054797065203D18
:101C10002000000000000000000000434950532055
:101C200052616E6765202B2F2D3556203D20000018
:101C30000047505320436F6F726420696E20444DFB
:101C400053203D200000004C6F63616C475053549B
:101C5000696D654F6666736574203D2000414320C1
:101C60004672657175656E6379203D200000000045
:101C700000000042726F6B656E5769726520416C9F
:101C800061726D203D200000004C6F7720506F7412
:101C900020416C61726D203D200000000000004971
:101CA0006E70757420496D706564616E6365203D6A
:101CB0002000000000444356474D44656C4F4E20C1
:101CC0003D20000000000000000000444356474D46
:101CD00044656C4F4646203D200000000000000097
:101CE0000043495053324D44656C4F4E203D200017
:101CF0000000000000000043495053324D44656C21
:101D00004F4646203D20000000000000004349509F
:101D100053314D44656C4F4E203D200000000000C3
:101D200000000043495053314D44656C4F464620F6
:101D30003D20000000000000005374617274576978
:101D40007468203D20000000000000000000004FEB
:101D5000666654696D65205B6D7365635D203D202B
:101D60000000000000546F74616C4379636C65205F
:101D70005B7365635D203D2000000054696D652044
:101D800056616C7565203D200000000000000000D9
:101D900000436861696E61676520446972656374B8
:101DA000696F6E203D200053746172742043686136
:101DB000696E616765203D20000000000044697382
:101DC00074616E63652056616C7565203D2000006E
:101DD0000000004D6561737572656D656E74205508
:101DE0006E697473203D20000053746F72616765E3
:101DF00020416374696F6E203D2000000000005395
:101E000075727665792054797065203D2000000058
:101E100000000000004F70657261746F72204E61A7
:101E20006D65203D2000000000000053757276654E
:101E300079204E616D65203D20000000000000000B
:101E40000054532D5453204F4E203D200054532D09
:101E50005453204F4646203D20004E4557205453B2
:101E6000204F4E203D20004E4557205453204F46D2
:101E700046203D20005453204F4E203D2000545317
:101E8000204F4646203D200011241FBECFEFCDBF7E
:101E9000DFE5DEBF00E00CBF1FE2A0E0B0E2E8E15A
:101EA000F3EB02E00BBF02C007900D92AC38B10714
:101EB000D9F724E5ACE8BFE201C01D92A630B20715
:101EC000E1F70E94093E0D948A590C940000CF93CB
:101ED000DF93CDB7DEB72B97CDBFDEBFBE016F5FFF
:101EE0007F4F80E092E00F94F250AE01485F5F4F69
:101EF00068E080E092E00F944E518A819B819F7848
:101F00009B8395E09D83817E8A831C82BE016F5FE7
:101F10007F4F80E092E00F94A25081E0888788E1B3
:101F20008987AE01485F5F4F68E080E092E00F94E0
:101F3000155180E092E00F94034F2B96CDBFDEBF8A
:101F4000DF91CF9108959FB7F894E0E0F2E08081AF
:101F5000806280839FBF0895009781F020910602E0
:101F600023FF0EC020913C0230913D02FC012083F2
:101F7000318388E08093060281E0089580E008952F
:101F800080E00895CF92DF92EF92FF92CF93DF939C
:101F90000097D1F061157105C9F0EB01FC01A0813A
:101FA000B18128EE33E00F94A2546B017C0183E1F0
:101FB0000E947DC19B01AC01C701B6010F944D5435
:101FC0002883398381E003C080E001C080E0DF9195
:101FD000CF91FF90EF90DF90CF900895E1EBF8E381
:101FE0001082118214821582128213821682178245
:101FF0008BE00E94A1C1672B682B692B19F410920A
:10200000B93803C081E08093B938E1EBF8E3118679
:1020100012860895CF93DF93EC01892B09F491C0C8
:10202000862F90E0FC013197EB30F10508F089C074
:102030008827E250FF4F8F4F0D948B548091B93811
:10204000811107C0888199818093B5389093B63803
:1020500078C08A819B818093B5389093B63871C0DF
:102060008091B938811107C08A819B818093B538EE
:102070009093B63866C08E819F818093B5389093D7
:10208000B6385FC08091B938811107C08C819D81BD
:102090008093B5389093B63854C08A859B858093D9
:1020A000B5389093B6384DC08091B93881110BC0C6
:1020B00088819981E1EBF8E3848395838A819B8110
:1020C000868397833EC08C819D81E1EBF8E3848316
:1020D00095838E819F818683978333C08091B938A1
:1020E00081110BC08A819B81E1EBF8E384839583A6
:1020F0008C819D818683978324C0E1EBF8E38885FA
:102100009985848395838A859B858683978319C067
:102110008091B93881110BC08C819D81E1EBF8E38E
:10212000848395838E819F81868397830AC0E1EBA8
:10213000F8E38C859D85848395838E859F85868332
:102140009783DF91CF910895E1EBF8E38481958146
:102150008083918386819781828393830895E1EBC5
:10216000F8E381E0818712860895E1EBF8E31186B8
:10217000128608958091BB38089583E10E94A1C121
:10218000672B682B692B19F08091BA38089580E08D
:102190000895CF92DF92EF92FF926B01072E000C11
:1021A000EE08FF08C216D306E406F5067CF486178F
:1021B0009707E4F0092E000CAA0BBB0BE1E02817EF
:1021C00039074A075B07ACF4E0E013C06C01092E45
:1021D000000CEE08FF08C216D306E406F50644F02C
:1021E000E1E0681779072CF4E0E003C0E0E001C00B
:1021F000E0E08E2FFF90EF90DF90CF900895FF9258
:102200000F931F93CF93DF93C1EBD8E305EB18E354
:10221000F12CE991F991309719F1AF010F2E000CD3
:10222000660B770BDB01CA0177231CF40196A11D15
:10223000B11DB595A795979587959A01AB01280F84
:10224000391F4A1F5B1FBF01FF2314F46F5F7F4FCD
:10225000759567958A819B819CDF813009F0F394A5
:10226000C017D107B1F6FF2011F079DF01C07DDF83
:102270006BDFDF91CF911F910F91FF900895E1EBFC
:10228000F8E381E090E0A0E0B0E08787908BA18B3D
:10229000B28B838B948BA58BB68B178A138614868F
:1022A00015861686108E0895E1EBF8E381E0878BA2
:1022B000108E0895E1EBF8E3178A108E089580914F
:1022C000C938089584E10E94A1C1672B682B692B4E
:1022D00019F08091C838089580E00895E1EBF8E3A3
:1022E00087859089A189B289838B948BA58BB68BC6
:1022F00083859485A585B6858787908BA18BB28BC6
:1023000008956093BC387093BD388093BE38909325
:10231000BF3808958F929F92AF92BF92CF92DF9273
:10232000EF92FF92E1EBF8E3C388D488E588F68862
:1023300087859089A189B289C816D906EA06FB0665
:1023400091F48090BC389090BD38A090BE38B09089
:10235000BF38C4DFC814D904EA04FB0411F4A4DFB5
:1023600004C0A8DF02C0BADFFCCFFF90EF90DF907F
:10237000CF90BF90AF909F908F9008958BE10E9477
:10238000A1C16093CA387093CB388093CC389093B6
:10239000CD38AEECB8E3E1EBF8E389EB98E31D92BE
:1023A00011A212A232968E179F07C9F7E1EBF8E34C
:1023B00011A612A6089581E09091DA38911101C01A
:1023C00080E008958AE10E94A1C1672B682B692BE8
:1023D00039F081E09091DA38911103C080E00895DE
:1023E00080E008950F931F938B019C018091CA3860
:1023F0009091CB38A091CC38B091CD380097A10501
:10240000B10529F1880F991FAA1FBB1FAC01BD019F
:10241000440F551F661F771F440F551F661F771FF8
:10242000840F951FA61FB71FB901A80133233CF4E1
:1024300044275527BA01401B510B620B730B21E057
:1024400084179507A607B7071CF020E001C020E01D
:10245000822F1F910F9108950F931F93CF93DF93B6
:10246000009709F40BC1A1EBB8E35D961C925D9750
:102470005E961C925E975F961C925F9790961C9258
:10248000462F50E0FA013297EA30F10508F0F6C025
:10249000EC018827E75FFE4F8F4F0D948B5480919E
:1024A000B938811108C06C817D818E819F819ADF4E
:1024B0008093CE38E3C0688179818A819B8192DFE5
:1024C0008093CE38DBC08091B938811108C068850F
:1024D00079858A859B8586DF8093CE38CFC06881D9
:1024E00079818A819B817EDF8093CE38C7C08091BD
:1024F000B938811111C0688579858A859B8572DF1D
:1025000001EB18E3F801858F6C857D858E859F85AD
:1025100069DFF801868FB2C0688179818A819B81E9
:1025200061DF01EB18E3F801858F6C817D818E817D
:102530009F8158DFF801868FA1C08091B938811141
:1025400011C06C857D858E859F854CDF01EB18E37E
:10255000F801858F688979898A899B8943DFF80129
:10256000868F8CC0688179818A819B813BDF01EBFA
:1025700018E3F801858F6C817D818E819F8132DF28
:10258000F801868F7BC08091B93881111FC068899E
:1025900079898A899B8926DF01EB18E3F801858F09
:1025A0006C897D898E899F891DDFF801868F688DF2
:1025B000798D8A8D9B8D16DFF801878F6C8D7D8DCF
:1025C0008E8D9F8D0FDFF80180A358C068817981BF
:1025D0008A819B8107DF01EB18E3F801858F6C810D
:1025E0007D818E819F81FEDEF801868F68857985E9
:1025F0008A859B85F7DEF801878F6C857D858E85C2
:102600009F85F0DEF80180A339C08091B93881112F
:1026100011C0688979898A899B89E4DE01EB18E316
:10262000F801858F6C897D898E899F89DBDEF801B1
:10263000868F24C0688179818A819B81D3DE01EBFA
:1026400018E3F801858F6C817D818E819F81CADEC0
:10265000F801868F13C08091B938811108C06C854C
:102660007D858E859F85BEDE8093CE3807C06881CC
:1026700079818A819B81B6DE8093CE38DF91CF91BC
:102680001F910F910895843040F5E1EBF8E341A5E7
:1026900052A5242F30E0082E02C0359527950A94C4
:1026A000E2F720FF0AC0252F30E0082E02C0359542
:1026B00027950A94E2F720FD10C021E030E0B9012F
:1026C00002C0660F771F8A95E2F7CB01E1EBF8E3D2
:1026D000462B41A78095852382A70895843090F4E6
:1026E00021E030E0A90102C0440F551F8A95E2F7AE
:1026F000CA018095E1EBF8E391A5982391A792A5F3
:10270000892382A70895BF92CF92DF92EF92FF9222
:102710000F931F93CF93DF930EEC18E3C1EBD8E335
:102720006E017801B12CF70181917F01F60121A1A1
:1027300090E0820F911D22A1820F911D039719F441
:102740008B2DA1DF02C08B2DC9DFB394F2E0CF0E39
:10275000D11C84E0B812E7CF29EB38E389A18AA322
:10276000F80181918F0189A32296C217D307B1F78F
:10277000DF91CF911F910F91FF90EF90DF90CF905D
:10278000BF900895843060F42091DA3830E0A901D8
:1027900002C0559547958A95E2F7CA018170089560
:1027A00080E00895843060F42091DB3830E0A901A6
:1027B00002C0559547958A95E2F7CA018170089540
:1027C00081E00895843000F5662379F0E1EBF8E3C9
:1027D00021E030E0A90102C0440F551F8A95E2F7BD
:1027E000CA0192A5892B82A70895E1EBF8E321E0C5
:1027F00030E0A90102C0440F551F8A95E2F7CA01D3
:10280000809592A5892382A70895CF93833009F1FB
:1028100028F4813031F0823061F02CC0883008F12A
:1028200029C08091C838882329F181E08093C93874
:1028300021C0C1DD8823F1F061E080E0C3DF61E009
:1028400081E0C0DF61E082E0BDDF61E083E0BADF0C
:1028500011C08091BA38882369F081E08093BB3839
:1028600009C0CCEFC80F8C2F8DDF882319F061E0F1
:102870008C2FA8DFCF910895009781F0FC01DC0137
:10288000AD5BBD4F80818C936083643021F481E027
:102890000D943F06089580E00D943F06089500973B
:1028A00019F0FC018081089580E008950F931F9333
:1028B000CF93DF931F92CDB7DEB7009709F4C6C060
:1028C0008C0181E0D8018C9311961C92119712967D
:1028D0001C92129713961C92139714961C9214979D
:1028E00015961C921597169682E1E0E2F4E20190AB
:1028F0000D928A95E1F7C80148960E94C8C6F80172
:10290000808D8783818D8087828D8187838D82876B
:10291000CE0101960E94E9C689818C3438F4D80131
:102920005C961C925C975D961C9211C08C3431F4BD
:1029300082E0F801848F81E0858F09C08D3439F4FD
:1029400082E0D8015C968C935C975D961C9280E047
:102950000E947DC1673EB3E07B0781059105BCF411
:102960009F938F937F936F9384EE90E29F938F93C7
:10297000C801C6969F938F930F94B856F80186A905
:10298000808B87A9818B80AD828BCDBFDEBFD801C4
:102990005E961C925E975F961C925F97D2961C92F1
:1029A000D297D3961C92F801EA5CFD4F10823196C3
:1029B000108231961082319681E0808331961082A8
:1029C000118212821382349681E090E0A0E0B0E0A0
:1029D00080839183A283B383349610823196D80189
:1029E0008C918083E751F24086E0DF011D928A9549
:1029F000E9F7E85EFD4F1082118232961082118253
:102A00003296108211823296108211823296108292
:102A10003196108232961082319610823196108251
:102A20003196108231961082319610823196108242
:102A3000118212821382349610823196108231965E
:102A40001082319688E690E1808391830F90DF9128
:102A5000CF911F910F910895009741F0613021F4BB
:102A600021E0FC0122AB0895FC0112AA0895009711
:102A700019F0FC0182A9089580E00895009741F0C3
:102A8000613021F421E0FC0123AB0895FC0113AA7D
:102A90000895009719F0FC0183A9089580E0089536
:102AA0008F929F92AF92BF92DF92EF92FF920F931D
:102AB0001F93CF93DF934115510509F46BC08A0131
:102AC0007B01C82F0E9497C5D82F8C2F0E94B4C5B8
:102AD000D82EDD2309F460C0882309F45FC08D2F50
:102AE0000E947DC14B015C018D2D0E947DC1672B31
:102AF000682B692B39F4F80110821182128213823B
:102B000080E04DC09701280D391D032E000C440BA9
:102B1000550BC63050F4A0E1B7E20F94A854F80169
:102B2000608371838283938309C0A8EEB3E00F941E
:102B3000A854F80160837183828393838D2D0E9452
:102B40007DC19B01AC01F80160817181828193811B
:102B50000F946F5488279927DC01821B930BA40BD9
:102B6000B50BF80180839183A283B3838C2F0E94DD
:102B70005AC9F80180809180A280B380DC01CB012A
:102B8000880D991DAA1DBB1D80839183A283B383E9
:102B900081E005C080E003C080E001C080E0DF91FB
:102BA000CF911F910F91FF90EF90DF90BF90AF906A
:102BB0009F908F900895CF93DF93009709F460C0A2
:102BC000EC010F94FF18813091F58C830F9467010D
:102BD0008823F9F08091DD3E811119C089E0EAEE89
:102BE000F0E2A1E2B4E401900D928A95E1F7E1E20E
:102BF000F4E401900020E9F73197AF0141525444C9
:102C000021E061E274E48EE399E30F946A210F946A
:102C1000A0010F946A01882399F18FE098E40E9443
:102C2000A8CF0F9464018A830F94B10129C01C823C
:102C30000F942B198823F9F08091DD3E811119C082
:102C400089E0E3EFF0E2A1E2B4E401900D928A950D
:102C5000E1F7E1E2F4E401900020E9F73197AF01F8
:102C60004152544421E061E274E48EE399E30F940D
:102C70006A210F942E190F94171981110F941A19A4
:102C8000DF91CF9108950F931F93CF93DF93009718
:102C900009F463C0EC010F94761B882381F18B81CA
:102CA00081115BC08091DD3E811126C00F943F19D8
:102CB000182F0F9464011F921F931F928F9385E02A
:102CC00091E29F938F9301E214E41F930F930F946B
:102CD000B856F80101900020E9F73197AF01415251
:102CE000544420E0B8018EE399E30F946A218DB734
:102CF0009EB708968DBF9EBF81E08B832EC08B81CF
:102D0000813059F51B828091DD3E811126C00F94E0
:102D10003F19C82F0F9464011F92CF931F928F9376
:102D20008CEF90E29F938F93C1E2D4E4DF93CF9333
:102D30000F94B85609900020E9F72197AE0141524F
:102D4000544420E061E274E48EE399E30F946A2135
:102D50008DB79EB708968DBF9EBFDF91CF911F9113
:102D60000F910895CF92DF92EF92FF920F931F93EE
:102D7000CF93DF93009709F4AAC06115710509F498
:102D8000A6C08B01EC010E9446CF882309F49FC0A6
:102D90000F94BE196B017C010F94631B86E10E94A6
:102DA000A1C1AB01BC0187EB9CE30E94DCCFD70142
:102DB000C6010197A109B109883E9340A105B1055B
:102DC00008F03FC00E94B6B9823088F18091DD3EA4
:102DD00081112DC00F9464011F928F9380917B53BA
:102DE0001F928F93FF92EF92DF92CF9288E191E250
:102DF0009F938F930F2EF1E2EF2EF4E4FF2EF02D30
:102E0000FF92EF920F94B856F70101900020E9F776
:102E10003197AF014152544421E0B7018EE399E369
:102E20000F946A218DB79EB70C968DBF9EBF26E288
:102E300035E440E457E46AE776E4C8010E944FDBDA
:102E400043C0D701C601895E9340A109B109843608
:102E50009105A105B105C0F580E495E40E943ECF3F
:102E6000811132C08091DD3E811125C0FF92EF9229
:102E7000DF92CF9284E291E29F938F930F2EF1E243
:102E8000EF2EF4E4FF2EF02DFF92EF920F94B85640
:102E9000F70101900020E9F73197AF014152544406
:102EA00021E0B7018EE399E30F946A218DB79EB7B5
:102EB00008968DBF9EBF26E235E440E457E46AE7FA
:102EC00076E4C8010E944FDBCE010E945FCFDF9104
:102ED000CF911F910F91FF90EF90DF90CF900895C9
:102EE000FC01892B39F0118689E0DF011D928A955A
:102EF000E9F712860895FC01892B41F0118689E0DB
:102F0000DF011D928A95E9F71286138608950F93C3
:102F10001F93CF93DF93CFEDD8E307E319E3CE01FF
:102F2000DFDF2B96C017D107D1F783E79CE3E3DF00
:102F30008FE79CE3E0DF0F94DC1DDF91CF911F91C1
:102F40000F910895FC01892B31F081E09285913039
:102F500019F080E0089580E008951F93CF93DF93E8
:102F6000CDB7DEB76097CDBFDEBF9C01FE013196C5
:102F7000AE014F5E5F4F21933193255F3F4FE417C2
:102F8000F507C9F7892B31F110E010C0E12FF0E00F
:102F9000EE0FFF1F81E090E08C0F9D1FE80FF91FDF
:102FA00080819181CFDF8823D1F01F5F0F94631C54
:102FB000181760F382E00E94A1C16B3068F0809125
:102FC0007E3C882359F081E090918A3C911107C0A2
:102FD00080E005C080E003C081E001C080E0609631
:102FE000CDBFDEBFDF91CF911F910895CF92DF92C9
:102FF000EF92FF920F931F93CF93DF93CDB7DEB77E
:103000002597CDBFDEBF19821A821B821C82411513
:10301000510559F16A017B01182FCA0161DFAE0128
:103020004F5F5F4FB701812F3BDD8823C9F00981D6
:103030001A812B813C814BE0BE016B5F7F4FC60143
:103040000F94EE28F60101900020E9F73197EC1972
:10305000FD09D6011996EC93199781E01A968C9385
:1030600069817A818B819C8103C060E070E0CB0133
:103070002596CDBFDEBFDF91CF911F910F91FF90BD
:10308000EF90DF90CF9008958F929F92AF92BF9272
:10309000EF92FF920F931F93CF93DF930097A1F0CE
:1030A0006115710589F0142F7B01EC010F947206F4
:1030B0004B015C01113009F424D9950184014BE0E6
:1030C000B701CE010F944027DF91CF911F910F914F
:1030D000FF90EF90BF90AF909F908F900895AF9228
:1030E000BF92CF92DF92EF92FF920F931F93CF93F5
:1030F000DF93CDB7DEB76097CDBFDEBF8C01CE01C9
:1031000001967C014096F70161937193655F7F4F53
:10311000E817F907C9F70115110509F475C282E02E
:103120000E94A1C1D62E96E0D91206C0C8010F9404
:10313000AD1781116FC243C38FEF8D0D823030F414
:10314000C8010F94AD17811111C039C38FEE8D0DD9
:10315000823030F4C8010F94AD17811107C02FC31E
:10316000C8010F94AD17882309F429C380E2E0EF6A
:10317000FFE3DF011D928A95E9F780E1ECE4FBE3D0
:10318000DF011D928A95E9F78D2D90E0FC013197C2
:10319000E231F10508F03AC28827ED5EFE4F8F4F0D
:1031A0000D948B5458010F2EF0EFCF2EFFE3DF2E3E
:1031B000F02D01E010E00EC10F94AA17C82E49812E
:1031C0005A81F8016081718111DF0F2EF0EFEF2E2F
:1031D000FFE3FF2EF02DD7016D937D938D939C938C
:1031E00013974B815C81F801628173818C2DFEDE27
:1031F000D70114966D937D938D939C931797B2E0AE
:10320000DB1206C28091F03F9091F13FA091F23F16
:10321000B091F33F80934C3B90934D3BA0934E3B3A
:10322000B0934F3B81E0CBC258010F2EF0EFCF2E71
:10323000FFE3DF2EF02D01E010E00BC01F5F0F5FFA
:10324000E2E0EE0EF11CF2E0AF0EB11C84E0C80E1D
:10325000D11C112309F4FBC1123009F4EAC1D701D2
:103260004D915C91F5016081718180E0BFDED601F6
:103270006D937D938D939C9313970430F8F2809116
:10328000F03F9091F13FA091F23FB091F33F8093D6
:103290004C3B90934D3BA0934E3BB0934F3B81E012
:1032A0008EC258010F2EF0EFCF2EFFE3DF2EF02D50
:1032B00001E010E00BC01F5F0F5FB2E0EB0EF11CEE
:1032C000E2E0AE0EB11CF4E0CF0ED11C112309F4E4
:1032D000DBC1123009F4CAC1D7014D915C91F501EF
:1032E0006081718182E082DED6016D937D938D9342
:1032F0009C9313970430F8F2ECE4FBE3A0EFBFE3F8
:103300004D915D916D917C911397408351836283C0
:10331000738314968D919D910D90BC91A02D848303
:103320009583A683B78381E04AC258010F2EF0EF40
:10333000CF2EFFE3DF2EF02D01E010E00BC01F5F6A
:103340000F5FB2E0EB0EF11CE2E0AE0EB11CF4E058
:10335000CF0ED11C112309F4B8C1133009F4A3C155
:10336000113009F4A2C1143009F4A1C1D7014D9163
:103370005C91F5016081718180E038DED6016D934A
:103380007D938D939C9313970630C8F2ECE4FBE396
:10339000A0EFBFE34D915D916D917C9113974083B8
:1033A00051836283738314968D919D910D90BC918E
:1033B000A02D84839583A683B78381E000C21F5F1D
:1033C0000F5FB2E0EB0EF11CE2E0AE0EB11CF4E0D8
:1033D000CF0ED11C112309F487C1143009F492C116
:1033E000812F8B7F813009F48FC1823009F48EC127
:1033F000D7014D915C91F5016081718185E0F6DD29
:10340000D6016D937D938D939C9313970830B8F2FA
:10341000ECE4FBE3A0EFBFE34D915D916D917C91F6
:103420001397408351836283738314964D915D910A
:103430006D917C91179744835583668377831896A3
:103440004D915D916D917C911B974087518762876B
:1034500073871C968D919D910D90BC91A02D8487B2
:103460009587A687B78781E0AAC158010F2EF0EF94
:10347000CF2EFFE3DF2EF02D01E010E00BC01F5F29
:103480000F5FB2E0EB0EF11CE2E0AE0EB11CF4E017
:10349000CF0ED11C112309F458C1143009F445C1D1
:1034A000812F8B7F813009F442C1D7014D915C910E
:1034B000F5016081718180E099DDD6016D937D9386
:1034C0008D939C9313970830D0F2ECE4FBE3A0EFCC
:1034D000BFE34D915D916D917C9113974083518332
:1034E0006283738314968D919D910D90BC91A02D54
:1034F00084839583A683B78381E061C1680100EF6F
:103500001FE35E01B9E0AB0EB11CF701419151918F
:103510007F01D6016D917D916D0180E067DDF8013D
:1035200061937193819391938F01EA14FB0469F77E
:1035300081E045C158010F2EF0EFCF2EFFE3DF2EC3
:10354000F02D01E010E00BC01F5F0F5FF2E0EF0E07
:10355000F11C82E0A80EB11C94E0C90ED11C11230D
:1035600009F410C1133009F4FFC0D7014D915C91EB
:10357000F5016081718180E039DDD6016D937D9325
:103580008D939C9313970630F8F28091F03F9091C1
:10359000F13FA091F23FB091F33F80934C3B909369
:1035A0004D3BA0934E3BB0934F3B81E008C1580187
:1035B0000F2EF0EFCF2EFFE3DF2EF02D01E010E015
:1035C0000BC01F5F0F5FB2E0EB0EF11CE2E0AE0E2E
:1035D000B11CF4E0CF0ED11C112309F4E2C0D701D5
:1035E0004D915C91F5016081718181E0123009F4A7
:1035F00080E0FCDCD6016D937D938D939C931397B3
:103600000430F8F281E0DBC080E0D9C080E0D7C0B0
:1036100081E0D5C080E2E0EFFFE3DF011D928A95F3
:10362000E9F780E1ECE4FBE3DF011D928A95E9F71D
:10363000B9CDF70140815181D5016D917C9183E035
:10364000D5DCF6016083718382839383F7CDD70144
:103650004D915C91F5016081718183E0C7DCD601F9
:103660006D937D938D939C931397E8CDF7014081E3
:103670005181D5016D917C9183E0B8DCF6016083C6
:1036800071838283938317CED7014D915C91F501AD
:103690006081718183E0AADCD6016D937D938D9367
:1036A0009C93139708CE83E003C082E001C082E0C0
:1036B000F70140815181D5016D917C9197DCF60134
:1036C00060837183828393833ACED7014D915C915D
:1036D000F5016081718183E089DCD6016D937D9372
:1036E0008D939C9313972BCEF70140815181D50187
:1036F0006D917C9183E07ADCF60160837183828333
:1037000093835DCE83E003C082E001C084E0D701F3
:103710004D915C91F5016081718168DCD6016D93FA
:103720007D938D939C9313974ACE83E001C082E0F2
:10373000F70140815181D5016D917C9157DCF601F3
:1037400060837183828393839ACED7014D915C917C
:10375000F5016081718183E049DCD6016D937D9331
:103760008D939C9313978BCEF70140815181D501A6
:103770006D917C9183E03ADCF601608371838283F2
:103780009383E2CED7014D915C91F5016081718107
:1037900083E02CDCD6016D937D938D939C931397DE
:1037A000D3CEF70140815181D5016D917C9180E0AC
:1037B0001DDCF601608371838283938302CF609660
:1037C000CDBFDEBFDF91CF911F910F91FF90EF90A2
:1037D000DF90CF90BF90AF9008950F942415882369
:1037E00029F00F94351584E0809327060895CF9330
:1037F000DF93009799F1EC0188818130A8F0833044
:1038000018F0863019F010C0E8DF25C08091280636
:1038100082FD03C084E0809325060F94BE148823A4
:10382000D1F00F94CF1417C00F94BE14882399F0D1
:103830000F94CF1484E0809327060DC08D818111F1
:103840000DC00F940215882349F00F94131584E0DE
:103850008093270603C08881863081F7DF91CF915E
:1038600008950E9480D30F94431A20E137E240E08C
:1038700050E00F944D54672B682B692BE1F40E94A4
:1038800080D3813019F40C9494D208950E9480D38F
:10389000823021F481E00C9483D308950E9480D378
:1038A000833019F40C9489D508950E9480D3843014
:1038B00011F40C94DDD508950F931F93CF93DF93EC
:1038C0001F921F92CDB7DEB719821A820097B9F006
:1038D0008C010E94D75490E006969E012F5F3F4FC7
:1038E00043E060E0800F911F0F949F25882339F0FB
:1038F00049815A8160E070E080E00E948CC10F90A5
:103900000F90DF91CF911F910F9108959F92AF92E9
:10391000BF92CF92DF92EF92FF920F931F93CF93BC
:10392000DF931F92CDB7DEB7009709F44BC05C015F
:1039300082E00E94A1C1962E8501085D1F4FBE0145
:103940006F5F7F4FC8010E945EDF882391F0F50111
:10395000C0A4D1A4E2A4F3A489E00E94A1C1AB0158
:10396000BC010BEB18E42BEA38E489810F945E1A52
:1039700017C0BE016F5F7F4FC8010E94AAE8F50122
:10398000C0A4D1A4E2A4F3A489E00E94AFC1AB011A
:10399000BC010BEB18E42BEA38E489810F945E1A22
:1039A000FAE0F91558F4F50140A551A562A573A5F3
:1039B00083EA98E40F94431D81E005C00F94AD1D88
:1039C00081E001C080E00F90DF91CF911F910F91B6
:1039D000FF90EF90DF90CF90BF90AF909F900895B1
:1039E000CF92DF92EF92FF920F931F93CF93DF93CB
:1039F0001F92CDB7DEB7009779F18C01BE016F5FE2
:103A00007F4F88960E94A5EB882399F0F801C0A407
:103A1000D1A4E2A4F3A489E00E94A1C1AB01BC013E
:103A20000BEB18E42BEA38E489810F945E1A81E0ED
:103A300014C0F801C0A4D1A4E2A4F3A489E00E94B8
:103A4000AFC1AB01BC010BEB18E42BEA38E4898170
:103A50000F945E1A81E001C080E00F90DF91CF915A
:103A60001F910F91FF90EF90DF90CF90089589E123
:103A70000E94A1C1623059F482E00E94A1C1673066
:103A800041F0693031F0613021F081E0089580E04B
:103A9000089580E0089589E10F946207623059F437
:103AA00082E00F946207673041F0693031F0613095
:103AB00021F081E0089580E0089580E008953F922C
:103AC0004F925F926F927F928F929F92AF92BF922E
:103AD000CF92DF92EF92FF920F931F93CF93DF93DA
:103AE000CDB7DEB76497CDBFDEBFB82E8B017A01AC
:103AF00089E10E94A1C1A62E0115110509F472C227
:103B00008091DD3E882339F00F2EFEE3CF2EF9E3BE
:103B1000DF2EF02D06C00F2EF5E4CF2EFAE3DF2EB8
:103B2000F02D82E08A1508F4A12C8BE7F801808340
:103B300083E781838CE28283F2E3BF1207C082E3D2
:103B40008A0DF80183838CE284830BC0F801B38271
:103B50008CE28483F0E3BF1609F4F1C182E3B8126A
:103B600018C28FED98E3FE0132969E012E5E3F4F04
:103B7000819391930B962E173F07D1F788E08983A5
:103B8000E114F10469F086E0F701D801159601907F
:103B90000D928A95E1F70F2EFBE0FF2EF02D04C069
:103BA0000F2EF5E0FF2EF02DF801EF0DF11D8CE248
:103BB000808382E00E94A1C1762E872D072C000C05
:103BC000990B9F937F9281E291E29F938F93F3945D
:103BD000C8018F0D911D9F938F930F94B856F801D4
:103BE00001900020E9F73197E01BF10B7F01FF24E2
:103BF000F801EE0DFF1D118221E0A701B801C601F9
:103C00000F946A210F900F900F900F900F900F90CC
:103C10008091DD3E811112C01A8A21E040E050E01F
:103C2000BE016E5E7F4F8EE399E30F946A2120E020
:103C3000A701B8018EE399E30F946A2191E09A15E8
:103C400008F402C11982912C0F2EFCE28F2EF02D68
:103C5000F8013196EB8BFC8B0F2EFDED4F2EFEE322
:103C60005F2EF02D5BC00F94631C6980861509F4EC
:103C70005BC0F8018082E62CF12CF701EE0FFF1FEC
:103C800081E090E08C0F9D1FE80FF91FA180B280AA
:103C9000F501418550E0B5018B899C890F948A56C6
:103CA000F50181856894332431F8380E8F5FF8016F
:103CB000E80FF11D8082F7013196EE0FFF1F81E0C2
:103CC00090E08C0F9D1FE80FF91FA180B280F501D5
:103CD000418550E0B501C801830D911D0F948A56AE
:103CE000F501E1843E0C639463946982E32CF12C2A
:103CF000F801EE0DFF1D118221E0A701B801C601F8
:103D00000F946A21F2018081811107C020E0A70190
:103D1000B8018EE399E30F946A2193940F94631C86
:103D20008695981608F49FCFFAE0F7150CF0D8C0E6
:103D30008CE078164CF09DE097150CF050C180EFA8
:103D4000870D833008F44BC1198280E00F2EFCE20E
:103D50003F2EF02D4801EFEF8E1A9E0A0F2EFDED3B
:103D60004F2EFEE35F2EF02DF8013082E82EF12C6D
:103D7000F701EE0FFF1FEE0DFF1DEE0FFF1FEE0F01
:103D8000FF1FED58F34C82858C3419F0823541F0D9
:103D90000EC080E39CE2F4018083918312820FC005
:103DA00081E39CE2F40180839183128208C085E064
:103DB000E6E3F1E2D40101900D928A95E1F7F80172
:103DC00001900020E9F731975F01A01AB10A37018D
:103DD000660C771CB3016E0D7F1D660F771F660F93
:103DE000771F6D58734CFB01418550E0C8018A0D67
:103DF000911D0F948A56F301EE0DFF1DEE0FFF1F6C
:103E0000EE0FFF1FED58F34C8185A80EB12CF80181
:103E1000EA0DFB1D118221E0A501B801C6010F9436
:103E20006A21F2018081811107C020E0A501B8015B
:103E30008EE399E30F946A21E98081E08E0D8983F6
:103E4000823008F491CF4CC01982612C0F2EFCE215
:103E50005F2EF02D4801FFEF8F1A9F0A0F2EFDED08
:103E6000AF2EFEE3BF2EF02D36C00F94631C798079
:103E70008715B1F1F8015082E72DF0E0EE0FFF1F3A
:103E800081E090E08C0F9D1FE80FF91FE180F28028
:103E9000F701418550E0B701C4010F948A56F7013C
:103EA000E184E39473947982F12CF801EE0DFF1D07
:103EB000118221E0A701B801C6010F946A21F50122
:103EC0008081811107C020E0A701B8018EE399E34A
:103ED0000F946A2163940F94631C8695681628F2E8
:103EE0000F2EFCE2FF2EF02DF801F08284E00E94FC
:103EF000A1C1605DF8016183F28240E0BE016F5FA5
:103F00007F4FC8010396C0D8898193E0980FF801CC
:103F1000E90FF11D9DE790838C5FE82EF12CF801ED
:103F2000EE0DFF1D118221E0A701B801C6010F941B
:103F30006A218091DD3E882309F445C053C00F2ECD
:103F4000F9E7EF2EF6E4FF2EF02DF701408150E067
:103F500062E476E4C80105960F948A56F7018081E1
:103F600095E0980FF801E90FF11D9DE790838A5FB6
:103F7000E82EF12CF801EE0DFF1D118221E0A701C2
:103F8000B801C6010F946A218091DD3E81112AC0DB
:103F900011C021E045E050E0B801C6010F946A214C
:103FA0008091DD3E81111EC0F0E3BF120FC045E0DD
:103FB00050E002C04E2D5F2D20E0B8018EE399E362
:103FC0000F946A210FC04E2D5F2D02C045E050E0D6
:103FD00021E0B8018EE399E30F946A2103C081E0E8
:103FE0008983B4CE6496CDBFDEBFDF91CF911F91A0
:103FF0000F91FF90EF90DF90CF90BF90AF909F9088
:104000008F907F906F905F904F903F900895CF93E7
:10401000892B81F00E94E553CAE00E94A8540E94B7
:10402000E253882321F00E94F853811105C0C1504A
:10403000A1F703C0C0E001C0C1E08C2FCF9108956B
:1040400089E10E94A1C1611104C00F947B01882302
:1040500071F081E04091805350918153609182537F
:1040600070918353452B462B472B09F080E0089530
:104070008F929F92AF92BF92CF92DF92EF92FF9278
:104080000F931F93CF93DF930097A9F1EC0186E084
:104090000E94A1C14B015C0184E00E94A1C1162FC6
:1040A00087E00E94A1C1062F812F0F9456060F941E
:1040B00072066B017C0186169706A806B906D9F030
:1040C000AB01BC0186E00E94F5C68823A1F00F94E5
:1040D000FF05B701A60186E00E9497C1B701A601BE
:1040E00086E00F947507602F812F0F94560668E0C5
:1040F000CE010E943C14DF91CF911F910F91FF9050
:10410000EF90DF90CF90BF90AF909F908F900895E9
:1041100082E10E94A1C128E0E2EBF3E5DF01322F4A
:104120001D923A95E9F7EAEBF3E5DF011D922A9536
:10413000E9F721E030E0672B682B692B11F420E0D0
:1041400030E0F901E153FF4D80818560E8E7F3E558
:1041500082AF83AF81E00895009761F0613031F460
:10416000FC01EA5CFD4F21E020830895FC01EA5C3C
:10417000FD4F108208950097B1F0FC0180818430DA
:10418000A1F40F949619823039F089E10E94A1C1FF
:10419000672B682B692B59F00F94731991E08111EB
:1041A00007C090E005C090E003C090E001C090E03F
:1041B000892F08950F931F93CF93DF938C01EB0109
:1041C000209709F442C01882892B19F189E10E94D5
:1041D000A1C1F80180818130C0F0833018F08530B2
:1041E000D0F013C0611106C02097B9F087E488832E
:1041F00080E02EC06150623090F0209791F087E40B
:10420000888380E025C0209771F082E4888380E075
:104210001FC080E01DC081E01BC080E019C081E0AC
:1042200017C080E015C080E013C081E011C080E0BD
:104230000FC089E10E94A1C1F8018081813018F38B
:10424000833080F2853088F3DECF892B91F7EFCF72
:10425000DF91CF911F910F910895009739F0FC01E4
:1042600080818150843020F481E0089580E00895B9
:1042700080E00895009751F0FC018081813040F08A
:10428000843010F0853021F481E0089580E00895B5
:1042900080E00895CF92DF92EF92FF92CF93DF9369
:1042A000009709F45FC0EC0183E00E94A1C16B019B
:1042B0007C01AB01BC0155276627772783E00E946C
:1042C000F5C6882309F44BC08C2DFE01E95CFD4F37
:1042D000C082813021F1823009F044C088E00E9420
:1042E000A1C1FE01E75CFD4F6083AB01BC01552716
:1042F0006627772788E00E94F5C6811105C081E016
:10430000FE01E75CFD4F8083FE01E85CFD4F1082FB
:10431000C65CDD4F188219821A821B8223C087E097
:104320000E94A1C1F62E84E00E94A1C1862F6F2DAC
:104330000F94560685E00E94A1C10F940707FE0165
:10434000E25CFD4F60837183828393830F941F0629
:10435000C65CDD4F188219821A821B8203C0C95CB9
:10436000DD4F1882DF91CF91FF90EF90DF90CF90DB
:104370000895009761F1FC01E85CFD4F20813196C2
:104380003081321710F021111BC0FC01E85CFD4F99
:10439000315030833296408151816281738140383F
:1043A00021E5520721E06207710598F44F5F5F4FE6
:1043B0006F4F7F4F408351836283738381E0089501
:1043C000FC01E85CFD4F2150208380E0089580E0EF
:1043D000089580E008950F931F93CF93DF93009784
:1043E00041F1EC010F943606FE01E25CFD4F0081C5
:1043F0001181228133816017710782079307D8F0FA
:104400000F941F06FE01E65CFD4F80819181A28121
:10441000B381803821E5920721E0A207B10568F455
:104420000196A11DB11D80839183A283B38381E096
:1044300005C080E003C080E001C080E0DF91CF9143
:104440001F910F910895CF93DF93009709F43DC01A
:10445000FC01EA5CFD4F20812223B9F1EC018BDEE7
:10446000813021F4CA5CDD4F18822FC089E10E949F
:10447000A1C161111AC00F949619813031F18230B7
:1044800089F4DEDD882309F10F945019CA5CDD4FF1
:10449000188280E495E40E9438CF8FE098E40E946F
:1044A0005FCF13C00F94841910C0CADD882369F050
:1044B0000F945019CA5CDD4F188280E495E40E9485
:1044C00038CF8FE098E40E945FCFDF91CF910895BD
:1044D000FF920F931F93CF93DF936115710509F43A
:1044E0007CC04115510509F478C08A01EB01F82E12
:1044F00082E10F94620721E0672B682B692B09F496
:1045000020E08F2D90E0FC013197E231F10508F0B9
:104510005BC08827EB5DFE4F8F4F0D948B54188244
:10452000E22FF0E0E153FF4D80818560F801808348
:1045300054C083E08883E22FF0E0E153FF4D808197
:10454000F80180834AC01882E22FF0E0E153FF4D6A
:1045500080818160F801808340C083E08883E22FFE
:10456000F0E0E153FF4D8081F801808336C018826E
:10457000E22FF0E0E153FF4D80818160F8018083FC
:104580002CC083E08883E22FF0E0E153FF4D80816F
:10459000F801808322C0188285E0F80180831DC065
:1045A000188281E0F801808318C01882E22FF0E0C1
:1045B000E153FF4D80818160F80180830EC0188235
:1045C00081E0F801808309C01882E22FF0E0E15316
:1045D000FF4D80818560F8018083DF91CF911F912D
:1045E0000F91FF9008958F929F92AF92BF92CF92BA
:1045F000DF92EF92FF920F931F93CF93DF93892B5C
:1046000009F486C089E00E94A1C19B01AC01A8EE1B
:10461000B3E00F94A8546B017C010F94A719C61640
:10462000D706E806F90609F475C0C701B60128EEF9
:1046300033E040E050E00F944D54F22ED22F2E3153
:1046400008F06AC0213009F469C00F94A71928EE58
:1046500033E040E050E00F944D54822FF21638F4CE
:104660006F2D0F941A54C92F992309F45CC00F942D
:104670003F19E82E6D2F0F941A54D92F892F90E0EF
:104680008E0D911DCA970CF04BC08D2E912CA12C34
:10469000B12C0F94BE19162F072FD82EC92EA8EEB5
:1046A000B3E0A50194010F94A8544F2D0F94EC1979
:1046B000C091DD3EC11136C00F94BE199F938F93F8
:1046C0007F936F93CF92DF920F931F931F92DF938D
:1046D0001F92EF928BE391E29F938F9301E214E498
:1046E0001F930F930F94B856F80101900020E9F73B
:1046F0003197AF014152544421E0B8018EE399E370
:104700000F946A218DB79EB740968DBF9EBF0BC098
:10471000C0E009C0C0E007C0C1E005C0C0E003C000
:10472000C1E001C0C0E08C2FDF91CF911F910F91AC
:10473000FF90EF90DF90CF90BF90AF909F908F90C1
:104740000895EF92FF920F931F93CF93DF932091E1
:10475000DD3E222339F00F2EFEE3EF2EF9E3FF2E8C
:10476000F02D06C00F2EF5E4EF2EFAE3FF2EF02D0C
:104770000097D1F1EC018BE7888388E689838CE28E
:104780008A8392E69B838C837F936F9386E791E283
:104790009F938F93CE0105969F938F930F94B85656
:1047A000FE0101900020E9F73197EC1BFD0B8F0112
:1047B000112721E0A801BE01C7010F946A210E94C0
:1047C000B6B90F900F900F900F900F900F90873009
:1047D00059F48091DD3E811107C021E0A801BE019E
:1047E0008EE399E30F946A21DF91CF911F910F918E
:1047F000FF90EF9008958F929F92AF92BF92CF92C9
:10480000DF92EF92FF920F931F93CF93DF93009766
:1048100009F470C02091DD3E222339F00F2EFEE313
:10482000EF2EF9E3FF2EF02D06C00F2EF5E4EF2E4C
:10483000FAE3FF2EF02DEC018BE7888388E689836D
:104840008CE28A8393E79B838C830BE81CE3F8015B
:10485000848C0E94FDA0982EA090DC3EB090D93EA2
:10486000F801C280D0800F947B011F928F921F921B
:104870009F921F92AF921F92BF921F92CF921F9250
:10488000DF921F928F93F80185811F928F9384810D
:104890001F928F9383811F928F938BE591E29F9359
:1048A0008F93CE0105969F938F930F94B856FE0178
:1048B00001900020E9F73197EC1BFD0B8F011127C8
:1048C00021E0A801BE01C7010F946A218DB79EB7F0
:1048D00048968DBF9EBF8091DD3E81110BC0A8011F
:1048E00042505109BE016F5F7F4F21E08EE399E393
:1048F0000F946A21DF91CF911F910F91FF90EF905C
:10490000DF90CF90BF90AF909F908F900895DF92EF
:10491000EF92FF920F931F93CF93DF9300D01F92DC
:10492000CDB7DEB78C010F944615882349F00F945C
:1049300057150E94A30F86EC92E45DDF80E066C00D
:10494000CE0101960E94AC0F882309F45FC0F0905D
:10495000A806E0906806D0902806BE016D5F7F4FE4
:10496000CE0101960E94C20F882309F44CC00E9418
:10497000C2B98823C9F18091DD3E811135C0D0FADA
:10498000DD24D0F81F92DF92E4FAEE24E0F81F92C3
:10499000EF92F6FAFF24F0F81F92FF928A818F932C
:1049A00089818F938C818F938B818F938AE791E29A
:1049B0009F938F930F2EF1E2EF2EF4E4FF2EF02D54
:1049C000FF92EF920F94B856F70101900020E9F79B
:1049D0003197AF014152544421E0B7018EE399E38E
:1049E0000F946A21CDBFDEBF6B817C8186EC92E49F
:1049F000A8DE0115110549F08B819C81F8018083A7
:104A0000918381E003C081E001C081E02496CDBFA5
:104A1000DEBFDF91CF911F910F91FF90EF90DF905C
:104A20000895882321F081E08093DC3E0895109260
:104A3000DC3E08950F931F93CF93DF9361157105AB
:104A400071F0009761F0EB018C010F9468158823D9
:104A500031F00F947915BE01C8010E94698EDF9173
:104A6000CF911F910F910895CF93DF93009751F04D
:104A7000EC010F94B415882329F0CE010E94AB906D
:104A80000F94C515DF91CF910895009791F0FC0127
:104A9000EC5BFD4F2FEF3FE720833183329620E020
:104AA00030E8208331833296108211823296108250
:104AB000118208950F93CF93DF930097A1F066239F
:104AC00071F0EA01FC01E45BFD4F81E08083C901E4
:104AD0000F94B51B602FCE010E94A2A204C0FC015E
:104AE000E45BFD4F1082DF91CF910F910895EF921B
:104AF000FF920F931F93CF93DF931F921F92CDB717
:104B0000DEB7009709F498C06115710509F494C0E7
:104B1000FC0122A9211104C023A9222309F48CC07D
:104B20008B017C01FC0112AA13AA0E94FF100E94B3
:104B30008A110E948313F70144A955A9B7016A5C41
:104B40007F4F9E012F5F3F4FC8010F94AF4AC801AE
:104B50000F945D4CF701E75AFD4FD701AD5ABD4F99
:104B60008C918083319611968C9180830F94BE191D
:104B70009F938F937F936F9389E991E29F938F9394
:104B800001E214E41F930F930F94B856F8010190BB
:104B90000020E9F73197AF014152544421E0B801B8
:104BA0008EE399E30F946A21CDBFDEBFF70124A9FC
:104BB00035A989819A812817390719F1C701069605
:104BC0009F938F9385EA91E29F938F931F930F9307
:104BD0000F94B856F80101900020E9F73197AF0122
:104BE0004152544421E0B8018EE399E30F946A21C5
:104BF0000E944FA30F900F900F900F900F900F9067
:104C000002C00E94DFA2E2E0F3E4808190E0DC01D8
:104C1000AE5FBC4B25853685880F991FFC01EE5F82
:104C2000FC4B418152811F960C9161E0C70142DF2C
:104C30000E940F930F941B1C0F900F90DF91CF9148
:104C40001F910F91FF90EF9008950F931F93CF93B3
:104C5000DF93009709F448C06115710509F444C059
:104C60008B01EC01FC01E45BFD4F80818823C1F1E5
:104C7000DB018C91882341F10F94D11B8823A1F192
:104C8000F801608161506083611108C00E9414A323
:104C90000E9401A3C45BDD4F188226C070E0F801BA
:104CA000E60FF71FD8011D962D913C911E97660FB8
:104CB000771FA60FB71F11964D915C91129707852C
:104CC00061E0CE01F7DE10C00F94D11B882361F0A4
:104CD0000E9414A30E9401A3C45BDD4F188204C08C
:104CE0000E9414A30E9401A3DF91CF911F910F9105
:104CF00008958F929F92BF92CF92DF92FF920F936F
:104D00001F93CF93DF93009709F4DAC06115710503
:104D100009F4D6C02091DD3E222309F4C0C0CEE3C1
:104D2000D9E3BFC08B014C010E946211B82E0E94D2
:104D3000E211D82E0E94BD10C82E8D2D90E08B0D53
:104D4000911D8C0D911D892B71F4F401E35BFD4FD6
:104D50008081813009F4B4C081E0808380E090E0FC
:104D60000F94E81BADC0F401E35BFD4F80818230FE
:104D700009F43EC0BB2051F00E945F11811108C0B0
:104D800061E0CE010E94E79201E003C000E001C0B3
:104D900000E0CC2009F48AC00E94BA10811186C0BC
:104DA00063E0CE010E94E79201E080C0DD2081F047
:104DB000812F0E94C213882359F0812F0E94D213A1
:104DC000811106C064E0610FCE010E94E79201E00C
:104DD0001F5F143059F7002309F472C0E401C35B6C
:104DE000DD4F82E0888384EF91E00F94E81B68C078
:104DF0000F94041C882309F463C0BB2009F45DC030
:104E00000E945F11811159C00E9466A3CC2009F451
:104E10004FC0FF24F39401C0F12C0E94BA108111FD
:104E200049C00E9466A316C0D0E0C0E0DD2069F052
:104E30008D2F0E94C213882341F08D2F0E94D21320
:104E4000811103C00E9464A3C1E0DF5FD43071F719
:104E5000CC23E1F084EF91E00F94E81BD8018C9112
:104E600090E0F801E80FF91F1D962D913C911E97D7
:104E7000880F991FA80FB91F11964D915C91129739
:104E8000078561E08BE89CE315DE1AC0F401E35B63
:104E9000FD4F80818230A1F481E0808311C0C5E4A0
:104EA000DAE3FC012081243059F43CCF10E07ECFBE
:104EB000FF24F394F110CECFB7CFC110ADCFB4CF54
:104EC000DF91CF911F910F91FF90DF90CF90BF9016
:104ED0009F908F900895009721F0FC01E35BFD4FB8
:104EE00060830895CF93DF930097C1F0EC0119829E
:104EF00018820E944B1D813031F482E0888389E161
:104F0000898391E006C0CE010E94D8EC91E0811126
:104F100090E081E0992319F080E001C080E0DF910A
:104F2000CF910895CF93892B09F44CC082E00E9461
:104F3000A1C1862F90E0FC013297E031F10508F025
:104F400043C08827E95CFE4F8F4F0D948B5440E09F
:104F500050E0BA0180E00E942CC937C040E050E028
:104F6000BA0180E00E942CC9C82F40E050E0BA018D
:104F700081E00E942CC9C80F81E0C23031F180E08D
:104F800024C040E050E0BA0180E00E942CC9C82F44
:104F900040E050E0BA0181E00E942CC9C80F40E017
:104FA00050E0BA0182E00E942CC9C80F40E050E0F6
:104FB000BA0183E00E942CC9C80F81E0C43029F0F7
:104FC00080E003C080E001C080E0CF910895CF92DF
:104FD000DF92EF92FF92843098F4E82FF0E0EE0F2A
:104FE000FF1FEE0FFF1FE45BF44CC080D180E28016
:104FF000F3800E94FCC86C197D098E099F0903C0CB
:1050000060E070E0CB01FF90EF90DF90CF900895CB
:10501000CF93892B09F453C082E00E94A1C1862F4F
:1050200090E0FC013297E031F10508F04AC0882792
:10503000E95BFE4F8F4F0D948B5480E0C8DFAB01CE
:10504000BC0180E00E942CC93DC080E0C0DFAB0104
:10505000BC0180E00E942CC9C82F81E0B8DFAB0101
:10506000BC0181E00E942CC9C80F81E0C23051F11F
:1050700080E028C080E0ABDFAB01BC0180E00E9493
:105080002CC9C82F81E0A3DFAB01BC0181E00E94E5
:105090002CC9C80F82E09BDFAB01BC0182E00E94FB
:1050A0002CC9C80F83E093DFAB01BC0183E00E94F1
:1050B0002CC9C80F81E0C43029F080E003C080E033
:1050C00001C080E0CF91089590E0FC013397EE306D
:1050D000F10508F0A7C08827E95AFE4F8F4F0D94BD
:1050E0008B54E8E7F3E5868D978DA0A1B1A1428DA1
:1050F000538D648D758D841B950BA60BB70B86396C
:105100009105A105B10508F48FC046A157A160A57E
:1051100071A582A193A1A4A1B5A1481B590B6A0B4B
:105120007B0B81E0463951056105710508F483C0A8
:1051300080E00895E8E7F3E582A193A1A4A1B5A1D9
:10514000468D578D60A171A1841B950BA60BB70BE3
:1051500086399105A105B10508F468C046A557A593
:1051600060A971A982A593A5A4A5B5A5481B590B53
:105170006A0B7B0B81E0463951056105710508F426
:105180005AC080E00895E8E7F3E582A193A1A4A1C5
:10519000B5A1468D578D60A171A1841B950BA60BFF
:1051A000B70B86399105A105B10508F441C042A9A4
:1051B00053A964A975A986A597A5A0A9B1A9481B5B
:1051C000590B6A0B7B0B81E046395105610571056E
:1051D00090F180E00895E8E7F3E5868D978DA0A132
:1051E000B1A1428D538D648D758D841B950BA60BDB
:1051F000B70B86399105A105B105E0F042A553A58D
:1052000064A575A586A197A1A0A5B1A5481B590BBA
:105210006A0B7B0B81E0463951056105710558F039
:1052200080E0089580E0089581E0089581E0089588
:1052300081E0089581E00895CF9382E10E94A1C1A9
:10524000C1E0672B682B692B09F4C0E082E00E9463
:10525000A1C188E0E2EBF3E5DF01982F1D929A955A
:10526000E9F7EAEBF3E5DF011D928A95E9F7862F6E
:1052700090E0FC013197E231F10508F0EFC088279A
:10528000EB59FE4F8F4F0D948B54EC2FF0E0E15310
:10529000FF4D80818560E8E7F3E582AF83AFE8C02A
:1052A000EC2FF0E0E153FF4D8081E8E7F3E582AFBA
:1052B00083AF83E08093BA538093BB53D9C0862FCA
:1052C00003DFEC2FF0E0E153FF4D908121E08111ED
:1052D00001C020E0822F892BE8E7F3E582AF84AF9D
:1052E00083E08093BA538093BC53892F816083AF4E
:1052F00085AFBEC0EC2FF0E0E153FF4D8081E8E7C1
:10530000F3E582AF84AF93E09093BA539093BC538C
:1053100083AF85AF82E08093BB538093BD53A8C019
:10532000862FD2DEEC2FF0E0E153FF4D208191E09B
:10533000811101C090E0892F822BE8E7F3E582AF6D
:1053400085AF93E09093BA539093BD5383AF86AFEC
:1053500082E08093BB538093BE53822F816084AFE1
:1053600087AF86C0EC2FF0E0E153FF4D8081E8E786
:10537000F3E582AF86AF93E09093BA539093BE5318
:1053800083AF87AF92E09093BB539093BF5384AFAA
:105390008093B85394E09093BC539093C05385AFDF
:1053A0008093B95385E08093BD538093C15360C00F
:1053B000862F8ADE91E0811101C090E0892F8F70E5
:1053C000E8E7F3E582AF86AF93E09093BA5390930A
:1053D000BE5383AF87AF82E08093BB538093BF53AC
:1053E00081E084AF8093B85395AF9093B95340C098
:1053F000E8E7F3E585E082AF84AF87E083AF85AF70
:1054000037C0862F61DE91E0811101C090E0EC2F62
:10541000F0E0E153FF4D8081892BE8E7F3E582AFAF
:1054200085AF83E08093BA538093BD5391E093AFEF
:1054300096AF84AF87AF1CC0EC2FF0E0E153FF4D77
:1054400080818160E8E7F3E582AF84AF83AF85AF09
:1054500081E08093BB538093BD530AC0EC2FF0E0F2
:10546000E153FF4D80818560E8E7F3E582AF83AFCC
:105470008091B25384700F947F0581E0CF9108959D
:105480001F93CF93DF930097E9F1EC011AAA1BAAAF
:105490000E94871787E00E94A1C1162F84E00E9416
:1054A000A1C1862F612F0F94560689E10E94A1C1E8
:1054B000613071058105910521F481E00F94D519C2
:1054C00003C080E00F94D5190E94371D813031F45C
:1054D000CE010E94F01C0E94882004C0CE010E94D0
:1054E000861CAADE0F94661C0F946205CE010E94F2
:1054F0004A210F94F11A0E94EE0F0E943F110E9460
:10550000BE111982DF91CF911F910895CF93DF9340
:10551000009791F0FC012081243071F4EC010E948D
:105520003820CE01ADDF0F9462191092D83E63E0AF
:10553000CE010E943C141982DF91CF9108958823F7
:1055400021F081E08093DD3E08951092DD3E0895C4
:105550008091DD3E0895AF92BF92CF92DF92EF929D
:10556000FF920F931F93CF93DF93DC01009709F411
:105570005AC04115510509F458C02115310509F4E7
:1055800056C0FA01C081D0E0F901008110E0611538
:10559000710561F0FC017C01E60EF71E9191C90FC7
:1055A000D11D0C0F1D1FEE16FF06C1F7F9017B017F
:1055B0006D01DA01CC930083F601E60FF71F8CE250
:1055C00080838BE181835B01A2E0AA0EB11CAC0C4D
:1055D000BD1C8C2F82958F700F948225F5018083DE
:1055E0005701F3E0AF0EB11CAC0CBD1C8C2F8F70BB
:1055F0000F948225D5018C93E7012496CC0DDD1DF7
:10560000802F82958F700F9482258883D7011596FD
:10561000E601CA0FDB1F802F8F700F9482258883CD
:10562000C701069605C0CB0103C0CB0101C0CB0169
:10563000DF91CF911F910F91FF90EF90DF90CF906E
:10564000BF90AF9008953F924F925F926F927F927A
:105650008F929F92AF92BF92CF92DF92EF92FF9282
:105660000F931F93CF93DF93CDB7DEB76397CDBF73
:10567000DEBF7C016B013A01290189E10E94A1C1D1
:10568000B62E82E00E94A1C1162FE114F10409F4A4
:1056900046C1C114D10409F444C16B3008F449C1B6
:1056A0006114710409F43FC14114510409F43DC16E
:1056B000FE013296CE014296C192D1922BE0C20EEB
:1056C000D11CE817F907C1F78DE0D701D6968C9366
:1056D000D69782E090E0D4968D939C93D5978AE0FC
:1056E000D7968C93F701F896EA8BFB8B41E0BE01CD
:1056F0006F5F7F4FCF010E9444182981D701D49654
:105700008D919C91D597820F911D9C012F5F3F4FEA
:10571000D4962D933C93D597F701E80FF91F2CE20F
:1057200026ABB1E0BB1590F5B12C0F2EFCE2AF2EED
:10573000F02D61C0EB2DF0E0EE0FFF1F81E090E057
:105740008C0F9D1FE80FF91FC180D280D701D4961E
:105750008D919C91D597C696F601418550E0B60192
:105760008E0D9F1D0F948A56D60119962C91F70124
:1057700084A995A9820F911D9C012F5F3F4F24ABF7
:1057800035ABE80FF91FA6AAB39405C0B12C0F2EB4
:10579000FCE2AF2EF02D0F94631CB81658F230C007
:1057A000EB2DF0E0EE0FFF1F81E090E08C0F9D1FCE
:1057B000E80FF91FC180D280D701D4968D919C91BA
:1057C000D597C696F601418550E0B6018E0D9F1D16
:1057D0000F948A56D60119962C91F70184A995A9A0
:1057E000820F911D9C012F5F3F4F24AB35ABE80F1B
:1057F000F91FA6AAB3940F94631C8695B81680F27D
:105800001B3008F466C01C3028F01E3028F0105100
:10581000133010F010E001C011E00F2EFAEB8F2EC4
:10582000F1E29F2EF02D5701F6E3AF0EB11C0F2EC3
:10583000FCE23F2EF02DC12ED12CC601880F991FFE
:10584000C80ED91ECC0CDD1CCC0CDD1CC60CD71C24
:10585000D6011A968C911F928F939F928F92F70187
:1058600084A995A9C6968E0D9F1D9F938F930F9423
:10587000B856F50101900020E9F73197EA19FB09C4
:10588000D701D496ED93FC93D597CF01C696F60138
:10589000418550E0B6018E0D9F1D0F948A56D601AA
:1058A00019962C91F70184A995A9820F911D9C014D
:1058B0002F5F3F4F24AB35ABE80FF91F36AA1F5FB0
:1058C0000F900F900F900F900F900F90123008F4E0
:1058D000B2CF0130D9F4D701D4968D919C91D59750
:1058E000C696820101501F4FF801408150E0B2017D
:1058F0008E0D9F1D0F948A56D8012C91F70184A913
:1059000095A9820F911D84AB95AB18C0D701D49691
:10591000ED91FC91D597EE0DFF1D16AA0FC080E00A
:105920002EC080E02CC080E02AC080E028C080E04B
:1059300026C04114510409F0BBCEF9CFA7014D5A3E
:105940005D4FF701E75AFD4F8081FA01808397018F
:105950002C5A3D4F37968081D9018C93F70164A969
:1059600075A9625071098A899B89F5DD0296D70174
:10597000D4968D939C93D59781E0D2968C93639621
:10598000CDBFDEBFDF91CF911F910F91FF90EF90C0
:10599000DF90CF90BF90AF909F908F907F906F904F
:1059A0005F904F903F9008952F923F924F925F9259
:1059B0006F927F928F929F92AF92BF92CF92DF921F
:1059C000EF92FF920F93CF93DF93CDB7DEB760973F
:1059D000CDBFDEBF009709F46EC06115710509F4F3
:1059E0006AC09B01FE013196DE01519621933193ED
:1059F000255F3F4FEA17FB07C9F76A017B011C01CE
:105A0000B12C12C0EB2DF0E0EE0FFF1F81E090E013
:105A10008C0F9D1FE80FF91F808191810E94A217B2
:105A2000882309F448C0B3940F94631CB81650F34C
:105A30000F94BE194B015C010F94A7192B013C0177
:105A400080E495E40E943ECF082F81110BC09EE1B7
:105A5000890E911CA11CB11C84149504A604B704E2
:105A600050F115C040E050E066EC72E480E30E9423
:105A70005F1D20E435E4A601B701C101E4DD42E485
:105A800056E466EC72E482E30E945F1D0EC000E003
:105A900020E435E4A601B701C101D5DD40E050E0C6
:105AA00066EC72E482E30E945F1D80E495E40E944C
:105AB00038CF0E9487176096CDBFDEBFDF91CF91B0
:105AC0000F91FF90EF90DF90CF90BF90AF909F909D
:105AD0008F907F906F905F904F903F902F900895A0
:105AE000009789F06115710571F04115510559F064
:105AF0002115310541F0FC011082FB011082FA01F1
:105B00001082F901108208952F923F924F925F9276
:105B10006F927F928F929F92AF92BF92CF92DF92BD
:105B2000EF92FF920F931F93CF93DF93CDB7DEB722
:105B30002597CDBFDEBF009709F461C0411551051F
:105B400009F45FC02115310509F45DC0613BE4E053
:105B50007E0708F45AC02B01E0EB4E1AE4E05E0A1F
:105B6000612C712CE2E04E165104610471040CF4B6
:105B700054C02C833D831A018C01C12CD12C760199
:105B8000C3944B01A12CB12CB501A4014C195D09A2
:105B90006E097F09C8010F94AF4C9E012F5F3F4FE4
:105BA00041E050E0BE016D5F7F4FC8010F94634933
:105BB00081112DC08B818B3191F18FEFC81AD80ADA
:105BC000E80AF80AC414D504E604F704ECF225C088
:105BD00089819A810497E8F0B10181E294E40F94FD
:105BE0007429982F882341F16C817D8183E294E4AC
:105BF0000F94742991E081111FC090E01DC090E0C6
:105C00001BC090E019C090E017C090E015C090E074
:105C100013C090E011C090E00FC090E00DC09E0155
:105C20002F5F3F4F44E050E061E274E4C8010F94FD
:105C30006349882369F2EFCF892F2596CDBFDEBF58
:105C4000DF91CF911F910F91FF90EF90DF90CF9058
:105C5000BF90AF909F908F907F906F905F904F908C
:105C60003F902F9008950097A9F061157105B1F04C
:105C7000FC019C01260F371F60E070E0CB014191D1
:105C80004D3021F46F5F7F4F8F4F9F4F2E173F078F
:105C9000B1F7089560E070E0CB01089560E070E036
:105CA000CB0108952F923F924F925F926F927F9215
:105CB0008F929F92AF92BF92CF92DF92EF92FF921C
:105CC0000F931F93CF93DF9300D01F92CDB7DEB712
:105CD000009709F455C00115110509F453C0613B43
:105CE0007440C0F4F801108211821282138280E0A5
:105CF0004CC009811A81B801C101B5DF460E571E9B
:105D0000681E791E0815190500F1C00ED11EE11C90
:105D1000F11C0BC00B831C8349011A015C01C12CCF
:105D2000D12C7601412C512C3201B701A601C501BD
:105D30000F94AF4C9E012F5F3F4FA401B101C501ED
:105D40000F9463498823A9F21FC0F6E24F1651044D
:105D50006104710440F4EB81FC8110821182128293
:105D6000138281E012C0F5E24F1A510861087108F0
:105D7000EB81FC81408251826282738281E005C0A6
:105D800080E003C080E001C080E02496CDBFDEBF8C
:105D9000DF91CF911F910F91FF90EF90DF90CF9007
:105DA000BF90AF909F908F907F906F905F904F903B
:105DB0003F902F900895009741F0FC01EB5AFD4F62
:105DC0006081718182819381089560E070E0CB01F0
:105DD0000895009739F0FC01EB5AFD4F10821182B3
:105DE000128213820895CF93DF93009781F120915F
:105DF000DD3E21112CC0EC010F944E16882339F1A1
:105E0000CE010E944B970F9427160F9464011F92A6
:105E10008F938EEB91E29F938F93C1E2D4E4DF9353
:105E2000CF930F94B85609900020E9F72197AE015F
:105E30004152544420E061E274E48EE399E30F940C
:105E40006A210F900F900F900F900F900F90DF919D
:105E5000CF9108952115310551F05058610971090C
:105E6000F901408351836283738381E0089580E068
:105E70000895009719F0FC01848D089580E008953D
:105E80004F925F926F927F928F929F92AF92BF924A
:105E9000EF92FF920F931F93CF93DF931F92CDB793
:105EA000DEB7E114F10409F465C0480159012A0183
:105EB0003B01182FC7010E947B17143031F484E195
:105EC0000E947DC19B01AC0105C085E10E947DC19E
:105ED0009B01AC012115310541055105F9F08418EC
:105EE0009508A608B708880C991CAA1CBB1CD501EC
:105EF000C401880F991FAA1FBB1F880F991FAA1FD3
:105F0000BB1FBC01CD01680D791D8A1D9B1D0F941F
:105F10006F54822E932EA42EB52E0EC088248A9400
:105F20000F2EF0EE9F2EF02D0F2EF5EFAF2EF02D51
:105F30000F2EF5E0BF2EF02D082D192D2A2D3B2D0B
:105F40004BE0BE016F5F7F4FC7010F94EE28F70152
:105F500001900020E9F73197EE19FF09D701199652
:105F6000EC93199781E01B968C93682D792D8A2DDF
:105F70009B2D04C060E070E080E090E00F90DF9126
:105F8000CF911F910F91FF90EF90BF90AF909F9096
:105F90008F907F906F905F904F9008952F923F92D7
:105FA0004F925F926F927F928F929F92AF92BF9229
:105FB000CF92DF92EF92FF920F931F93CF93DF93D5
:105FC000CDB7DEB72A97CDBFDEBFC501611571051C
:105FD00009F402C14115510509F400C1E114F104AD
:105FE00009F4FEC0802E912EA22EB32E25EB821630
:105FF0009104A104B10438F00F2EF4EB8F2E912CF4
:10600000A12CB12CF02D8B839C83CD82DE82EF827C
:10601000F88649835A838B01FB01E453FD4F80814D
:106020009181A281B381892B8A2B8B2B81F53497A7
:1060300080819181A281B38180324EE49407A105D1
:10604000B1052CF1349680839183A283B383BF93EF
:10605000AF939F938F9389ED91E29F938F9381E20A
:1060600094E49F938F930F94B856E1E2F4E4019087
:106070000020E9F73197AF014152544420E061E23A
:1060800074E48EE399E30F946A21CDBFDEBFD8019B
:10609000CD90DD90ED90FC90B0E8DB1AE108F108BE
:1060A000F801C082D182E282F38281E08093633280
:1060B000F2E08F169104A104B10408F46FC0F80156
:1060C00063E672E321E0821A20EC920A880C991CA4
:1060D000880C991C1801280C391C4601570100E056
:1060E00010E0980169877A874481558166817781BC
:1060F0002A013B0180E8581A6108710844825582E0
:10610000668277824191519161917191441A550A49
:10611000660A770A141415041604170434F481E08F
:10612000A985BA8511968C9304C0A985BA85119664
:106130001C92A985BA8511965C901197CD010196A4
:1061400089879A879C91591691F0D801AA0FBB1F95
:10615000AA0FBB1F89819A81A80FB91F4D935D9328
:106160006D937C9313970F5F1F4F2F4F3F4F4081CD
:10617000518162817381C416D506E606F70614F4D0
:106180006A017B01481559056A057B0514F44A012B
:106190005B01E215F30509F0A7CF05C046015701E1
:1061A00000E010E09801AF81B8850D931D932D9309
:1061B0003C931397ED81FE81309721F0808291828C
:1061C000A282B382EB81FC81309761F0C082D182E0
:1061D000E282F38281E007C080E005C080E003C076
:1061E00080E001C081E02A96CDBFDEBFDF91CF9174
:1061F0001F910F91FF90EF90DF90CF90BF90AF90E5
:106200009F908F907F906F905F904F903F902F90D6
:1062100008958F929F92AF92BF92CF92DF92EF92AA
:10622000FF920F931F93FC01892BA1F1611571055A
:1062300099F1008111812281338184819581A68128
:10624000B781081719072A073B0744F5C084D18492
:10625000E284F384C816D906EA06FB060CF58484AA
:106260009584A684B784C814D904EA04FB04D4F442
:1062700088159905AA05BB05BCF40C151D052E054E
:106280003F0524F481E0FB0180830FC0FB011082F5
:1062900081E00BC080E009C080E007C080E005C05D
:1062A00080E003C080E001C080E01F910F91FF906B
:1062B000EF90DF90CF90BF90AF909F908F90089518
:1062C0003F924F925F926F927F928F929F92AF9286
:1062D000BF92CF92DF92EF92FF920F931F93CF93D3
:1062E000DF93009709F448C02115310509F446C031
:1062F000443051056105710508F442C06A017B0113
:10630000E4E0CE1AD108E108F108E1F159018C016D
:10631000912C312C812C412C512C3201E501C90DDD
:10632000D11DBE01C201880F991F880F991F800FD0
:10633000911F6FDF882379F08881882311F083947F
:1063400001C0339483E0480E511C611C711C93946E
:10635000E2E0E91550F08FEF481A580A680A780A07
:106360004C145D046E047F04C8F2882069F081E05B
:10637000332059F080E009C080E007C080E005C00C
:1063800080E003C081E001C081E0DF91CF911F91E7
:106390000F91FF90EF90DF90CF90BF90AF909F90C4
:1063A0008F907F906F905F904F903F9008952F92C5
:1063B0003F924F925F926F927F928F929F92AF9295
:1063C000BF92CF92DF92EF92FF920F931F93CF93E2
:1063D000DF93CDB7DEB76B97CDBFDEBF782ED92E5A
:1063E000662E798B19821A821B821C821D821E8264
:1063F0001F82188619861A861B861C861D861E8695
:106400001F86188A82E00E94A1C16B3008F4BBC0CD
:106410000F949C1D882309F4CEC00F948B1D80918E
:10642000A73C823009F0B1C080E390E40F945D4C4A
:10643000ACC08F8A988E530162010F2EFCE8EF2EBC
:10644000FFE2FF2EF02D04EB10E020E030E043E906
:106450005FE2B401832DA2DD882331F140918C2FBE
:1064600050918D2F60918E2F70918F2F20E93FE2F8
:1064700083E99FE225DF882361F08091902F90E0EF
:10648000A0E0B0E0EF89F88D80839183A283B3838D
:1064900014C08EEF90E0A0E0B0E0EF89F88D80832B
:1064A0009183A283B38309C08FEF90E0A0E0B0E0B6
:1064B000F40180839183A283B3833394F0E38F1A32
:1064C000FDEF9F0A84E0480E511C94E0690E711C98
:1064D000A6E03A12AECF298C3A8C6B8C862C998828
:1064E0006894552452F80F2EF5E44F2EF02D0F2E00
:1064F000F2E5DF2EF02D0F2EFCE4CF2EF02DAB8831
:10650000BC886D887E88898A9A8AF30101911191ED
:10651000219131913F01D5014D915D916D917D9119
:106520005D017401852DACDC653171058105910536
:106530001CF4F40142861AC0F10180819181A2818C
:10654000B3810097A105B10529F4A989BA891A96E2
:10655000CC920CC00197A105B10521F4E989FA8913
:10656000D28604C0A989BA891A964C925394BCE089
:106570008B0E911CE0E32E1AEDEF3E0AF6E05F125F
:10658000C2CF81E018C080E016C0272C3D2CCE0180
:1065900001968B8B9C8BDE011996AD8BBE8B2C01EB
:1065A000872C9D2C6894772472F8298E3A8E372C8C
:1065B0006B8E3D013ECF6B96CDBFDEBFDF91CF919D
:1065C0001F910F91FF90EF90DF90CF90BF90AF9011
:1065D0009F908F907F906F905F904F903F902F9003
:1065E00008951F93CF93DF93009709F4DAC0EC016D
:1065F0008881843069F128F4813049F08230C9F013
:10660000D0C0883011F1893009F4A7C0CAC08B818D
:10661000813009F0C6C08C81813009F0C2C00F946E
:106620008419CE010E94402A62E0CE010E943C14EF
:10663000B8C080919B48813029F463E0CE010E946C
:106640003C14AFC00E94311CACC00E94394FA9C09D
:10665000CE010E94232282E00E94A1C16B3040F44F
:106660006FED78E383E69CE30E946F18182F10C04B
:106670000F949C1D8823E1F06FED78E383E69CE3A3
:106680000E946F18182F63E77CE388ED9DE48FDE8E
:10669000113071F482E00E94A1C1162F83E69CE3C1
:1066A0000E940A10612F80EF9FE30E942C1207C006
:1066B0008FED98E30E94AD17882309F465C043E786
:1066C0005CE36FED78E3CE016FD95EC00F944707AE
:1066D000882309F463C00F94021B60E370E4CE01C9
:1066E0000E9477250F94360759C08981811159C0BE
:1066F000CE010E94EB21882341F00F94021B60E33E
:1067000070E4CE010E9477254CC01AAA81E08BABC1
:1067100048C08AA9882309F444C08981811141C0F5
:10672000CE010E94B921882341F00F94021B60E33F
:1067300070E4CE010E94772534C01AAA32C00F94AB
:106740004707882371F10F94021B60E370E4CE01C8
:106750000E9477250F94360724C0CE010E94232281
:106760006FED78E383E69CE30F948D0B813031F07D
:106770008FED98E30F94E20B882399F06FED78E3A7
:10678000CE010F940B0F0DC0FE01E95CFD4F80811F
:10679000813009F49BCF823091F6BBCF8AA9811159
:1067A000A4CFDF91CF911F910895CF930E949BC9F1
:1067B000C82F88E10E94A1C1C61741F061E080E0C6
:1067C0000F94640361E081E00F946403CF91089516
:1067D000CF930E949BC9C82F88E10E94A1C1C61710
:1067E00049F061E080E00F94640361E081E00F9480
:1067F000640308C060E080E00F94640360E081E01F
:106800000F946403CF910895CF93DF93EC018091AF
:10681000DD3E882319F0EEE3F9E302C0E5E4FAE394
:10682000209729F18BE7888388E689839CE29A8305
:1068300082E68B839C838CE68D838DE78E831F821B
:1068400021E047E050E0BE01CF010F946A210E9491
:10685000B6B9873061F48091DD3E811108C021E036
:1068600047E050E0BE018EE399E30F946A21DF9187
:10687000CF9108958091A83C0895CF92DF92FF9226
:106880000F931F93CF93DF931F921F92CDB7DEB765
:106890009FEF980F923008F045C09091A83C992343
:1068A00009F443C0813019F009EE1EE302C005E48B
:1068B0001AE3F82E81E6898384E78A8321E042E0A7
:1068C00050E0BE016F5F7F4FC8010F946A210F94A3
:1068D0002C1A0F94431A643F714081059105C8F347
:1068E000C8010E9400A10F942C1A0F94431A643F10
:1068F000714081059105C8F38F2D0E94EDC96C018F
:106900008F2D0E94EDC9FC0101900020E9F731971D
:10691000AF01481B590B41F0B601C8010E9470A19C
:1069200091E003C090E001C090E0892F0F900F909C
:10693000DF91CF911F910F91FF90DF90CF9008953D
:10694000EF92FF920F931F93CF93DF93CDB7DEB7F4
:106950002797CDBFDEBF7C01FB0184818D838581BC
:106960008E8386818F8380819181A281B381898387
:106970009A83AB83BC83870180EAE81688E0F80637
:1069800029F460E183E00F94D53314C080EBE8165E
:1069900088E0F80629F460E283E00F94D53313C051
:1069A00080EAE81689E0F80629F460E184E00F94B3
:1069B000D53312C0003B89E0180729F460E284E077
:1069C0000F94D53312C0003A8AE0180729F460E129
:1069D00085E00F94D53310C0003B8AE0180729F4F6
:1069E00060E285E00F94D53307C0003A1B4021F4E4
:1069F00060E186E00F94D533BE016F5F7F4FC70122
:106A00000E94976F2796CDBFDEBFDF91CF911F9178
:106A10000F91FF90EF900895DC01892BE1F0E62FB4
:106A2000E695E695E69580E2E89FF0011124FA5F8D
:106A30008085677021E030E002C0220F331F6A9525
:106A4000E2F7282381E009F480E08C9311968C937F
:106A5000119712961C920895CF93DF93009709F433
:106A6000A5C06D3209F0A4C03091A80621E0432FE3
:106A7000407235FF20E0FC0120833181231709F4A7
:106A800099C0EC01442309F46BC0311169C00F9423
:106A9000D6150097F9F40E94A82A811119C086E042
:106AA000E4EFF1E2A1E2B4E401900D928A95E1F7FE
:106AB000E1E2F4E401900020E9F73197AF0141529F
:106AC000544421E061E274E48EE399E30F946A2177
:106AD0001A8268C0803D974008F50E94A82A81115B
:106AE00019C086E0EAEFF1E2A1E2B4E401900D9270
:106AF0008A95E1F7E1E2F4E401900020E9F73197AB
:106B0000AF014152544421E061E274E48EE399E321
:106B10000F946A210F94EA151A8244C081E08A8397
:106B20000F94EA150E94A82A81113CC086E0E0E09B
:106B3000F2E2A1E2B4E401900D928A95E1F7E1E27C
:106B4000F4E401900020E9F73197AF014152544439
:106B500021E061E274E48EE399E30F946A2122C09C
:106B60001A8281E090E00F94FD150E94A82A8111FD
:106B700019C086E0E6E0F2E2A1E2B4E401900D92F1
:106B80008A95E1F7E1E2F4E401900020E9F731971A
:106B9000AF014152544421E061E274E48EE399E391
:106BA0000F946A21888189838A8105C080E003C0AF
:106BB00080E001C080E0DF91CF9108958FE098E4FC
:106BC0000C940BD708950E94A82A811117C063EA7C
:106BD00074E48EE399E30F9416218091254581306A
:106BE00029F543EA54E465EA74E48EE399E30E94EC
:106BF00023BF83EA94E40D940721089563EA74E4C3
:106C00008EE399E30E944F9E80912545813071F477
:106C10002BE83CE343EA54E465EA74E48EE399E349
:106C20000E94409E83EA94E40D94072108950E94F7
:106C30003E92882341F01EDE811105C081EA91E475
:106C40000C94342508950E94A82A81112EC06FEB60
:106C500071E485E49AE30E944F9E80914142813025
:106C600021F50E94A82A811112C062E480913E3968
:106C700090913F390E947C6E4091BF415091C0413C
:106C800021E061EC71E48EE399E30F946A212BE833
:106C90003CE34FEB51E461EC71E485E49AE30E943C
:106CA000409E8FEB91E40D9407210895CF92DF92DF
:106CB000EF92FF920F931F93CF93DF930E94A82A26
:106CC000882319F00EE319E302C005E41AE380EB10
:106CD00091E40E947BA0882349F0CCDD811106C09D
:106CE00060EB71E4C8010E941A258BC28091BE41FD
:106CF0008150823008F057C10E94FDA0811104C06C
:106D0000B9DD882309F414C36BE670E489EE9EE3D1
:106D10000E94F29F80919C41813009F072C2E09004
:106D20006B40F0906C4082E0E816F10408F400C378
:106D30008091BE41813039F4809170408F7D8C34D8
:106D400009F0CBC00AC080917040843209F0C5C000
:106D500080917140833509F0C0C00E94A82A81113A
:106D600056C087E0ECE0F2E2A1E2B4E401900D92BB
:106D70008A95E1F7E1E2F4E401900020E9F7319728
:106D8000AF014152544420E061E274E48EE399E3A0
:106D90000F946A2110926D4010926E40E114F1043C
:106DA000A1F080E090E0CBE6D0E4FC01E559FF4B98
:106DB00065818EE399E30F94F6218A819B81019688
:106DC0008A839B838E159F0580F30F94141B1F925B
:106DD0008F9383E192E29F938F93C1E2D4E4DF9398
:106DE000CF930F94B85609900020E9F72197AE0190
:106DF0004152544421E061E274E48EE399E30F943C
:106E00006A210F900F900F900F900F900F900F949A
:106E1000141B882371F181E00E94AC8D813069F4EC
:106E20008BE690E40E9448A08BE690E40E945AA072
:106E30000F94F11A0E94EEA202C00E944FA3E2E05A
:106E4000F3E4808190E0DC01AE5FBC4B25853685A4
:106E5000880F991FFC01EE5FFC4B418152811F9608
:106E60000C9161E08BE89CE30E945A250F941B1C57
:106E700093C0E0929F41F092A0410F94141B682FA1
:106E8000C8010E948A900E94A82A811185C00F948F
:106E9000141B1F928F938091BE411F928F9389E1A3
:106EA00092E29F938F93C1E2D4E4DF93CF930F9448
:106EB000B85609900020E9F72197AE014152544499
:106EC00021E061E274E48EE399E30F946A21EDB767
:106ED000FEB73896EDBFFEBF5FC00E94A82A8111A1
:106EE00057C08091BE41823049F480917040843215
:106EF00029F480917140873409F44AC086E0E7E3C1
:106F0000F2E2A1E2B4E401900D928A95E1F7E1E2A8
:106F1000F4E401900020E9F73197AF014152544465
:106F200020E061E274E48EE399E30F946A21EBE6DA
:106F3000F0E41282138280819181892BA9F080E094
:106F400090E0EF01FC01E559FF4B65818EE399E389
:106F50000F94F6218A819B8101968A839B832881E5
:106F600039818217930770F3E1E2F4E480E290E064
:106F70008083918301900020E9F73197AF0141525E
:106F8000544421E061E274E48EE399E30F946A21B2
:106F90008BE690E40E945AA08BE690E40E9448A001
:106FA0000F94F11A2EC10F9458166B017C016BE6F9
:106FB00070E489EE9EE30E94769F80919C4181302F
:106FC00039F0F5E6CF16D104E104F10408F419C153
:106FD0000F946F1680919C41813079F48BE690E498
:106FE0000E94CBA0882321F0E0909E41F12C40C06C
:106FF000E0906B40F0906C403BC00F2EFBE6EF2E14
:10700000F0E4FF2EF02DF70181818F9380818F9323
:107010008DE392E29F938F93C1E2D4E4DF93CF9309
:107020000F94B85609900020E9F72197AE0141521C
:10703000544421E061E274E48EE399E30F946A2101
:1070400010929E410F900F900F900F900F900F9005
:10705000F701808191818739910530F086E990E0D0
:1070600080936B4090936C40E0906B40F0906C404C
:107070000E94A82A81115DC0FF92EF928CE592E2F6
:107080009F938F93C1E2D4E4DF93CF930F94B856CC
:1070900009900020E9F72197AE014152544420E0C5
:1070A00061E274E48EE399E30F946A2110926D40DB
:1070B00010926E400F900F900F900F900F900F90C6
:1070C000E114F104A1F080E090E0CBE6D0E4FC0113
:1070D000E559FF4B65818EE399E30F94F6218A8190
:1070E0009B8101968A839B838E159F0580F30F9465
:1070F000141B1F928F9383E192E29F938F93C1E2BF
:10710000D4E4DF93CF930F94B85609900020E9F7A9
:107110002197AE014152544421E061E274E48EE3D0
:1071200099E30F946A210F900F900F900F900F909A
:107130000F900F94141B882371F181E00E94AC8D95
:10714000813069F48BE690E40E9448A08BE690E4DD
:107150000E945AA00F94F11A0E94EEA202C00E944F
:107160004FA3E2E0F3E4808190E0DC01AE5FBC4B32
:1071700025853685880F991FFC01EE5FFC4B418108
:1071800052811F960C9161E08BE89CE30E945A2586
:107190000F941B1C30C0E0929F41F092A0410F94CD
:1071A000141B682FC8010E948A900E94A82A81118E
:1071B00022C00F94141B1F928F9389E692E29F9333
:1071C0008F93C1E2D4E4DF93CF930F94B856099024
:1071D0000020E9F72197AE014152544421E061E2D9
:1071E00074E48EE399E30F946A210F900F900F904F
:1071F0000F900F900F908BE690E40E9448A00F94A0
:10720000F11A0F94A116693C71058105910508F4E6
:107210008FC00F94B8160E94A82A81114AC08AE034
:10722000EDE7F2E2A1E2B4E401900D928A95E1F774
:10723000E1E2F4E401900020E9F73197AF01415217
:10724000544420E061E274E48EE399E30F946A21F0
:10725000EBE6F0E41282138280819181892BA9F000
:1072600080E090E0EF01FC01E559FF4B65818EE382
:1072700099E30F94F6218A819B8101968A839B83EF
:10728000288139818217930770F3E1E2F4E480E208
:1072900090E08083918301900020E9F73197AF015E
:1072A0004152544421E061E274E48EE399E30F9487
:1072B0006A2180E790E40E94D9A18823A9F18091F6
:1072C000BE4181110BC0E6ECF2E481E3808382E3EE
:1072D000818383E3828384E3838314C0813041F418
:1072E000E6ECF2E480E380838183828383830AC0B7
:1072F000E6ECF2E481E3808382E3818383E38283AB
:1073000084E3838321E044E050E066EC72E489EE9C
:107310009EE30F946A2121E044E050E066EC72E4C1
:107320008EE399E30F946A218BE690E40E9448A0D3
:10733000DF91CF911F910F91FF90EF90DF90CF9051
:1073400008958F929F92AF92BF92CF92DF92EF9269
:107350000F931F93CF93DF93EC0180E00E947DC1D8
:107360004B015C01209709F45CC11F8EFE01E05BBC
:10737000FD4F1082CE010E940720882309F451C1DD
:107380006E0186E3C80ED11CBE01615E7F4FC6014F
:107390000E9403FA8E8F81111FC00E94A82A8111BA
:1073A00019C08BE1E7E8F2E2A1E2B4E401900D92AA
:1073B0008A95E1F7E1E2F4E401900020E9F73197E2
:1073C000AF014152544421E061E274E48EE399E359
:1073D0000F946A2181E08F8F6DEC76E4C6010E94E4
:1073E00070FFFE01E15BFD4F80838DEC96E40E940F
:1073F00065C88823A1F181E0FE01E05BFD4F808339
:107400008DEC96E40E9402C80E94A82A811127C030
:10741000FE01E05BFD4F80811F928F933197808149
:107420001F928F9382EA92E29F938F9301E214E47A
:107430001F930F930F94B856F80101900020E9F7BD
:107440003197AF014152544421E0B8018EE399E3F2
:107450000F946A21ADB7BEB71896ADBFBEBF8F8D72
:10746000813039F0FE01E05BFD4F8081813009F011
:107470005CC00E94A82A811119C08CE1E5EBF2E200
:10748000A1E2B4E401900D928A95E1F7E1E2F4E41F
:1074900001900020E9F73197AF014152544421E0B7
:1074A00061E274E48EE399E30F946A216894EE2418
:1074B000E2F801ED12E2A5019401BE01685E7F4F82
:1074C000CE0106960E94C1578D8340E050E0BA017C
:1074D000CE010E94E92E8D81882309F4A2C082E0AA
:1074E0000E94A1C1062F8BE00E94A1C121E0611181
:1074F00020E0BE016C5C7F4F40E350E4C6010E9477
:10750000C450CE010E945C1C9E01265A3D4FAE0124
:10751000475A5D4FBE016C5A7D4FCE018D5A9D4F2B
:107520000E94702D0F943B087CC08E010A5F1F4F94
:10753000B80180E390E40E9499568D83811139C08F
:10754000A5019401BE01685E7F4FC8010E94FB53F4
:107550008D8340E050E0BA01CE010E94E92E8D817A
:10756000882309F45EC082E00E94A1C1062F8BE04F
:107570000E94A1C121E0611120E0BE016C5C7F4F3F
:1075800040E350E4C6010E94C450CE010E945C1C3E
:107590009E01265A3D4FAE01475A5D4FBE016C5ABF
:1075A0007D4FCE018D5A9D4F0E94702D0F943B0848
:1075B00038C08E010B5A1D4F0F2EF0E3AF2EF0E4B2
:1075C000BF2EF02DF5016285738520E032E0A60123
:1075D000C5010E94522E015011096E01FDEACF1A19
:1075E000FDEFDF0AD5011A966D917C911B979801EA
:1075F000A601C5010E94842DFE01E75AFD4FD60168
:107600008C918083C65ADD4FF80180818883D50133
:107610001A964D915D916D917C911D97C5010F94C6
:10762000AF4CDF91CF911F910F91EF90DF90CF90F2
:10763000BF90AF909F908F9008956DE28CED98E38E
:107640000BDA882309F467C080911733882309F483
:1076500046C00E94E46184E0809326060F941315CF
:107660008DEC96E40E94BCD58BE89CE36ADE8091A9
:10767000DB3E8823F1F00E9480D3813019F0823004
:1076800069F017C08091DA3E882329F08DEC96E4EA
:107690000E941ED30EC00E94F1D20BC08091DA3E30
:1076A000882329F08DEC96E40E94A0D402C00E94A9
:1076B0006BD4109217330F941B1C8BE89CE30E9431
:1076C000F32281110F9484198BE89CE30E94402AD5
:1076D0006091CE3E8BE89CE30E943C141CC00F944A
:1076E0001B1C0F94621966E08BE89CE30E943C141B
:1076F00061E081E99CE30E9467560E94E6530F9483
:10770000972A0E94BA6181E08093173384E08093C6
:1077100025060F94131580911733882331F00E94AA
:1077200038608111FCCF8091173308954F925F929A
:107730006F927F928F929F92AF92BF92CF92DF9281
:10774000EF92FF921F93CF93DF93CDB7DEB72797CA
:10775000CDBFDEBF7C0110929C4810E00F2E812C23
:10776000FBE49F2EA12CB12CF02D0F2EF1E2CF2E99
:10777000F4E4DF2EF02D0F2EF0E84F2EF5E25F2E11
:10778000612C712CF02D111120C080E096E9A0E051
:10779000B0E0F70180839183A283B3838AE0E6EDB2
:1077A000F2E2D60101900D928A95E1F7F60101907F
:1077B0000020E9F73197AF014152544421E0B6016E
:1077C0008EE399E30F946A215CC0113001F580ECDF
:1077D00092E1A0E0B0E0F70180839183A283B383BC
:1077E00089E0E0EEF2E2D60101900D928A95E1F790
:1077F000F60101900020E9F73197AF01415254445E
:1078000021E0B6018EE399E30F946A213AC0123069
:10781000E9F4D7014D925D926D927C92139789E0C5
:10782000E9EEF2E2D60101900D928A95E1F7F601B8
:1078300001900020E9F73197AF014152544421E013
:10784000B6018EE399E30F946A211BC0F701808291
:107850009182A282B38289E0E2EFF2E2D601019046
:107860000D928A95E1F7F60101900020E9F7319732
:10787000AF014152544421E0B6018EE399E30F94E5
:107880006A21D70114968C9114978D8315968C914B
:1078900015978E8316968C9116978F838D919D9157
:1078A0000D90BC91A02D89839A83AB83BC8360E14A
:1078B00085E00F94D533BE016F5F7F4F80EA9AE079
:1078C0000E94976F0F948E1B08C08FE098E40E946F
:1078D0000BD7813041F00E94ED1B0F94A11B803A21
:1078E0009F4098F37AC011111DC08CE0EBEFF2E2DB
:1078F000A1E2B4E401900D928A95E1F7E1E2F4E4AB
:1079000001900020E9F73197AF014152544421E042
:1079100061E274E48EE399E30F946A2182E080933C
:107920009C4878C01130E9F48BE0E7E0F3E2A1E293
:10793000B4E401900D928A95E1F7E1E2F4E401905C
:107940000020E9F73197AF014152544421E061E250
:1079500074E48EE399E30F946A2181E080939C485C
:1079600059C01230E9F48BE0E2E1F3E2A1E2B4E4C1
:1079700001900D928A95E1F7E1E2F4E40190002094
:10798000E9F73197AF014152544421E061E274E4D8
:107990008EE399E30F946A2183E080939C483AC078
:1079A0008BE0EDE1F3E2A1E2B4E401900D928A955F
:1079B000E1F7E1E2F4E401900020E9F73197AF014B
:1079C0004152544421E061E274E48EE399E30F9460
:1079D0006A2184E080939C481DC01F5F143009F029
:1079E000D2CE89E0E8E2F3E2A1E2B4E401900D92A4
:1079F0008A95E1F7E1E2F4E401900020E9F731979C
:107A0000AF014152544421E061E274E48EE399E312
:107A10000F946A212796CDBFDEBFDF91CF911F91D2
:107A2000FF90EF90DF90CF90BF90AF909F908F909E
:107A30007F906F905F904F900895CF92DF92EF927A
:107A4000FF920F931F93CF938BE89CE30E944F14F8
:107A5000883009F4D6C08BE89CE30E944F1486302E
:107A600009F4CFC08091E73E9091E83E8E349C406F
:107A700008F4BEC00E947DC98111B4C0C2C00F9479
:107A80005C1C81111FC00F945F1C0E94A82A8111E9
:107A900019C088E1E1E3F3E2A1E2B4E401900D92C0
:107AA0008A95E1F7E1E2F4E401900020E9F73197EB
:107AB000AF014152544421E061E274E48EE399E362
:107AC0000F946A210F94481C811129C09AC08CE13F
:107AD000E9E4F3E2A1E2B4E401900D928A95E1F7C2
:107AE000E1E2F4E401900020E9F73197AF0141525F
:107AF000544421E061E274E48EE399E30F946A2137
:107B00000F94F114C0E00F94E014882331F00F9427
:107B1000F114CF5FCA30B9F702C0CA30A0F30F9496
:107B200062190E94E6530E94A82A811119C08EE0B2
:107B3000E7E5F3E2A1E2B4E401900D928A95E1F762
:107B4000E1E2F4E401900020E9F73197AF014152FE
:107B5000544421E061E274E48EE399E30F946A21D6
:107B60000F94F11401E010E0C0E00F2EF3E1CF2EEE
:107B7000F1E2DF2EF02D0F2EF1E2EF2EF4E4FF2ED6
:107B8000F02D0F94E014882341F10F94F114CF5F8E
:107B90000E94A82A81111CC01F930F93DF92CF92DD
:107BA000FF92EF920F94B856F70101900020E9F789
:107BB0003197AF014152544421E0B7018EE399E37C
:107BC0000F946A210F900F900F900F900F900F90CD
:107BD0000F5F1F4FC33019F0D4CFC33090F20F9412
:107BE000A4000FC00F94521C882309F46BCF47CF19
:107BF00086EC92E40E9404340E94A82A811180CF6E
:107C000066CFCF911F910F91FF90EF90DF90CF90B3
:107C10000895F8940E94EC640F9480330F94C3038A
:107C20000F94240460E080E00F94BC040F94972A22
:107C30000E94099F0F9440030E94C5DD41E060EA65
:107C400078E085E49AE30F94CC2165E170E280EA64
:107C500098E00E94A034E0EAF8E083818F7C8061A4
:107C600083838FEB91E40F94072161E081EA91E433
:107C70000E946BA041E060EA7BE089EE9EE30F94F6
:107C8000CC216EE070E280EA9BE00E94A034E0EA42
:107C9000FBE083818F7C806183838BE690E40E948C
:107CA00048A08BE690E40E945AA061E080EB91E44A
:107CB0000E946BA01092BE411092C54282E492E4F1
:107CC0000F94072141E060EA7AE08CE59BE30F9492
:107CD000CC2167E070E280EA9AE00E94A034E0EAFA
:107CE000FAE083818F7C8061838341E060EA79E000
:107CF0008EE399E30F94CC2160E070E280EA99E092
:107D00000E94A034E0EAF9E083818F7C8061838364
:107D100083EA94E40F9407210F947B140F94EA16DE
:107D20000F948E180F942A1B0F9410170F94FA1C9F
:107D30000F9453010F94C6060E94670FC0E060E0E5
:107D40008C2F0F946403CF5FC830C9F787E080930E
:107D5000A2007894E0E2F6E082E0868384E0868305
:107D60000E9439C1811116C00E943FC20E9469C29F
:107D70000E94B9C60E9456C80E944EC90E9495C969
:107D800081E00E9442CA82E00E9442CA81E0809360
:107D9000D93E27C00E942CC6882309F181E0809338
:107DA000D93E0E94A82A81111CC08DE1E5E6F3E2CC
:107DB000A1E2B4E401900D928A95E1F7E1E2F4E4E6
:107DC00001900020E9F73197AF014152544421E07E
:107DD00061E274E48EE399E30F946A2102C0109289
:107DE000D93E0E94E2C70F943B080E940CC681E076
:107DF0000F9440186DE28CED98E30E940C350E94C0
:107E000001A360E475E48FE098E40E947FCF8FE0E7
:107E100098E40E9461CA8BE89CE30E94561480E0BB
:107E20000F943F068DEC96E40E94BCD50F94740528
:107E30008BE89CE386DA81E00E94B9B980E00E9479
:107E4000B3B980E00E94BCB980E00E94BFB90E9433
:107E500087170E94D5330E940D9F8FE098E40E94FF
:107E600061CA87E090E262DC0E9480D3813029F40D
:107E70008091DA3E0E944ED925C00E9480D3823084
:107E800091F481E00E9483D38091DA3E882329F027
:107E90008DEC96E40E94A0D402C00E946BD481E0D5
:107EA0000E9435D40FC00E9480D3833029F481E230
:107EB00094E40E9465D506C00E9480D3843011F4FA
:107EC0000E948CD984E0809326060E94D1DD81E057
:107ED0000E943D3482E00E943D348BE89CE30E9486
:107EE000402A8EE399E30E9429AB0E94A30F0F94CE
:107EF000DC1D02E813E2C1E2D4E40E94DE3560E456
:107F000075E48FE098E40E94B2168BE89CE30E942F
:107F100043168BE89CE30E94DB158BE89CE30E94F0
:107F2000F32E8BE89CE30E94F1320E94E33585DB5F
:107F30000E9417360E9456368BE89CE30E94F71B7E
:107F40000E94FEDD0E94B6B9833031F50E942020E8
:107F5000882311F10E94A82A81111EC00F943F1995
:107F60001F928F931F930F93DF93CF930F94B85665
:107F7000FE0101900020E9F73197AF0141525444CE
:107F800021E0BE018EE399E30F946A210F900F90D8
:107F90000F900F900F900F9087EE9EE30E94872422
:107FA00062E073E48BE89CE30E94252662E073E4C0
:107FB0008BE89CE30E9479260F944A073EDD0FB6BA
:107FC00007FC9BCF80E00E94937A0E94A77AFFCFA4
:107FD000EF92FF920F931F93CF93DF93009749F196
:107FE0006115710541F14115510539F18A017B0196
:107FF000EC010F943F56F80180839183892B89F01F
:10800000D70120E030E0FE01E20FF31FE491ED9391
:108010002F5F3F4FF801808191812817390798F32E
:1080200002C020E030E0F701E20FF31F108281E090
:1080300005C080E003C080E001C080E0DF91CF9107
:108040001F910F91FF90EF9008950F931F93CF937F
:10805000DF930097C9F061157105C1F04115510515
:10806000B9F0EA018B01FC0165917491C8010F948C
:108070003856F80101900020E9F73197E01BF10B29
:10808000E883F98381E005C080E003C080E001C09F
:1080900080E0DF91CF911F910F9108957F928F9291
:1080A0009F92AF92BF92CF92DF92EF92FF920F9387
:1080B0001F93CF93DF931F921F92CDB7DEB7009728
:1080C00009F49BC06115710509F497C0D42E7B019A
:1080D0008C01AE014F5F5F4FBC0180E594E178DF1A
:1080E000882309F48AC089819A815C012FEFA21A42
:1080F000B20AF801E80FF91F20E22083B8016A0DE7
:108100007B1DAE014F5F5F4F89E394E161DF882300
:1081100009F473C089819A81A80EB91EF801EA0D8D
:10812000FB1D8DE0808382E0A80EB11C8AE0818374
:10813000B8016A0D7B1DAE014F5F5F4F82E294E193
:1081400047DF882309F459C0A981BA81AA0EBB1E52
:1081500048018A0C9B1C0F2EFDE07F2EF02DF401B0
:1081600070820F2EFAE0CF2EF02DC182C50102964B
:10817000800F911F0E945FC1F401748ED5015E963D
:10818000C58EDD2059F1A00FB11F8AE0EAE8F3E2C5
:1081900001900D928A95E1F7F7E2AF0EB11C0E94B3
:1081A0008CC6BC01C8018A0D9B1D0F949A560E9473
:1081B0008CC6FC0101900020E9F73197E81BF90B10
:1081C000E131F10518F4E983FA8304C080E190E01D
:1081D00089839A83A981BA81AA0DBB1DF801EA0F90
:1081E000FB1F8DE0808312968AE08183F801EA0FFD
:1081F000FB1F1082F701A083B1830F900F90DF91D6
:10820000CF911F910F91FF90EF90DF90CF90BF9093
:10821000AF909F908F907F900895CF92DF92EF92D2
:10822000FF920F931F93CF93DF931F921F92CDB7AF
:10823000DEB76115710591F14115510579F100978E
:1082400069F17A016B018C0119821A82AE014F5FCC
:108250005F4F89EF92E1BCDE882301F1C8010696E9
:108260009F938F9384E993E29F938F9389819A815F
:108270008C0D9D1D9F938F930F94B856F60101901E
:108280000020E9F73197EC19FD09D701ED93FC9334
:108290000F900F900F900F900F900F900F900F90E6
:1082A000DF91CF911F910F91FF90EF90DF90CF90D2
:1082B0000895BF92CF92DF92EF92FF920F931F9398
:1082C000CF93DF931F921F92CDB7DEB7009709F4CB
:1082D00082C06115710509F47EC06B018C011982A1
:1082E0001A82DB011D921C92AE014F5F5F4FBC01F1
:1082F0008DEE92E16DDE882309F46DC0E8E7F3E5C9
:1083000087858F9386858F9385858F9384858F93BB
:1083100081EE9AE29F938F9389819A81800F911FBA
:108320009F938F930F94B856F80101900020E9F7BE
:108330003197E01BF10BE983FA83CDBFDEBFB12C8F
:108340000F2EF9E9EF2EF3E2FF2EF02D2DC0EB2DCD
:10835000F0E0EE0FFF1FEE0FFF1FE858FC4ADF01B1
:108360005A9613968C9113978F9312968C9112971D
:108370008F9311968C918F93828D8F93FF92EF92B2
:1083800089819A81800F911F9F938F930F94B85684
:10839000F80101900020E9F73197E01BF10BE98328
:1083A000FA83B394CDBFDEBF0F94631CB81678F286
:1083B000E981FA81E00FF11F8DE09AE080839183DB
:1083C0001282F80101900020E9F73197E01BF10BD0
:1083D000D601ED93FC930F900F90DF91CF911F91F9
:1083E0000F91FF90EF90DF90CF90BF900895BF92D4
:1083F000CF92DF92EF92FF920F931F93CF93DF9371
:1084000000D01F92CDB7DEB719821A821B821C8260
:10841000009709F4CDC06115710509F4C9C0022F98
:10842000B42E6B017C011FEF120F123108F0B5C0A2
:10843000AE014F5F5F4FBC0185E093E1C9DD88234A
:1084400009F4B6C01A3079F5BB2069F069817A81E8
:108450006E0D7F1DAE014D5F5F4F86E999E0F5DD42
:1084600081110EC0A5C069817A816E0D7F1DAE019C
:108470004D5F5F4F82E799E0E8DD882309F498C0FB
:1084800069817A818B819C81680F791F69837A83E6
:108490006E0D7F1DAE014D5F5F4F88EF9AE098DD56
:1084A000811171C085C084EF800F873008F046C00D
:1084B000BB2089F069817A816E0D7F1D812F90E04C
:1084C000880F991FAE014D5F5F4F8C57964FBDDDF2
:1084D000811112C06DC069817A816E0D7F1D812F5F
:1084E00090E0880F991FAE014D5F5F4F805A964F05
:1084F000ACDD882309F45CC069817A818B819C8121
:10850000680F791F69837A8322EF200F223058F495
:108510006E0D7F1DAE014D5F5F4F84E799E095DDE5
:10852000811131C045C06E0D7F1DAE014D5F5F4FA3
:1085300083EE9AE04DDD811126C03AC0BB2091F058
:1085400069817A816E0D7F1D212F30E0C901880F6E
:10855000991FAE014D5F5F4F8C57964F76DD8111AD
:1085600012C026C069817A816E0D7F1D212F30E0F7
:10857000C901880F991FAE014D5F5F4F805A964F1A
:1085800064DD8823A9F029813A818B819C81820F47
:10859000931FF601808391830BC0AE014F5F5F4F45
:1085A000BC0185E093E114DD882311F010E0C6CF13
:1085B0002496CDBFDEBFDF91CF911F910F91FF9029
:1085C000EF90DF90CF90BF90089589E10E94A1C104
:1085D00081E0623009F080E00895CF92DF92EF925F
:1085E000FF921F93CF93DF9300D01F92CDB7DEB7DA
:1085F00019821A821B821C82009709F453C06115EC
:10860000710509F44FC0142F6B017C01AE014F5F5F
:108610005F4FBC0185E093E1DBDC882309F442C0B5
:10862000173089F01930E1F0113039F569817A811C
:108630006E0D7F1DAE014D5F5F4F82E89AE0C8DC92
:10864000811127C02FC069817A816E0D7F1DAE0117
:108650004D5F5F4F81E29AE0BBDC81111AC022C0FE
:1086600069817A816E0D7F1DAE014D5F5F4F80EC99
:1086700099E0AEDC81110DC015C069817A816E0D63
:108680007F1DAE014D5F5F4F82E89AE0A1DC882339
:1086900049F029813A818B819C81820F931FF601D9
:1086A000808391832496CDBFDEBFDF91CF911F9150
:1086B000FF90EF90DF90CF900895EF92FF920F938D
:1086C0001F93CF93DF931F921F92CDB7DEB719820E
:1086D0001A82009751F16115710539F17B018C0106
:1086E00087E10E94A1C1662351F0AE014F5F5F4F49
:1086F000B8018EE893E16CDC81110AC016C0AE01AE
:108700004F5F5F4FB80181E193E162DC882369F03C
:1087100089819A81F801E80FF91F2DE020832AE072
:1087200021830296F701808391830F900F90DF9150
:10873000CF911F910F91FF90EF900895EF92FF92CC
:108740000F931F93CF93DF931F921F92CDB7DEB786
:10875000009709F47EC04115510509F47CC0F22E42
:108760008A01E62EAE014F5F5F4FB8016EDC8111CA
:1087700002C019821A8283E0E81629F18E1538F0BA
:1087800091E0E91659F082E0E81699F03AC094E0D9
:10879000E91619F185E0E81651F133C0EDECF6E485
:1087A00001900020E9F73197ED5CF6446DEC76E43A
:1087B0002BC0E4EEF6E401900020E9F7E55EF64414
:1087C00064EE76E421C0EBEFF6E401900020E9F7D7
:1087D000EC5FF6446BEF76E417C0E2E1F7E401905A
:1087E0000020E9F7E351F74462E177E40DC0E9E2E4
:1087F000F7E401900020E9F7EA52F74469E277E4F0
:1088000003C06DEC76E4E0E0EF3008F0EEE0CB0181
:108810008E0F911DFC01108289819A81800F911F1A
:108820000F949A56F80101900020E9F73197E01B68
:10883000F10BFF2091F0C8018E0F911DFC018CE21D
:108840009DE0808391838AE090E08283938381E03E
:1088500005C080E003C080E001C081E00F900F9070
:10886000DF91CF911F910F91FF90EF9008958F921C
:108870009F92AF92BF92CF92DF92EF92FF920F93AF
:108880001F93CF93DF931F921F92CDB7DEB7309126
:10889000DA3E311104C0FB011082118236C000970C
:1088A000A1F1672B91F14115510579F1022F4A0190
:1088B0006C010F2EFCEDEF2EF9E1FF2EF02D11E0F3
:1088C000202FA601612FC70139DF8823A9F0F60107
:1088D00001900020E9F731975F01AC18BD089E01B7
:1088E0002F5F3F4FA501B601C4010F94AF4A8981A4
:1088F0009A81A816B90631F41F5FF2E0EF0EF11C61
:108900001630F1F6C4010F945D4C0F900F90DF917B
:10891000CF911F910F91FF90EF90DF90CF90BF907C
:10892000AF909F908F9008958F929F92AF92BF9239
:10893000DF92EF92FF920F931F93CF93DF93CDB708
:10894000DEB72597CDBFDEBF009709F497C4411568
:10895000510509F495C4D22E7A01162FAE014F5F4E
:108960005F4FB70172DB811102C019821A82163182
:1089700009F06DC00E94BBF54B015C01672B682BB1
:10898000692BE1F486E10E94A1C120E13EE040E0D4
:1089900050E00F946F545F934F933F932F9384EA6B
:1089A00093E29F938F9389819A818E0D9F1D9F9350
:1089B0008F930F94B856CDBFDEBF49C486E10E94A5
:1089C000A1C1992324F586E10E94A1C120E13EE0E6
:1089D00040E050E00F946F54CA01B9010F94E726AC
:1089E000BF92AF929F928F929F938F937F936F933B
:1089F0008FE993E29F938F9389819A818E0D9F1DBA
:108A00009F938F930F94B856CDBFDEBF20C486E1ED
:108A10000E94A1C1BF92AF929F928F9220E13EE04F
:108A200040E050E00F946F545F934F933F932F9328
:108A300080EA93E29F938F9389819A818E0D9F1D87
:108A40009F938F930F94B856CDBFDEBF00C41230F2
:108A500060F4812F0E9406C229813A81BC01C701BE
:108A6000820F931F0F949A56F2C3163081F486E05A
:108A70000E94A1C18B019C0189819A814BE0BE01BA
:108A80006B5F7F4F8E0D9F1D0F944027E0C3153005
:108A900081F485E00E94A1C18B019C0189819A81AA
:108AA0004BE0BE016B5F7F4F8E0D9F1D0F948C2896
:108AB000CEC3123009F06EC082E00E94A1C16331C2
:108AC00071058105910524F061E070E080E090E09F
:108AD000013009F049C029813A812E0D3F1DDC018A
:108AE000CB010197A109B109880F991FAE014D5F14
:108AF0005F4FB9018D5A974FA8DA8130F9F4F70129
:108B000001900020E9F73197EE19FF09E983FA8314
:108B100082E00E94A1C19F938F937F936F9389EA14
:108B200093E29F938F9389819A818E0D9F1D9F93CE
:108B30008F930F94B856CDBFDEBF89C382E00E94E9
:108B4000A1C19F938F937F936F938AEA93E29F9340
:108B50008F9389819A818E0D9F1D9F938F930F9480
:108B6000B856CDBFDEBF73C382E00E94A1C19F9300
:108B70008F937F936F9382EE9AE29F938F93898175
:108B80009A818E0D9F1D9F938F930F94B856CDBFE2
:108B9000DEBF5DC31B3059F08DEE810F823038F09F
:108BA00089EE810F823018F01A3109F05CC0812FF4
:108BB0000E94A1C14B015C01011113C0BF92AF9291
:108BC0009F926F9382EE9AE29F938F9389819A810D
:108BD0008E0D9F1D9F938F930F94B856CDBFDEBF10
:108BE00036C3672B682B692BF9F469817A816E0D86
:108BF0007F1DAE014D5F5F4F8FE498E0E9D9811191
:108C000026C31F921F921F921F9282EE9AE29F9399
:108C10008F9389819A818E0D9F1D9F938F930F94BF
:108C2000B856CDBFDEBF13C369817A816E0D7F1D3B
:108C3000AE014D5F5F4F8CE498E0CAD9811107C344
:108C4000BF92AF929F928F9282EE9AE29F938F9300
:108C500089819A818E0D9F1D9F938F930F94B85693
:108C6000CDBFDEBFF4C2173009F05CC087E00E94C0
:108C7000A1C14B015C01011113C0BF92AF929F9241
:108C80006F9382EE9AE29F938F9389819A818E0DE2
:108C90009F1D9F938F930F94B856CDBFDEBFD7C251
:108CA000672B682B692BF9F469817A816E0D7F1D22
:108CB000AE014D5F5F4F88E498E08AD98111C7C249
:108CC0001F921F921F921F9282EE9AE29F938F93A0
:108CD00089819A818E0D9F1D9F938F930F94B85613
:108CE000CDBFDEBFB4C269817A816E0D7F1DAE013A
:108CF0004D5F5F4F84E498E06BD98111A8C2BF92A9
:108D0000AF929F928F9282EE9AE29F938F93898186
:108D10009A818E0D9F1D9F938F930F94B856CDBF50
:108D2000DEBF95C2143009F05CC084E00E94A1C18E
:108D30004B015C01011113C0BF92AF929F926F93E0
:108D400082EE9AE29F938F9389819A818E0D9F1D67
:108D50009F938F930F94B856CDBFDEBF78C2672B19
:108D6000682B692BF9F469817A816E0D7F1DAE0144
:108D70004D5F5F4F8DE398E02BD9811168C21F9240
:108D80001F921F921F9282EE9AE29F938F93898186
:108D90009A818E0D9F1D9F938F930F94B856CDBFD0
:108DA000DEBF55C269817A816E0D7F1DAE014D5FB8
:108DB0005F4F84E398E00CD9811149C2BF92AF9212
:108DC0009F928F9282EE9AE29F938F9389819A81EC
:108DD0008E0D9F1D9F938F930F94B856CDBFDEBF0E
:108DE00036C2133009F0ABC083E00E94A1C14B0131
:108DF0005C01011113C0BF92AF929F926F9382EEFC
:108E00009AE29F938F9389819A818E0D9F1D9F93E4
:108E10008F930F94B856CDBFDEBF19C291E089166B
:108E20009104A104B10461F182E088169104A104C7
:108E3000B10409F445C081149104A104B10409F0FE
:108E40005FC069817A816E0D7F1DAE014D5F5F4FFE
:108E500088E298E0BDD88111FAC11F921F921F923B
:108E60001F9282EE9AE29F938F9389819A818E0D51
:108E70009F1D9F938F930F94B856CDBFDEBFE7C160
:108E800069817A816E0D7F1DAE014D5F5F4F8FE16D
:108E900098E09ED88111DBC11F921F921F9281E042
:108EA0008F9382EE9AE29F938F9389819A818E0DA0
:108EB0009F1D9F938F930F94B856CDBFDEBFC7C140
:108EC00069817A816E0D7F1DAE014D5F5F4F8AE132
:108ED00098E07ED88111BBC11F921F921F9282E041
:108EE0008F9382EE9AE29F938F9389819A818E0D60
:108EF0009F1D9F938F930F94B856CDBFDEBFA7C120
:108F000069817A816E0D7F1DAE014D5F5F4F88E2F2
:108F100098E05ED881119BC1BF92AF929F928F92D1
:108F200082EE9AE29F938F9389819A818E0D9F1D85
:108F30009F938F930F94B856CDBFDEBF88C1193170
:108F400009F0AEC089E10E94A1C14B015C01011191
:108F500013C0BF92AF929F926F9382EE9AE29F935B
:108F60008F9389819A818E0D9F1D9F938F930F946C
:108F7000B856CDBFDEBF6BC191E089169104A10444
:108F8000B10461F182E088169104A104B10409F4EE
:108F900046C081149104A104B10409F061C0698143
:108FA0007A816E0D7F1DAE014D5F5F4F86E198E0C7
:108FB0000FD881114CC11F921F921F921F9282EEF7
:108FC0009AE29F938F9389819A818E0D9F1D9F9323
:108FD0008F930F94B856CDBFDEBF39C169817A81B6
:108FE0006E0D7F1DAE014D5F5F4F80E198E00E94E6
:108FF000E83F81112CC11F921F921F9281E08F9335
:1090000082EE9AE29F938F9389819A818E0D9F1DA4
:109010009F938F930F94B856CDBFDEBF18C169815F
:109020007A816E0D7F1DAE014D5F5F4F88E098E045
:109030000E94E83F81110BC11F921F921F9282E094
:109040008F9382EE9AE29F938F9389819A818E0DFE
:109050009F1D9F938F930F94B856CDBFDEBFF7C06F
:1090600069817A816E0D7F1DAE014D5F5F4F86E194
:1090700098E00E94E83F8111EAC0BF92AF929F92B0
:109080008F9282EE9AE29F938F9389819A818E0DBF
:109090009F1D9F938F930F94B856CDBFDEBFD7C04F
:1090A000123109F05EC082E10E94A1C14B015C0156
:1090B000011113C0BF92AF929F926F9382EE9AE21A
:1090C0009F938F9389819A818E0D9F1D9F938F937C
:1090D0000F94B856CDBFDEBFBAC0672B682B692B83
:1090E00001F569817A816E0D7F1DAE014D5F5F4F85
:1090F00087EF97E00E94E83F8111A9C01F921F925D
:109100001F921F9282EE9AE29F938F9389819A8198
:109110008E0D9F1D9F938F930F94B856CDBFDEBFCA
:1091200096C069817A816E0D7F1DAE014D5F5F4FE4
:109130008FEE97E00E94E83F811189C0BF92AF9205
:109140009F928F9282EE9AE29F938F9389819A8168
:109150008E0D9F1D9F938F930F94B856CDBFDEBF8A
:1091600076C0153109F05EC085E10E94A1C14B01B6
:109170005C01011113C0BF92AF929F926F9382EE78
:109180009AE29F938F9389819A818E0D9F1D9F9361
:109190008F930F94B856CDBFDEBF59C0672B682B95
:1091A000692B01F569817A816E0D7F1DAE014D5FDE
:1091B0005F4F83E098E00E94E83F811148C01F9212
:1091C0001F921F921F9282EE9AE29F938F93898142
:1091D0009A818E0D9F1D9F938F930F94B856CDBF8C
:1091E000DEBF35C069817A816E0D7F1DAE014D5F96
:1091F0005F4F8EEF97E00E94E83F811128C0BF9239
:10920000AF929F928F9282EE9AE29F938F93898181
:109210009A818E0D9F1D9F938F930F94B856CDBF4B
:10922000DEBF15C0812F0E94A1C19F938F937F93B2
:109230006F9382EE9AE29F938F9389819A818E0D2C
:109240009F1D9F938F930F94B856CDBFDEBFF7013C
:1092500001900020E9F73197EE19FF09DD2091F028
:10926000C7018E0F911DFC018CE29DE080839183EC
:109270008AE090E08283938381E005C080E003C0B0
:1092800080E001C081E02596CDBFDEBFDF91CF91A8
:109290001F910F91FF90EF90DF90BF90AF909F9044
:1092A0008F9008956F927F928F929F92AF92BF920C
:1092B000CF92DF92EF92FF920F931F93CF93DF93A2
:1092C0001F921F92CDB7DEB70097B1F1672BA1F1C6
:1092D0004115510589F1802E922E3A016C010F2E15
:1092E000FBE8EF2EFBE1FF2EF02D10E0082D292DDD
:1092F000A601612FC70118DB8823A9F0F6010190B0
:109300000020E9F731975F01AC18BD089E012F5F7F
:109310003F4FA501B601C3010F94AF4A89819A81DD
:10932000A816B90631F41F5F82E0E80EF11C1C316B
:10933000E9F6C3010F945D4C0F900F90DF91CF9130
:109340001F910F91FF90EF90DF90CF90BF90AF9063
:109350009F908F907F906F9008958F929F92AF9281
:10936000BF92DF92EF92FF920F931F93CF93DF9301
:109370001F921F92CDB7DEB7009709F48FC0611519
:10938000710509F48BC04B017C010E948CC69F9330
:109390008F9380EB93E29F938F93FF92EF920F94C2
:1093A000B856F70101900020E9F73197AF014E1947
:1093B0005F094231510510F041E150E09E012F5FFD
:1093C0003F4FB701C4010F94AF4A0F900F900F9019
:1093D0000F900F900F90D12C0F2EFEEDAF2EF9E2D3
:1093E000BF2EF02D8D2D0E947DC19F938F937F9373
:1093F0006F93BF92AF92FF92EF920F94B856F7011E
:1094000001900020E9F731978F010E191F099E0185
:109410002F5F3F4FA801B701C4010F94AF4ACDBFE2
:10942000DEBF89819A810817190731F4D39496E138
:10943000D912D8CF11E001C011E00F2EF0EBAF2E02
:10944000F3E2BF2EF02D812F0E94EDC99F938F93E1
:10945000BF92AF92FF92EF920F94B856F70101902E
:109460000020E9F73197AF014E195F0942315105EC
:1094700010F041E150E09E012F5F3F4FB701C40162
:109480000F94AF4A1F5F0F900F900F900F900F90A7
:109490000F901330C1F6C4010F945D4C0F900F90E4
:1094A000DF91CF911F910F91FF90EF90DF90BF90D0
:1094B000AF909F908F9008952F923F924F925F921E
:1094C0006F927F928F929F92AF92BF92CF92DF92D4
:1094D000EF92FF920F931F93CF93DF93CDB7DEB739
:1094E000E197CDBFDEBF91E09BA76115710509F43F
:1094F000B7C34115510509F4B5C38A017B0189AB96
:109500000F941B1C29A9213089F4A80168E173E399
:10951000CE010B960E940C55182F86E08BA70F9456
:10952000E9086DA77EA78FA798AB1AC0A80168E1CC
:1095300073E3CE010B960E948155182F0F94E90812
:109540006DA77EA78FA798AB82E00F946207862F46
:10955000AE01445D5F4FBE01655D7F4F0E94682292
:10956000112309F481C341E0BE01675F7F4FC7014A
:109570000E944E4049855A85CA01A0E0B0E0898327
:109580009A83AB83BC839E01275F3F4FB701CE0117
:109590000B960F94AF4ACE010B960F945D4CBE0113
:1095A000655F7F4FC701D9DE0DE0D7010C931AE04C
:1095B00011961C939E01275F3F4F42E050E0B70198
:1095C000CE010B960F94AF4ACE010B960F945D4CD3
:1095D000E8E1F3E3018B128B9E01275F3F4F43E1EC
:1095E00050E0BF01CE010B960F94AF4ACE010B960F
:1095F0000F945D4CB9A9B1113DC30F943E090F946E
:10960000270938C301E021E0A701612FC6018CD9E9
:10961000882381F0F70101900020E9F73197AF012D
:109620004E195F099E01275F3F4FB701CE010B9690
:109630000F94AF4AE2E0CE0ED11C1F5F133011F73A
:109640000F2EFDE9CF2EFBE1DF2EF02D19E001E01A
:1096500021E0A701612FC60167D9882381F0F701B6
:1096600001900020E9F73197AF014E195F099E0183
:10967000275F3F4FB701CE010B960F94AF4AF2E040
:10968000CF0ED11C1F5F1B3011F70F2EF2E18F2E72
:10969000912CA12CB12CF02D28E182169104A1046B
:1096A000B10451F401E021E0A70169E18DEB9BE1F8
:1096B0003BD981110EC030C001E021E0A701682D27
:1096C000C401880F991F8557944E2ED98823C1F065
:1096D00007C00F2EF9E18F2E912CA12CB12CF02D6B
:1096E000F70101900020E9F73197AF014E195F09AA
:1096F0009E01275F3F4FB701CE010B960F94AF4AF3
:1097000033E0830E911CA11CB11C4AE18416910424
:10971000A104B10408F4C0CFCE010B960F945D4CA8
:1097200089E00E94A1C16F31710581059105C0F4E6
:10973000DC01CB01072E7CE0880F991FAA1FBB1FFD
:109740007A95D1F7702D89839A83AB83BC8380E0AF
:1097500090E1A0E0B0E08D839E83AF83B88717C00F
:10976000DC01CB01072E79E0880F991FAA1FBB1FD0
:109770007A95D1F7702D89839A83AB83BC8380E07F
:1097800092E0A0E0B0E08D839E83AF83B8878981AB
:109790009A81AB81BC812DA53EA54FA558A928175C
:1097A00039074A075B07A1F1AE01475F5F4FB70179
:1097B00084EB99E00E94E83F813081F4F701019049
:1097C0000020E9F73197AF014E195F099E01275F2D
:1097D0003F4FB701CE010B960F94AF4ACE010B96C7
:1097E0000F945D4CCE010B960F94A44C39A9311106
:1097F0003DC20F94B5098BE89CE30E94F3228111CE
:109800000F9484198BE89CE30E94402A80E03AC2BE
:10981000AE01475F5F4FB70188EA99E00E94E83FD9
:10982000813081F4F70101900020E9F73197AF0111
:109830004E195F099E01275F3F4FB701CE010B967E
:109840000F94AF4A48A94F935FA55F938EA58F935E
:109850009DA59F9388858F938F818F938E818F9302
:109860008D818F9384EB93E29F938F93FF92EF927E
:109870000F94B856F70101900020E9F73197AF0136
:109880004E195F099E01275F3F4FB701CE010B962E
:109890000F94AF4A88E290E089879A8768E2C7010F
:1098A0000E9463AA482F50E060E070E049835A8329
:1098B0006B837C83682F70E0C7010F94D028CDBFE5
:1098C000DEBF8823C9F049815A819E01275F3F4F3F
:1098D000B701CE010B960F94AF4A8DE0F70180835C
:1098E0008AE081839E01275F3F4F42E050E0B7014D
:1098F000CE010B960F94AF4ABE016F5F7F4FC70139
:109900000E945D4349815A819E01275F3F4FB70105
:10991000CE010B960F94AF4A6BE370E0C7010E9433
:10992000B6A9A0E0B0E089839A83AB83BC830E9490
:10993000A82A81110EC0F70101900020E9F73197A4
:10994000AF014E195F0920E0B7018EE399E30F9450
:109950006A2149815A816B817C81411551056105DC
:109960007105C1F09E01275F3F4FB701CE010B96F5
:109970000F94AF4A8DE0D7018C938AE011968C93B7
:109980009E01275F3F4F42E050E0B701CE010B96AA
:109990000F94AF4ACE010B960F945D4C0E94A059D4
:1099A00019821A821B821C822DA53EA54FA558A99B
:1099B000232B242B252B09F433C180E090E0DC011C
:1099C0000F2EFDEE2F2EF3E23F2EF02D0F2EFFEB8C
:1099D0008F2EF3E29F2EF02D880F991FAA1FBB1F19
:1099E000BC01CD017E5F8F4F9F4F0E94A8590E94FE
:1099F000335C8111FCCF80E091E0E7E1F3E4DF012B
:109A00009C011D9221503040E1F76F010F2EF7E1CC
:109A1000AF2EF4E4BF2EF02D8F010E9477A9D8015C
:109A20008D939D938D01AA16BB06B9F70E94735AB8
:109A30000F94972ACE010B960F945D4C412C512C1C
:109A40003201F601619171916F01AE014B5F5F4F81
:109A50008BA50E945015882309F496C088858F93A2
:109A60008F818F938E818F938D818F9389819A813E
:109A7000AB81BC81840D951DA61DB71DBF93AF930F
:109A80009F938F939F928F92FF92EF920F94B8566D
:109A9000F70101900020E9F73197AF014E195F09F6
:109AA0009E01275F3F4FB701CE010B960F94AF4A3F
:109AB000182FCDBFDEBF882309F48CC00E94A82ACE
:109AC000811126C089819A81AB81BC81840D951D4D
:109AD000A61DB71DBF93AF939F938F931F921F93A4
:109AE00049EC53E25F934F93FF92EF920F94B85675
:109AF000F70101900020E9F73197AF014E195F0996
:109B000020E0B7018EE399E30F946A21CDBFDEBF59
:109B1000F70101900020E9F73197AF014E195F0975
:109B20009E01275F3F4FB701CE010B960F94AF4ABE
:109B3000182F0E94A82A81114DC089819A81AB817A
:109B4000BC81840D951DA61DB71DBF93AF939F9338
:109B50008F931F921F93EAEDF3E2FF93EF93FF922F
:109B6000EF920F94B856F70101900020E9F7319772
:109B7000AF014E195F0920E0B7018EE399E30F941E
:109B80006A21CDBFDEBF26C00E94A82A811122C053
:109B900089819A81AB81BC81840D951DA61DB71D5D
:109BA000BF93AF939F938F933F922F92FF92EF9229
:109BB0000F94B856F70101900020E9F73197AF01F3
:109BC0004E195F0920E0B7018EE399E30F946A21F3
:109BD000CDBFDEBF9FEF491A590A690A790AA0E88A
:109BE0004A1651046104710409F02BCFCE010B9683
:109BF0000F945D4C89819A81AB81BC8180589F4FC5
:109C0000AF4FBF4F89839A83AB83BC832DA53EA5FD
:109C10004FA558A982179307A407B50708F4DCCE0F
:109C2000CE010B960F945D4CCE010B960F94A44C75
:109C30001092293388E193E30E94605639A93111CB
:109C400017C00F94B5098BE89CE30E94F3228111A1
:109C50000F9484198BE89CE30E94402A81E012C093
:109C600080E010C080E00EC080E00CC080E00AC040
:109C700081E008C00F2EFBE8CF2EFBE1DF2EF02D98
:109C800010E0C0CCE196CDBFDEBFDF91CF911F9138
:109C90000F91FF90EF90DF90CF90BF90AF909F908B
:109CA0008F907F906F905F904F903F902F9008958E
:109CB000CF92DF92EF92FF920F931F93CF93DF9398
:109CC0001F921F92CDB7DEB7009709F457C06115F8
:109CD000710509F453C07B018C01AE014F5F5F4FEA
:109CE000BC0180E594E10E94E83F882309F446C066
:109CF00089819A816C012FEFC21AD20AF801E80F0C
:109D0000F91F20E22083B8016C0D7D1DAE014F5F6D
:109D10005F4F89E394E10E94E83F882379F18981CC
:109D20009A81C80ED91EF801EC0DFD1D8DE08083CF
:109D300082E0C80ED11C8AE08183B8016C0D7D1DC4
:109D4000AE014F5F5F4F8BE094E10E94E83F8823B4
:109D5000A9F089819A81C80ED91EF801EC0DFD1D6C
:109D60008DE0808322E0C20ED11C8AE08183F8015D
:109D7000EC0DFD1D1082F701C082D1820F900F9073
:109D8000DF91CF911F910F91FF90EF90DF90CF90D7
:109D90000895EF92FF920F931F93CF93DF93CDB768
:109DA000DEB7A297CDBFDEBF009709F451C06115A1
:109DB000710509F44FC07B018C0160E0CE01039670
:109DC00015D7882309F44BC0B701C80171DFF7012B
:109DD000408151819E012F5F3F4FB801CE01039614
:109DE0000F94AF4ACE0103960F945D4CF70120818A
:109DF000318189819A812817390771F5BE016D5F1C
:109E00007F4FC801AADAA701B80183EC9BE10E9449
:109E1000E83F813099F4F701408151819E012F5F25
:109E20003F4FB801CE0103960F94AF4AF70120814E
:109E3000318189819A812817390781F4CE010396EF
:109E40000F94A44C81E012D70F941B1C81E007C033
:109E500080E005C080E003C080E001C080E0A29601
:109E6000CDBFDEBFDF91CF911F910F91FF90EF909B
:109E700008950F931F93CF93DF931F921F92CDB737
:109E8000DEB70F941B1C8091CD3E823009F462C076
:109E900028F4882359F0813081F1D6C0843009F448
:109EA00085C008F464C08A30E1F0CEC060E080E193
:109EB00090E47FD5811107C06091CE3E8BE89CE392
:109EC0000E943C14C9C00F947B01811104C081E041
:109ED0008093CD3EC1C08AE08093CD3E0F942C1A72
:109EE000BBC00F94431A6C3D75408105910508F481
:109EF000B3C081E08093CD3EAFC040E06FEB7CE328
:109F000081EC9CE30E944E400BE81CE3F80144A95D
:109F100055A99E012F5F3F4F61EC7CE380E190E407
:109F20000F94AF4A80E190E40F945D4CF80124A9AE
:109F300035A989819A812817390741F01092CD3EC1
:109F40006091CE3EC8010E943C1486C082E080939E
:109F5000CD3E82C000E021E040E150E46FEB7CE3C5
:109F600081EC9CE39FD983E08093CD3E75C04FEB9D
:109F70005CE361EC7CE383EC9BE10E94E83F813091
:109F800069F44091BF3C5091C03C9E012F5F3F4F10
:109F900061EC7CE380E190E40F94AF4A80E190E4CF
:109FA0000F94A44C84E08093CD3E56C00E9480D391
:109FB000882381F10F94761B8823C9F00E9420200A
:109FC000882309F449C08BE89CE30E94F3228111A5
:109FD0000F9484198BE89CE30E94402A1092CD3E96
:109FE0006091CE3E8BE89CE30E943C1435C08BE828
:109FF0009CE30E94F32281110F9484198BE89CE367
:10A000000E94402A1092CD3E61E08BE89CE30E94C2
:10A010003C1422C00F94BE19672B682B692BE1F406
:10A020008BE89CE30E94F32281110F9484198BE842
:10A030009CE30E94402A1092CD3E6091CE3E8BE878
:10A040009CE30E943C1408C01092CD3E6091CE3E2D
:10A050008BE89CE30E943C140F900F90DF91CF910E
:10A060001F910F9108959F92AF92BF92CF92DF926E
:10A07000EF92FF920F931F93CF93DF9300D0CDB752
:10A08000DEB7009709F471C06115710509F46DC060
:10A09000A42E6B017C018EE0E8EFF3E2D701019082
:10A0A0000D928A95E1F7F70101900020E9F73197C9
:10A0B000EE19FF09E983AF0155279E012E5F3F4F3F
:10A0C000B701C6010F94AF4AB12C0F2EFCE29F2EB0
:10A0D000F02D8B2D0E94FCC88B019C0148E0BE0135
:10A0E0006F5F7F4FC7010F94EE2882E08B1550F011
:10A0F0008981F701E80FF11D90828F5FF701E80F6A
:10A10000F11D1082F70101900020E9F73197EE1957
:10A11000FF09E983AF0155279E012E5F3F4FB7012D
:10A12000C6010F94AF4A898190E02A813B81821752
:10A13000930721F4B394E4E0BE12CBCFAA2081F0C0
:10A140008DE0F70180838AE0818382E089839E012C
:10A150002E5F3F4F42E050E0B701C6010F94AF4A77
:10A16000C6010F945D4C0F941B1C2396CDBFDEBF20
:10A17000DF91CF911F910F91FF90EF90DF90CF90E3
:10A18000BF90AF909F9008959F92AF92BF92CF9251
:10A19000DF92EF92FF920F931F93CF93DF931F9263
:10A1A0001F92CDB7DEB7009709F4E1C061157105C4
:10A1B00009F4DFC04115510509F4DDC0902E122FBE
:10A1C0005A016B017C010F941B1C41E0B601C701D1
:10A1D0000E944E40F601408151819E012F5F3F4F0A
:10A1E000B701C5010F94AF4AC5010F945D4CF6014C
:10A1F0002081318189819A812817390709F0BDC0F2
:10A200008DE0E6E0F4E2D70101900D928A95E1F746
:10A21000F70101900020E9F73197AF014E195F096E
:10A2200055279E012F5F3F4FB701C5010F94AF4ADD
:10A23000C5010F945D4CB501C7018FD88DE0F701C2
:10A2400080838AE081839E012F5F3F4F42E050E090
:10A25000B701C5010F94AF4AC5010F945D4C41E0B1
:10A26000B501C70100DFA601B7018BE89CE30E949E
:10A270000D41F601408151819E012F5F3F4FB70193
:10A28000C5010F94AF4AC5010F945D4CF6012081C2
:10A29000318189819A812817390709F070C0B60188
:10A2A000C7010E945941F601408151819E012F5FF3
:10A2B0003F4FB701C5010F94AF4AC5010F945D4CE4
:10A2C000F6012081318189819A812817390709F0A7
:10A2D00058C001E021E0A501B601C7010E94524922
:10A2E00021E0A501B601C7010E9437440E94E54262
:10A2F000882331F0492DB601C7010E94ED4206C006
:10A30000292D412FB601C7010E94F741F601408176
:10A3100051819E012F5F3F4FB701C5010F94AF4A96
:10A32000C5010F945D4CF6012081318189819A81AC
:10A330002817390741F5B601C7010E945D43F601B0
:10A34000408151819E012F5F3F4FB701C5010F949E
:10A35000AF4AC5010F945D4C81E0F6014081518107
:10A3600029813A814217530779F080E00DC080E0DF
:10A370000BC080E009C080E007C080E005C080E03D
:10A3800003C080E001C080E00F900F90DF91CF917B
:10A390001F910F91FF90EF90DF90CF90BF90AF9003
:10A3A0009F9008952F923F924F925F926F927F926B
:10A3B0008F929F92AF92BF92CF92DF92EF92FF92D5
:10A3C0000F931F93CF93DF93CDB7DEB7A897CDBF81
:10A3D000DEBF4115510509F4D7C12115310509F436
:10A3E000D5C16115710509F4D3C1280169011A01AC
:10A3F0007B0188A70F941B1CA60168E173E3CE01C3
:10A400000796A7D6882309F4C5C141E0BE016B5F5A
:10A410007F4FC1010E944E404D815E819E012B5FA6
:10A420003F4FB101CE0107960F94AF4ACE01079678
:10A430000F945D4CBE01695F7F4FC1010E94AD4921
:10A440001DE0F10110830AE001839E012B5F3F4F65
:10A4500042E050E0B101CE0107960F94AF4ACE0121
:10A4600007960F945D4CE8E1F3E3118B028B9E019C
:10A470002B5F3F4F43E150E0BF01CE0107960F94A1
:10A48000AF4ACE0107960F945D4C0F2EFBE8CF2EFE
:10A49000FBE1DF2EF02D10E001E021E0A101612FB2
:10A4A000C6010E949444882381F0F10101900020AC
:10A4B000E9F73197AF01421953099E012B5F3F4FD6
:10A4C000B101CE0107960F94AF4AF2E0CF0ED11C36
:10A4D0001F5F133009F70F2EFDE9CF2EFBE1DF2EB2
:10A4E000F02D19E001E021E0A101612FC6010E94D9
:10A4F0009444882381F0F10101900020E9F731971D
:10A50000AF01421953099E012B5F3F4FB101CE01AC
:10A5100007960F94AF4A22E0C20ED11C1F5F1B307A
:10A5200009F70F2EF2E18F2E912CA12CB12CF02DDA
:10A5300088E188169104A104B10491F401E021E0BE
:10A54000A10169E18DEB9BE10E949444811116C049
:10A550000F2EFCE18F2E912CA12CB12CF02D31C0AF
:10A5600001E021E0A101682DC401880F991F8557E2
:10A57000944E0E9494448823C1F007C00F2EF9E145
:10A580008F2E912CA12CB12CF02DF10101900020E7
:10A59000E9F73197AF01421953099E012B5F3F4FF5
:10A5A000B101CE0107960F94AF4A93E0890E911C3A
:10A5B000A11CB11CEAE18E169104A104B10408F4B7
:10A5C000B7CF1F92F8A5FF9383E194E29F938F93F7
:10A5D0003F922F920F94B856F10101900020E9F7B5
:10A5E0003197AF01421953099E012B5F3F4FB101D3
:10A5F000CE0107960F94AF4ACE0107960F945D4C9B
:10A60000612C712C0F900F900F900F900F900F9066
:10A61000411451046104710409F4A7C08701750154
:10A620006401812C912C5401F80141915191619167
:10A6300071918F019E012F5F3F4F88A50E942A2FA5
:10A64000882309F482C08C818F938B818F938A81B8
:10A650008F9389818F93BF92AF929F928F928FEB4E
:10A6600093E29F938F933F922F920F94B856F101EC
:10A6700001900020E9F73197AF01421953099E017B
:10A680002B5F3F4FB101CE0107960F94AF4A8FA3C6
:10A69000CDBFDEBF9FA1992309F457C00E94A82A0D
:10A6A00081111FC0FF92EF92DF92CF921F92EFA114
:10A6B000EF9389EC93E29F938F933F922F920F94A5
:10A6C000B856F10101900020E9F73197AF01421926
:10A6D000530920E0B1018EE399E30F946A21CDBFC5
:10A6E000DEBFF10101900020E9F73197AF01421977
:10A6F00053099E012B5F3F4FB101CE0107960F9486
:10A70000AF4A8FA30E94A82A81111FC0FF92EF9227
:10A71000DF92CF921F929FA19F93EAEDF3E2FF9306
:10A72000EF933F922F920F94B856F10101900020C1
:10A73000E9F73197AF014219530920E0B1018EE3E7
:10A7400099E30F946A21CDBFDEBF9FEF891A990A62
:10A75000A90AB90AEFEFCE1ADE0AEE0AFE0A84143D
:10A760009504A604B70408F45FCFCE0107960F94B2
:10A770005D4CCE0107960F94A44C1092293388E1CA
:10A7800093E39ED281E007C080E005C080E003C073
:10A7900080E001C080E0A896CDBFDEBFDF91CF9101
:10A7A0001F910F91FF90EF90DF90CF90BF90AF90EF
:10A7B0009F908F907F906F905F904F903F902F90E1
:10A7C0000895089580912D330895089510922D33A2
:10A7D00080912C33882331F010922C3380E390E465
:10A7E0000D94A44C089580E390E40D94A44C089536
:10A7F00080912C330895CF92DF92EF92FF921F93B6
:10A80000CF93DF93CDB7DEB76897CDBFDEBF6C01C6
:10A810007B0184E1EEE1F4E2DE01159601900D92F8
:10A820008A95E1F7DA01C9010196A11DB11D883EA3
:10A8300023E09207A105B1050CF460C01F921F929E
:10A840001F9281E08F9384EE90E29F938F93CE01CD
:10A8500001969F938F930F94B8568981898B8A8133
:10A860008A8B8B818B8B80E38D838AE38E83CDBF34
:10A87000DEBFE114F10459F0D701FE0138969E01C4
:10A88000245F3F4F8D918193E217F307D9F710E3CF
:10A8900046E0BE016B5F7F4F80E390E40F94114868
:10A8A00099EF980F9230C8F48B89893399F48A898B
:10A8B000893361F48989893321F410922C3380E043
:10A8C0003CC08F5F898B1A8B1B8BE2CF1B8B8F5FFA
:10A8D0008A8BDECF8F5F8B8BDBCF882321F01092AA
:10A8E0002C3380E02AC081E080932C33BE01695F65
:10A8F0007F4FC6010F949A5681E01FC0BF93AF935C
:10A900009F938F9384EE90E29F938F93CE01019655
:10A910009F938F930F94B8568981898B8A818A8BF4
:10A920008B818B8B80E38D838AE38E83CDBFDEBFEB
:10A93000E114F10409F0A0CFAACF6896CDBFDEBF25
:10A94000DF91CF911F91FF90EF90DF90CF9008950E
:10A9500080E00F94C201882361F08250823030F58C
:10A9600080912D33882311F110922D3310922C33C6
:10A97000089580912D33811119C081E080932D338A
:10A980008EE292E0EEE2F3E3DF019C011D922150A2
:10A990003040E1F7BF0180E00F94F3478B3019F4AA
:10A9A00010922C33089581E080932C3308958AE02F
:10A9B0000895CF93DF93CDB7DEB76097CDBFDEBFED
:10A9C000009719F120E329832AE32A832BE0E2E3AD
:10A9D000F4E2DE01139601900D922A95E1F76130C1
:10A9E00041F441E0BE016F5F7F4F0F941148982FF3
:10A9F00007C04AE0BE016F5F7F4F0F941148982F48
:10AA000081E0992319F080E001C080E06096CDBF1D
:10AA1000DEBFDF91CF910895DF92EF92FF920F9307
:10AA20001F93CF93DF93CDB7DEB76497CDBFDEBF63
:10AA30008C0184E1EDE3F4E2DE01119601900D92C8
:10AA40008A95E1F70115110509F449C061157105F1
:10AA500009F447C080E389838AE38A83411551055D
:10AA600059F0DA01FE0134969E01285F3F4F9D9117
:10AA70009193E217F307D9F77B010F2EF0E3DF2E56
:10AA8000F02D46E0BE016F5F7F4FC8010F94114863
:10AA900099EF980F9230A8F49F85993379F48E85B9
:10AAA000893341F48D858933F1F08F5F8D87DE86A0
:10AAB000DF86E7CFDF868F5F8E87E3CF9F5F9F873D
:10AAC000E0CF811112C081E1FE013396D7010190E0
:10AAD0000D928A95E1F7F701118A81E007C080E0C5
:10AAE00005C080E003C080E001C080E06496CDBF77
:10AAF000DEBFDF91CF911F910F91FF90EF90DF901C
:10AB00000895DF92EF92FF920F931F93CF93DF93FD
:10AB1000CDB7DEB76497CDBFDEBF8C0184E1E1E540
:10AB2000F4E2DE01119601900D928A95E1F701158C
:10AB3000110509F449C06115710509F447C080E3A6
:10AB400089838AE38A834115510559F0DA01FE01B0
:10AB500034969E01285F3F4F9D919193E217F30732
:10AB6000D9F77B010F2EF0E3DF2EF02D46E0BE017A
:10AB70006F5F7F4FC8010F94114899EF980F923083
:10AB8000A8F49F85993379F48E85893341F48D85B6
:10AB90008933F1F08F5F8D87DE86DF86E7CFDF8632
:10ABA0008F5F8E87E3CF9F5F9F87E0CF811112C0B9
:10ABB00081E1FE013396D70101900D928A95E1F76C
:10ABC000F701118A81E007C080E005C080E003C082
:10ABD00080E001C080E06496CDBFDEBFDF91CF9101
:10ABE0001F910F91FF90EF90DF9008950F931F93A7
:10ABF000CF93DF93CDB7DEB76097CDBFDEBF0097B1
:10AC000061F18C0180E389838AE38A838BE0E5E646
:10AC1000F4E2DE01139601900D928A95E1F761301E
:10AC200049F441E0BE016F5F7F4FC8010F941148A6
:10AC3000982F0EC041E060E0CE0103960F94814E44
:10AC40004AE0BE016F5F7F4FC8010F941148982FF3
:10AC500081E0992319F080E001C080E06096CDBFCB
:10AC6000DEBFDF91CF911F910F910895CF93DF93B6
:10AC7000CDB7DEB76097CDBFDEBF9BE0E5E6F4E27F
:10AC8000DE01119601900D929A95E1F7813041F421
:10AC900041E061E0CE0101960F94814E982F07C0EC
:10ACA00041E060E0CE0101960F94814E982F81E043
:10ACB000911180E06096CDBFDEBFDF91CF91089506
:10ACC000009721F041E061E00D94814E08951F93BB
:10ACD000CF93DF93CDB7DEB76497CDBFDEBF0097CC
:10ACE00001F1162FBC0180E389838AE38A83CE01B8
:10ACF00003960F949A56113041F441E061E0CE0181
:10AD000001960F94814E982F07C041E060E0CE017C
:10AD100001960F94814E982F81E0992319F080E0DD
:10AD200001C080E06496CDBFDEBFDF91CF911F915F
:10AD30000895EF92FF920F931F93CF93DF93CDB7B8
:10AD4000DEB76497CDBFDEBF6115710589F100974D
:10AD500089F18B017C0180E389838AE38A83CE01B8
:10AD600003960F949A5643E0BE016F5F7F4FC70171
:10AD70000F941148873069F460E0C801A8DF982F6C
:10AD80008823D9F043E0BE016F5F7F4FC7010F9466
:10AD90001148811111C0F70142855385648575857D
:10ADA000C7010F94AF4C91E0882339F090E005C0C3
:10ADB00090E003C090E001C090E0892F6496CDBF81
:10ADC000DEBFDF91CF911F910F91FF90EF9008951B
:10ADD000CF93DF93CDB7DEB76097CDBFDEBF0097CF
:10ADE000C1F020E329832AE32A832AE0E0E7F4E2A2
:10ADF000DE01139601900D922A95E1F741E0BE0124
:10AE00006F5F7F4F0F94114891E0882319F090E015
:10AE100001C090E0892F6096CDBFDEBFDF91CF915A
:10AE200008953F924F925F926F927F928F929F927E
:10AE3000AF92BF92CF92DF92EF92FF920F931F9348
:10AE4000CF93DF93CDB7DEB76197CDBFDEBF61157E
:10AE5000710509F470C0009709F46FC041155105E0
:10AE600009F46DC03FEF320F383008F06AC0322E5F
:10AE70007A018C01FB01138A41E00F941148811182
:10AE800062C0F8014285538564857585483EF3E0CC
:10AE90005F076105710508F458C0413B84E058071D
:10AEA0006105710508F053C0C32CD12C5601E6E0B2
:10AEB000AE0EB11C25010B2C000C66087708441956
:10AEC000550966097709C8010F94AF4C811141C03B
:10AED000A50160E070E0CE0103960F9493569E01A9
:10AEE0002F5F3F4FA501BE016D5F7F4FC8010F94DB
:10AEF0006349C8010F94A44CFE01EC0DFD1D1286A0
:10AF00008E010D5F1F4F812C912C5401A601B801B9
:10AF1000C7010F947D56892BF1F0FFEF8F1A9F0A1E
:10AF2000AF0ABF0A0F5F1F4F481459046A047B041D
:10AF300068F780E011C080E00FC080E00DC080E0C5
:10AF40000BC080E009C080E007C081E005C080E060
:10AF500003C080E001C081E06196CDBFDEBFDF911C
:10AF6000CF911F910F91FF90EF90DF90CF90BF9006
:10AF7000AF909F908F907F906F905F904F903F9099
:10AF800008954F925F926F927F92AF92BF92CF924D
:10AF9000DF92EF92FF920F931F93CF93DF93CDB782
:10AFA000DEB76897CDBFDEBF680114E1EEE1F4E2E1
:10AFB000DE01159601900D921A95E1F7009709F4BC
:10AFC00091C0C114D10409F48FC0EFEFEE0DE83049
:10AFD00008F08CC0860129013A015B016C01283E12
:10AFE00083E03807410551050CF482C01F921F927F
:10AFF0001F9281E08F9384EE90E29F938F93CE0116
:10B0000001969F938F930F94B8568981898B8A817B
:10B010008A8B8B818B8B80E38D838AE38E83CDBF7C
:10B02000DEBFA114B10459F0D501FE0138969E018E
:10B03000245F3F4F8D918193E217F307D9F70F2ECD
:10B04000F0E3FF2EF02D46E0BE016B5F7F4F80E303
:10B0500090E40F94114899EF980F923090F52E2DAF
:10B06000A801BE016B5F7F4F80E390E4DADE8823A6
:10B0700079F060E0C6012BDE882351F04AE0BE0182
:10B080006B5F7F4F80E390E40F9411488823F9F0C1
:10B090009B89993399F48A89893361F48989893341
:10B0A00021F410922C3380E042C08F5F898BFA8AA2
:10B0B000FB8AC9CFFB8A8F5F8A8BC5CF9F5F9B8B33
:10B0C000C2CF882321F010922C3380E030C081E081
:10B0D00080932C33BE01695F7F4FC6010F949A564F
:10B0E00081E025C080E023C080E021C080E01FC057
:10B0F0007F926F925F922F9384EE90E29F938F9353
:10B10000CE0101969F938F930F94B8568981898BB6
:10B110008A818A8B8B818B8B80E38D838AE38E83FC
:10B12000CDBFDEBFA114B10409F07ECF88CF6896F1
:10B13000CDBFDEBFDF91CF911F910F91FF90EF90B8
:10B14000DF90CF90BF90AF907F906F905F904F90C7
:10B150000895DF92EF92FF920F931F93CF93DF93A7
:10B16000CDB7DEB76497CDBFDEBF8C0184E1EAE7DF
:10B17000F4E2DE01119601900D928A95E1F7011536
:10B18000110509F449C06115710509F447C080E350
:10B1900089838AE38A834115510559F0DA01FE015A
:10B1A00034969E01285F3F4F9D919193E217F307DC
:10B1B000D9F77B010F2EF0E3DF2EF02D46E0BE0124
:10B1C0006F5F7F4FC8010F94114899EF980F92302D
:10B1D000A8F49F85993379F48E85893341F48D8560
:10B1E0008933F1F08F5F8D87DE86DF86E7CFDF86DC
:10B1F0008F5F8E87E3CF9F5F9F87E0CF811112C063
:10B2000081E1FE013396D70101900D928A95E1F715
:10B21000F701118A81E007C080E005C080E003C02B
:10B2200080E001C080E06496CDBFDEBFDF91CF91AA
:10B230001F910F91FF90EF90DF90089580915C3502
:10B2400008950895089581E080935C3508951092E3
:10B250005C350895CF92DF92EF92FF920F931F9388
:10B260006623B9F081111DC0C12CD12C760100E0FC
:10B2700010E62AEE30E040E06CE170E280EB98E00E
:10B280000F948B346CE170E280EB98E00F94D5342E
:10B2900008C0811106C06CE170E280EB98E00F9469
:10B2A000EB341F910F91FF90EF90DF90CF900895B6
:10B2B000CF93DF931F921F92CDB7DEB780915D359C
:10B2C00090915E35A0915F35B0916035072E75E1A4
:10B2D000B695A795979587957A95D1F7702D61E0EA
:10B2E000B9DF87ED8A8341E050E0BE016E5F7F4F9A
:10B2F00080EB98E00F94A63441E050E0BE016F5F10
:10B300007F4F80EB98E00F94BD3489818823A4F7A8
:10B3100080915D3590915E35A0915F35B09160353B
:10B32000072E75E1B695A795979587957A95D1F7EC
:10B33000702D60E08FDF0F900F90DF91CF91089517
:10B3400080EB98E00F9454341092613581E00895B9
:10B350001F93CF93DF93CDB7DEB72C97CDBFDEBF62
:10B360006115710520E28207910508F0A1C0DC019A
:10B37000CB0180935D3590935E35A0935F35B0939C
:10B38000603580916135811193DF10926135809134
:10B390005D3590915E35A0915F35B0916035072E97
:10B3A00075E1B695A795979587957A95D1F7702D04
:10B3B00061E050DF82ED8C8741E050E0BE01645FC8
:10B3C0007F4F80EB98E00F94A63480915D3590918B
:10B3D0005E35A0915F35B0916035AC01BD01032EA3
:10B3E00039E076956795579547953A95D1F7302D81
:10B3F000032E3AE0440F551F661F771F3A95D1F789
:10B40000302D9170AA27BB27842B952BA62BB72B09
:10B4100089839A83AB83BC838B818D8341E050E029
:10B42000BE016B5F7F4F80EB98E00F94A6348A815A
:10B430008E8341E050E0BE016A5F7F4F80EB98E071
:10B440000F94A63489818F8341E050E0BE01695F8B
:10B450007F4F80EB98E00F94A63415E5188741E004
:10B4600050E0BE01685F7F4F80EB98E00F94A634F8
:10B47000198741E050E0BE01675F7F4F80EB98E0A5
:10B480000F94A6341A8741E050E0BE01665F7F4FFB
:10B4900080EB98E00F94A6341B8741E050E0BE019A
:10B4A000655F7F4F80EB98E00F94A63481E001C088
:10B4B00080E02C96CDBFDEBFDF91CF911F91089524
:10B4C000052E59E0660F771F881F991F5A95D1F7EF
:10B4D000502D6115710520E28207910510F438CFD7
:10B4E000089580E0089580915D3590915E35A0913A
:10B4F0005F35B09160350097A105B10569F00197FE
:10B50000A109B109072E75E1B695A795979587957D
:10B510007A95D1F7702D01C080E060E09BDE10923B
:10B5200061350895CF93DF93CDB7DEB72897CDBFB0
:10B53000DEBF6115710520E28207910508F078C031
:10B54000DC01CB0180935D3590935E35A0935F3530
:10B55000B0936035809161358111AADE109261351A
:10B5600080915D3590915E35A0915F35B0916035E9
:10B57000072E75E1B695A795979587957A95D1F79A
:10B58000702D61E067DE82E8888741E050E0BE010F
:10B59000685F7F4F80EB98E00F94A63480915D3513
:10B5A00090915E35A0915F35B0916035AC01BD01E1
:10B5B000032E39E076956795579547953A95D1F7DB
:10B5C000302D032E3AE0440F551F661F771F3A9522
:10B5D000D1F7302D9170AA27BB27842B952BA62B52
:10B5E000B72B89839A83AB83BC838B818D8341E0A6
:10B5F00050E0BE016B5F7F4F80EB98E00F94A63464
:10B600008A818E8341E050E0BE016A5F7F4F80EB0C
:10B6100098E00F94A63489818F8341E050E0BE0109
:10B62000695F7F4F80EB98E00F94A63481E001C002
:10B6300080E02896CDBFDEBFDF91CF910895CF93F4
:10B64000DF931F92CDB7DEB780915D3590915E3567
:10B65000A0915F35B0916035AC01BD015170662796
:10B660007727452B462B472B31F1198241E050E0DB
:10B67000BE016F5F7F4F80EB98E00F94A6348091FE
:10B680005D3590915E35A0915F35B0916035019642
:10B69000A11DB11D80935D3590935E35A0935F35FC
:10B6A000B0936035AC01BD01517066277727452BFB
:10B6B000462B472BD1F60097A105B10569F00197FC
:10B6C000A109B109072E75E1B695A79597958795BC
:10B6D0007A95D1F7702D01C080E060E0BBDD81E09C
:10B6E000809361350F90DF91CF9108950F931F9351
:10B6F000CF93DF931F92CDB7DEB78091613588235A
:10B70000B1F01092613580915D3590915E35A091D8
:10B710005F35B0916035BC01CD01052E59E096959D
:10B720008795779567955A95D1F7502DC9DE41E0F9
:10B7300050E0BE016F5F7F4F80EB98E00F94BD3407
:10B7400080915D3590915E35A0915F35B091603507
:10B75000AC01BD014F5F5F4F6F4F7F4F40935D3531
:10B7600050935E3560935F35709360358A019B011D
:10B77000117022273327012B022B032BA1F4452B19
:10B78000462B472B51F0072E75E1B695A795979557
:10B7900087957A95D1F7702D01C080E060E05ADD81
:10B7A00081E08093613589810F90DF91CF911F9166
:10B7B0000F9108950F931F93CF93DF931F92CDB7EF
:10B7C000DEB7182F80916135882349F060915D358F
:10B7D00070915E3580915F3590916035A3DE19835D
:10B7E00041E050E0BE016F5F7F4F80EB98E00F9427
:10B7F000A63480915D3590915E35A0915F35B09112
:10B800006035AC01BD014F5F5F4F6F4F7F4F40937D
:10B810005D3550935E3560935F35709360358A0176
:10B820009B01117022273327012B022B032BA1F43C
:10B83000452B462B472B51F0072E75E1B695A79562
:10B84000979587957A95D1F7702D01C080E060E0DB
:10B8500001DD81E08093613581E00F90DF91CF9130
:10B860001F910F910895CF93DF931F921F92CDB731
:10B87000DEB780916135882309F440C080915D3541
:10B8800090915E35A0915F35B0916035072E75E1DE
:10B89000B695A795979587957A95D1F7702D61E024
:10B8A000D9DC87ED8A8341E050E0BE016E5F7F4FB7
:10B8B00080EB98E00F94A63441E050E0BE016F5F4A
:10B8C0007F4F80EB98E00F94BD3480915D3590916F
:10B8D0005E35A0915F35B0916035072E75E1B69564
:10B8E000A795979587957A95D1F7702D60E0B2DC92
:10B8F00089818095881F8827881F01C080E00F906C
:10B900000F90DF91CF910895CF93DF93EC01803CAE
:10B9100028E0920729F468E083E00F94D53310C043
:10B92000803C29E0920729F468E084E00F94D53345
:10B9300007C0803C9A4021F468E085E00F94D5333D
:10B94000888180618883DF91CF910895EF92FF9283
:10B950000F931F93CF937C01C42FB901A80100E07E
:10B9600010E62AEE30E00E94DA66882344F0F70100
:10B970008081CC0FCC0FCC70837FC82BC083CF913C
:10B980001F910F91FF90EF90089580E0089591E04E
:10B99000811101C090E09093504081E08093442059
:10B9A00008950F931F9305EA1EE52FE130E044EA66
:10B9B00055E361E082E00E945D77811105C061ED91
:10B9C0007CE582E00E94AD781F910F910895CF939E
:10B9D000DF9310928735109288350F9401358111CD
:10B9E00004C01092A035D0E012C081508093A035E1
:10B9F0002ADCD82F882359F0C0E060E08C2F0F9408
:10BA00001735CF5F8091A0358C17B8F7CADF8D2F1F
:10BA1000DF91CF910895C5CF08950F931F930BE049
:10BA20001DE52DE030E048E450E260E081E80E944E
:10BA30005D77811105C06DE07DE581E80E94AD78FC
:10BA40001F910F91089580918835882341F082E0FD
:10BA50000E94867863E27DE582E00C94AD780895DB
:10BA600080918835882341F081E80E94867860E3E0
:10BA70007DE581E80C94AD780895809150209091F7
:10BA80005120A0915220B0915320892B8A2B8B2BCF
:10BA900059F08091B035882324F481E80E9486789B
:10BAA00003C082E00E9486788091A8359091A935E4
:10BAB000A091AA35B091AB3580934C2090934D2046
:10BAC000A0934E20B0934F20A8CF0895ECE8F5E363
:10BAD00082E1DF011D928A95E9F780EF80838AE099
:10BAE00087830895DF92EF92FF920F931F93CF9376
:10BAF000DF93D82EC62FD72F122F032FF42EE52E2B
:10BB0000E5DF81E080935420ECE8F5E3D282E38224
:10BB1000F48205831683D487C587DF91CF911F9167
:10BB20000F91FF90EF90DF90089520E030E0A901A1
:10BB300060E074E285E0D6CF08950F931F932091C3
:10BB4000B03542276CF00091502010915120209187
:10BB5000522030915320061717072807390720F481
:10BB6000E4DF8BDF80E001C081E01F910F91089539
:10BB700020E030E0A90160E070E084E0B3CF0895F8
:10BB80000F931F93262F30E006EE1DE5AC0161E018
:10BB900081E80E945D77811102C0EADF6EDF1F91AC
:10BBA0000F91089520E030E0A90160E078E286E09E
:10BBB00099CF089520E030E0A90160E07AE382E0C7
:10BBC00091CF089583DF109254200895CF93DF938F
:10BBD000811111C0EB01F6DFE8E4F0E28085918588
:10BBE000A285B3858C1B9D0BA109B1098087918724
:10BBF000A287B38742DFDF91CF9108951F93CF9340
:10BC0000DF93D82F84E1ECE6F5E3DF011D928A95FE
:10BC1000E9F7DD2331F09091BB35E4E7F5E318E077
:10BC200005C09091B735E0E7F5E314E08091B535B4
:10BC30008F738C3111F08F3339F48CE180838AE07B
:10BC4000818385E08383145FC12F911708F4C92F86
:10BC50008C2F90E0A0E0B0E040E8BC01CD016DDFAA
:10BC6000882309F18091B1350F941E35811102C0EE
:10BC700020E001C020E8DD2361F0ECE6F5E3812F50
:10BC800090E00297982789279827808391832383C0
:10BC900006C0ECE6F5E38FEF810F808322836C2FE3
:10BCA0008CE695E36DDFDF91CF911F910895CF93DF
:10BCB000C82F81110FC08091B1350F941E35882394
:10BCC00049F020E030E0A90160E077E287E00ADF98
:10BCD000D4DE39C0A2E8B5E3E4EAF5E3818913963E
:10BCE0008C931397828912968C931297838911965D
:10BCF0008C93119784898C93A0E8B5E3868911967B
:10BD00008C93119787898C936091803570918135E0
:10BD1000CB01A0E0B0E0BC01CD01052E59E0660FDB
:10BD2000771F881F991F5A95D1F7502DC11102C056
:10BD300040E001C040E801DF882329F0C093863548
:10BD400081E080938735CF9108950F931F93CF9310
:10BD5000DF93811132C16F31710569F48091A4358F
:10BD60009091A535A091A635B091A735853593451D
:10BD7000A244B34431F081E08093883564DE70DE04
:10BD80001CC1E4EAF5E395859F7095878091A03505
:10BD9000891718F4CADE71DE10C1E4EAF5E34085C4
:10BDA0005185628573854093502050935120609354
:10BDB000522070935320478550E04B35510508F0D1
:10BDC000EEC0FA018827E958FE4F8F4F0D948B542F
:10BDD000C091B735C33108F0C2E18C2F90E0A0E0EC
:10BDE000B0E040E8BC01CD01A8DE882309F4E5C03D
:10BDF0006C2F8CE895E3C4DEE0C0C091B735C53246
:10BE000008F0C4E28C2F90E0A0E0B0E040E8BC0174
:10BE1000CD0193DE882309F4D0C08091B4358370BE
:10BE200021F4D091B535DD2319F07FDE26DEC5C0C3
:10BE30008091B1350F9425358111D0E800E210E2F0
:10BE4000F801D1838091B1350F942C3520E1FC01AC
:10BE50003196A0E3B0E201900D922A95E1F7F80146
:10BE60008089882309F4A4C0823209F4A3C0E1E3E5
:10BE7000F0E281E09191992309F49DC0923209F496
:10BE80009AC08F5F8031B1F708C0E82FF0E0E05E24
:10BE9000FF4D908B8F5F8031C1F76C2F80E290E275
:10BEA0006FDE8BC080E0AADE88C081E0A7DE85C09F
:10BEB000892F0F940335823039F0833019F08111C6
:10BEC00005C006C06FDE05C075DE03C051DE01C0CF
:10BED00079DED3DD72C040E868E070E080E090E099
:10BEE0002CDE882309F469C064E675E38091B135DE
:10BEF0000F940A35823041F0833019F0811107C068
:10BF000009C050DEBADD59C055DEB7DD56C030DE9F
:10BF1000B4DD53C0E4E6F5E380E090E0A2E0B0E0F9
:10BF200084839583A683B78380819181A281B38125
:10BF30005A2F4B2F60E070E0982789279827A0E0C0
:10BF4000B0E0DC0199278827842B952BA62BB72BF3
:10BF500080839183A283B38368E0CF0111DE2DC07B
:10BF60008091B73581FF06C08095682F6170892F59
:10BF70000F94173527DE81DD20C08091B735811100
:10BF800002C020DE01C0D1DD78DD17C01BDE75DD0B
:10BF900014C081E08CDE11C080E089DE0EC020E09C
:10BFA00030E0A90160E070E285E09CDD66DD05C05F
:10BFB00080E001C080E090E268CFDF91CF911F91D7
:10BFC0000F9108951092873542C908958091594084
:10BFD0008823F4F480768032D9F580915A408E3FE0
:10BFE000C9F580915F40909160400197A9F58091DB
:10BFF0005B4090915C40892B89F5E9E5F0E480EAAB
:10C0000095E38087918781E090E082879387089508
:10C010008076803229F580915A408F3F19F58091C2
:10C020005F4090916040892BF9F480915B40909142
:10C030005C40892BD9F4109288351092873582E0C4
:10C040000E941B7881E80E941B78ABDC81E0089598
:10C0500080E0089580E0089580E0089580E00895EC
:10C0600080E0089580E0089580E0089580E00895DC
:10C07000CF93C0918735CC23A9F110928735809159
:10C080008635882389F02091803530918135409123
:10C0900082355091833560918435709185358091DA
:10C0A000B1350F94343510C02091803530918135F1
:10C0B00040918235509183356091843570918535FA
:10C0C0008091B1350F945835823041F0833021F0A2
:10C0D000811106C077DD05C065DD03C06BDD01C0E1
:10C0E00047DDCBDC8C2FCF910895EF92FF920F9319
:10C0F0001F93CF93DF93982F80914420882309F4D6
:10C1000048C0109244202115310511F0890102C068
:10C1100007EC1CE5911102C082E001C081E8E90151
:10C120007A01AB01970160E00E945D77811104C044
:10C1300091E0909344202DC0CD2BD9F480914420E0
:10C140008823E1F380915040811122C0E8E4F0E2BD
:10C1500080859185A285B3858E199F09A109B109B2
:10C1600080879187A287B3879091504081E089278B
:10C1700010C0E8E4F0E240855185628573854E1970
:10C180005F0961097109408751876287738701C020
:10C1900080E0DF91CF911F910F91FF90EF90089574
:10C1A000E091C935F091CA350190F081E02D2281EE
:10C1B00033812E0F3F1FFC014081E40FF11DE21778
:10C1C000F307A0F481818430A1F0861306C014C067
:10C1D00081818430A1F08617A9F08081E80FF11DDC
:10C1E000E217F307A8F380E090E0089580E090E084
:10C1F000089580E090E008958E2F9F2F089580E0AD
:10C2000090E008958E2F9F2F089580915B408F7747
:10C210000C94787608959091CB35992381F1E09133
:10C22000C935F091CA350190F081E02D94818917CC
:10C2300040F5E093C735F093C835228133812E0F46
:10C240003F1FE217F307F8F49181943061F4928173
:10C25000891309C09381961306C0E093C735F09304
:10C26000C83581E008959081E90FF11DE217F307C9
:10C2700058F3E093C735F093C83580E0089580E027
:10C28000089580E0089580E00895EF92FF921F9353
:10C29000CF93DF93C82F60E0BEDF182F882381F192
:10C2A000A091C935B091CA35EC2FF0E0EE0FFF1F19
:10C2B00012968D919C911397E80FF91FE080F18001
:10C2C000D7011696ED91FC9117971995682F8C2F31
:10C2D000A2DF182F8823A1F0C091C735D091C835AF
:10C2E00065E0CE015DDFEC01892B21F08A810E949F
:10C2F0006A78F6CFD7011296ED91FC9113971995B4
:10C30000812FDF91CF911F91FF90EF9008951F93A0
:10C31000CF93DF93182F7FDF882341F1C091C7357A
:10C32000D091C83565E0CE013BDFEC01892B49F0A7
:10C330004C815D816B818A810E9485768111F2CF6B
:10C3400015C0A091C935B091CA35E12FF0E0EE0FCC
:10C35000FF1F12968D919C911397E80FF91F019082
:10C36000F081E02D0190F081E02D1995DF91CF91C2
:10C370001F9108950C9410760895CF938091CB353A
:10C380008823C1F0E091C935F091CA350190F08160
:10C39000E02D8481882371F0C0E08C2F76DFCF5FA1
:10C3A000E091C935F091CA350190F081E02D84818A
:10C3B000C81798F31092CB3581E090E08093CC358C
:10C3C0009093CD35CF9108950E94DC75D6CF089516
:10C3D000CF938091CB35882349F1A091C935B09195
:10C3E000CA35ED91FC91119784818823F9F0C0E062
:10C3F000EC2FF0E0EE0FFF1F12968D919C9113979A
:10C40000E80FF91F0190F081E02D0084F185E02D07
:10C41000309709F01995CF5FA091C935B091CA3511
:10C42000ED91FC9111978481C81710F3CF91089575
:10C430000F931F93CF93DF93E9E5F0E41286138601
:10C440001486158616861786808188230CF060C2B4
:10C4500020915F40309160402115310509F05DC2A7
:10C460004FC28F7109F097C090915A40963081F079
:10C47000983009F485C091118EC02230310509F041
:10C48000FBC162E070E08CEC95E30E947E764EC2C8
:10C4900080915B4090915C40292F332722303105F9
:10C4A00089F02330310579F12130310509F0A6C139
:10C4B0008091622090916320DC016C9170E00E9479
:10C4C0007E764FC0E0916220F0916320218982172F
:10C4D00008F0D2C19927880F991F880F991FE09102
:10C4E0006420F0916520E80FF91F80819181FC01A3
:10C4F000628173810E947E76E0916140F09162409A
:10C5000082E081832EC099278130910599F058F0FF
:10C510008230910509F406C2039709F078C13CE026
:10C52000EEE8F4E20AC064E070E088EC90E20E9479
:10C530007E7617C0EEEBF0E239E0A2EAB0E220E04E
:10C54000819190E08D939D932F5F2317C8F3632F04
:10C55000660F6E5F6093A02070E080EA90E20E9418
:10C560007E76E9E5F0E4868197812285338582171E
:10C57000930708F0DBC18093634090936440D6C179
:10C580002130310509F078C161E070E08BEC95E372
:10C590000E947E76CBC18130E9F590915A409A3065
:10C5A000C9F52130310509F037C18091CB35882399
:10C5B00009F432C1C0915D40D0915E400091C9350F
:10C5C0001091CA35D801ED91FC918481C81708F00B
:10C5D00023C160E08C2F1FDE882309F418C1CE012F
:10C5E0009927880F991FD8011296ED91FC91139706
:10C5F000E80FF91F0190F081E02D86819781FC0101
:10C6000019958093C63561E070E086EC95E30E9451
:10C610007E768CC1823009F0FAC080915A40811137
:10C62000EFC02230310509F027C180915D400E94A2
:10C630000D7790E08093C4359093C53562E070E04B
:10C6400084EC95E30E947E7671C18F7109F084C0FD
:10C6500090915A40933009F4D5C018F49130A1F06C
:10C660007BC0953019F0993039F176C080915F40E8
:10C6700090916040892B09F0FFC085E091E680939E
:10C6800065409093664052C180915F4090916040B8
:10C69000892B09F0F1C080915B4090915C4001973B
:10C6A00009F0EAC08091CC359091CD358D7F809393
:10C6B000CC359093CD353AC180915F4090916040E8
:10C6C000892B09F0D9C00E947B76882309F49FC08A
:10C6D00020915B4030915C403327E0916220F091E3
:10C6E0006320818990E08217930708F490C045DEAB
:10C6F00080915B4090915C408093CB35882309F416
:10C7000015C199278150904C880F991F880F991F48
:10C71000E0916420F0916520E80FF91FE093C9359E
:10C72000F093CA350190F081E02D8481882309F4CB
:10C73000FDC0C0E060E08C2FEADD882309F467C00B
:10C74000CF5FE091C935F091CA350190F081E02DBD
:10C750008481C81778F3EAC08130E9F490915A4097
:10C760009B30C9F480915F4090916040892B09F023
:10C7700053C08091CB35882309F44EC0E9E5F0E43D
:10C78000C481D2818C2F81DD882309F440C06D2FB4
:10C790008C2FBDDD3AC08230D1F580915A40813076
:10C7A00019F08330A1F030C080915F4090916040DB
:10C7B000892B09F061C080915B4090915C40892B8E
:10C7C00009F05AC080915D400E9428771EC0809178
:10C7D0005F4090916040892B09F04EC080915B4092
:10C7E00090915C40892B09F047C0C9E5D0E48C8169
:10C7F0000E941B788C810E94867807C080E005C06B
:10C8000080E003C080E001C080E0811190C0809191
:10C8100059408F71813081F58091CB35882309F49F
:10C8200071C000915D4010915E40C091C935D091BA
:10C83000CA35E881F9818481081708F065C060E095
:10C84000802FE9DC8823C1F0F801FF27CF01880F92
:10C85000991FEA81FB81E80FF91FC081D181EE8128
:10C86000FF811995682F802FD6DC882329F0EC8171
:10C87000FD81199581115BC0809159408F71823083
:10C8800009F044C08091CB358823B1F1A091C9351E
:10C89000B091CA35ED91FC9111978481882371F193
:10C8A000C0E0EC2FF0E0EE0FFF1F12968D919C91EF
:10C8B0001397E80FF91F00811181D8011696ED91A9
:10C8C000FC9117971995682F8C2FA5DC882379F197
:10C8D000D8011496ED91FC9115971995811127C0F7
:10C8E000CF5FA091C935B091CA35ED91FC911197F8
:10C8F0009481C917B0F21BC080E019C080E017C056
:10C9000080E015C080E013C080E011C080E00FC05F
:10C91000982F907609F07BCF98CE982F907609F0DB
:10C9200076CF9FCD33E0EAEBF0E207CE81E0DF91F6
:10C93000CF911F910F9108958038910558F1672B81
:10C9400021F4873C910571F41CC08F3F910509F0DB
:10C95000F8F49C01220F331FF901E55AF84D80814C
:10C9600091810895EDE5F8E221E030E041915191A7
:10C970008417950741F02F5F3F4F20383105B1F7FD
:10C9800002C020E030E020583F4FC90199270895A8
:10C9900080E090E008958136910589F0EDE7F6E2B8
:10C9A00040E050E04F5F5F4F2191319121153105FB
:10C9B00091F028173907B1F7892B19F40AC040E024
:10C9C00050E0440F551FFA01E556FB4D80819181DF
:10C9D000089580E090E0089543E050E060E880E052
:10C9E00096E00F942D3443E050E064E080E296E05E
:10C9F0000F942D3443E050E062E080E296E00F9423
:10CA00002D3440E058E160E280EA96E00F942D3446
:10CA100041E050E062E080EA96E00F942D3443E07C
:10CA200050E060E180E896E00F942D3443E050E060
:10CA300060E180E496E00F942D3441E050E061E045
:10CA400080E496E00F942D3441E050E062E080E411
:10CA500096E00F942D3441E050E060E280E696E0ED
:10CA60000F942D3441E050E062E080E096E00F94B6
:10CA70002D3443E050E062E080E696E00F942D34E0
:10CA800040E050E061E080EA96E00F942D3440E011
:10CA900050E061E080E096E00F942D3440E050E0FB
:10CAA00068E080E096E00F942D3441E050E060E4CF
:10CAB00080E096E00F942D3440E058E161E080E89A
:10CAC00096E00F942D3440E050E061E080E096E085
:10CAD0000F942D3440E050E060E280E096E00F9447
:10CAE0002D3440E050E064E080E096E00F942D3477
:10CAF00040E050E061E080EA96E00F942D3443E09E
:10CB000050E060E880E496E00F942D3443E050E07C
:10CB100060E280E496E00F942D3440E050E060E461
:10CB200080E496E00F942D3441E050E060E880E826
:10CB300096E00F942D3441E050E060E280E896E00A
:10CB40000F942D3440E050E060E480E896E00F94CC
:10CB50002D3443E050E068E080E496E00F942D34FB
:10CB600040E050E064E080E496E00F942D3443E030
:10CB700050E068E080E696E00F942D3440E050E00D
:10CB800064E080E696E00F942D3443E050E068E0E6
:10CB900080E896E00F942D3440E050E064E080E8B7
:10CBA00096E00F942D3443E050E068E080EA96E090
:10CBB0000F942D3440E050E064E080EA96E00F945A
:10CBC0002D3440E058E160E480EA96E00F942D3483
:10CBD00040E058E160E180E696E00F942D3440E0BB
:10CBE00058E161E080E296E00F942D3443E050E09C
:10CBF00060E880E496E00F942D3443E050E060E27A
:10CC000080E496E00F942D3440E050E060E480E44E
:10CC100096E00F942D3443E050E060E880EA96E01F
:10CC20000F942D3443E050E060E880E496E00F94E8
:10CC30002D3443E050E060E280E496E00F942D3420
:10CC400040E050E060E480E496E00F942D3443E04F
:10CC500050E068E080E296E00F942D3441E050E02F
:10CC600062E080E896E00F942D3440E050E061E00F
:10CC700080E696E00F942D3440E050E060E180E0E3
:10CC800096E00D942D3408951F920F920FB60F92D7
:10CC900011240BB60F928F939F93EF93FF93E1E5CF
:10CCA000F0E480819181019680839183FF91EF91DF
:10CCB0009F918F910F900BBE0F900FBE0F901F9002
:10CCC00018951F920F920FB60F9211240BB60F9268
:10CCD000CF92DF92EF92FF920F931F932F933F9388
:10CCE0004F935F936F937F938F939F93AF93BF9374
:10CCF000EF93FF93E1E5F0E480819181228133811C
:10CD000082179307F0F121E020930204E09157404D
:10CD1000F09158403097A9F160910804709109048E
:10CD2000A0E0B0E0DC0199278827AB0160E070E06B
:10CD30008C019D01042B152B262B372BC901B80123
:10CD4000A1E5B0E412960D911C91139720E030E01C
:10CD50009801112700271496CD90DC901597E12CAF
:10CD6000F12C0C291D292E293F2906171707280702
:10CD7000390730F0C901B8016F5F7F4F8F4F9F4F68
:10CD80001995FF91EF91BF91AF919F918F917F91F5
:10CD90006F915F914F913F912F911F910F91FF9054
:10CDA000EF90DF90CF900F900BBE0F900FBE0F90C3
:10CDB0001F901895CF92DF92EF92FF920F931F93DF
:10CDC000CF93DF93EC016A017B01DB01CA0101977C
:10CDD000A109B109BC01CD01600F711F821F931F12
:10CDE000A70196010F944D54213831054105510595
:10CDF000F8F4213460F4213260F4213160F42930F8
:10CE000060F4253060F4233060F490E80BC093E0C8
:10CE100009C092E007C092E805C091E003C091E824
:10CE200001C090E088818C77892B888381E001C0E4
:10CE30008FEFDF91CF911F910F91FF90EF90DF90D7
:10CE4000CF9008951F920F920FB60F9211240BB638
:10CE50000F922F933F934F935F936F937F938F9393
:10CE60009F93AF93BF93EF93FF93E0911436F091AC
:10CE70001536309709F01995FF91EF91BF91AF9159
:10CE80009F918F917F916F915F914F913F912F91E2
:10CE90000F900BBE0F900FBE0F901F9018951F9212
:10CEA0000F920FB60F9211240BB60F922F933F9350
:10CEB0004F935F936F937F938F939F93AF93BF93A2
:10CEC000EF93FF93E0911236F0911336309709F00B
:10CED0001995FF91EF91BF91AF919F918F917F91A4
:10CEE0006F915F914F913F912F910F900BBE0F90DB
:10CEF0000FBE0F901F9018951F920F920FB60F92B2
:10CF000011240BB60F922F933F934F935F936F9320
:10CF10007F938F939F93AF93BF93EF93FF93E09192
:10CF20001036F0911136309709F01995FF91EF9175
:10CF3000BF91AF919F918F917F916F915F914F9131
:10CF40003F912F910F900BBE0F900FBE0F901F902F
:10CF500018951F920F920FB60F9211240BB60F92D5
:10CF60002F933F934F935F936F937F938F939F93F1
:10CF7000AF93BF93EF93FF93E0910E36F0910F368E
:10CF8000309709F01995FF91EF91BF91AF919F9163
:10CF90008F917F916F915F914F913F912F910F9062
:10CFA0000BBE0F900FBE0F901F9018951F920F92FF
:10CFB0000FB60F9211240BB60F922F933F934F93FE
:10CFC0005F936F937F938F939F93AF93BF93EF93F1
:10CFD000FF93E0910C36F0910D36309709F01995DA
:10CFE000FF91EF91BF91AF919F918F917F916F9141
:10CFF0005F914F913F912F910F900BBE0F900FBEFD
:10D000000F901F9018951F920F920FB60F92112438
:10D010000BB60F922F933F934F935F936F937F9332
:10D020008F939F93AF93BF93EF93FF93E0910A3653
:10D03000F0910B36309709F01995FF91EF91BF9160
:10D04000AF919F918F917F916F915F914F913F91A0
:10D050002F910F900BBE0F900FBE0F901F90189541
:10D060001F920F920FB60F9211240BB60F922F93AF
:10D070003F934F935F936F937F938F939F93AF9360
:10D08000BF93EF93FF93E0910836F0910936309704
:10D0900009F01995FF91EF91BF91AF919F918F91F9
:10D0A0007F916F915F914F913F912F910F900BBEA8
:10D0B0000F900FBE0F901F9018951F920F920FB6F2
:10D0C0000F9211240BB60F922F933F934F935F93C0
:10D0D0006F937F938F939F93AF93BF93EF93FF9340
:10D0E000E0910636F0910736309709F01995FF91D7
:10D0F000EF91BF91AF919F918F917F916F915F91D0
:10D100004F913F912F910F900BBE0F900FBE0F903C
:10D110001F9018951F920F920FB60F9211240BB605
:10D120000F922F933F934F935F936F937F938F93C0
:10D130009F93AF93BF93EF93FF93E0910436F091E9
:10D140000536309709F01995FF91EF91BF91AF9196
:10D150009F918F917F916F915F914F913F912F910F
:10D160000F900BBE0F900FBE0F901F9018951F923F
:10D170000F920FB60F9211240BB60F922F933F937D
:10D180004F935F936F937F938F939F93AF93BF93CF
:10D19000EF93FF93E0910236F0910336309709F058
:10D1A0001995FF91EF91BF91AF919F918F917F91D1
:10D1B0006F915F914F913F912F910F900BBE0F9008
:10D1C0000FBE0F901F9018951F920F920FB60F92DF
:10D1D00011240BB60F922F933F934F935F936F934E
:10D1E0007F938F939F93AF93BF93EF93FF93E091C0
:10D1F0000036F0910136309709F01995FF91EF91C3
:10D20000BF91AF919F918F917F916F915F914F915E
:10D210003F912F910F900BBE0F900FBE0F901F905C
:10D2200018951F920F920FB60F9211240BB60F9202
:10D230002F933F934F935F936F937F938F939F931E
:10D24000AF93BF93EF93FF93E091FE35F091FF35DD
:10D25000309709F01995FF91EF91BF91AF919F9190
:10D260008F917F916F915F914F913F912F910F908F
:10D270000BBE0F900FBE0F901F9018951F920F922C
:10D280000FB60F9211240BB60F922F933F934F932B
:10D290005F936F937F938F939F93AF93BF93EF931E
:10D2A000FF93E091FC35F091FD35309709F0199529
:10D2B000FF91EF91BF91AF919F918F917F916F916E
:10D2C0005F914F913F912F910F900BBE0F900FBE2A
:10D2D0000F901F9018951F920F920FB60F92112466
:10D2E0000BB60F922F933F934F935F936F937F9360
:10D2F0008F939F93AF93BF93EF93FF93E091FA3592
:10D30000F091FB35309709F01995FF91EF91BF919E
:10D31000AF919F918F917F916F915F914F913F91CD
:10D320002F910F900BBE0F900FBE0F901F9018956E
:10D330001F920F920FB60F9211240BB60F922F93DC
:10D340003F934F935F936F937F938F939F93AF938D
:10D35000BF93EF93FF93E091F835F091F935309753
:10D3600009F01995FF91EF91BF91AF919F918F9126
:10D370007F916F915F914F913F912F910F900BBED5
:10D380000F900FBE0F901F9018951F920F920FB61F
:10D390000F9211240BB60F922F933F934F935F93ED
:10D3A0006F937F938F939F93AF93BF93EF93FF936D
:10D3B000E091F635F091F735309709F01995FF9126
:10D3C000EF91BF91AF919F918F917F916F915F91FD
:10D3D0004F913F912F910F900BBE0F900FBE0F906A
:10D3E0001F9018951F920F920FB60F9211240BB633
:10D3F0000F922F933F934F935F936F937F938F93EE
:10D400009F93AF93BF93EF93FF93E091F435F09127
:10D41000F535309709F01995FF91EF91BF91AF91D4
:10D420009F918F917F916F915F914F913F912F913C
:10D430000F900BBE0F900FBE0F901F9018951F926C
:10D440000F920FB60F9211240BB60F922F933F93AA
:10D450004F935F936F937F938F939F93AF93BF93FC
:10D46000EF93FF93E091F235F091F335309709F0A7
:10D470001995FF91EF91BF91AF919F918F917F91FE
:10D480006F915F914F913F912F910F900BBE0F9035
:10D490000FBE0F901F9018951F920F920FB60F920C
:10D4A00011240BB60F922F933F934F935F936F937B
:10D4B0007F938F939F93AF93BF93EF93FF93E091ED
:10D4C000F035F091F135309709F01995FF91EF9112
:10D4D000BF91AF919F918F917F916F915F914F918C
:10D4E0003F912F910F900BBE0F900FBE0F901F908A
:10D4F00018951F920F920FB60F9211240BB60F9230
:10D500002F933F934F935F936F937F938F939F934B
:10D51000AF93BF93EF93FF93E091EE35F091EF352A
:10D52000309709F01995FF91EF91BF91AF919F91BD
:10D530008F917F916F915F914F913F912F910F90BC
:10D540000BBE0F900FBE0F901F9018951F920F9259
:10D550000FB60F9211240BB60F922F933F934F9358
:10D560005F936F937F938F939F93AF93BF93EF934B
:10D57000FF93E091EC35F091ED35309709F0199576
:10D58000FF91EF91BF91AF919F918F917F916F919B
:10D590005F914F913F912F910F900BBE0F900FBE57
:10D5A0000F901F9018951F920F920FB60F92112493
:10D5B0000BB60F922F933F934F935F936F937F938D
:10D5C0008F939F93AF93BF93EF93FF93E091EA35CF
:10D5D000F091EB35309709F01995FF91EF91BF91DC
:10D5E000AF919F918F917F916F915F914F913F91FB
:10D5F0002F910F900BBE0F900FBE0F901F9018959C
:10D600001F920F920FB60F9211240BB60F922F9309
:10D610003F934F935F936F937F938F939F93AF93BA
:10D62000BF93EF93FF93E091E835F091E9353097A0
:10D6300009F01995FF91EF91BF91AF919F918F9153
:10D640007F916F915F914F913F912F910F900BBE02
:10D650000F900FBE0F901F9018951F920F920FB64C
:10D660000F9211240BB60F922F933F934F935F931A
:10D670006F937F938F939F93AF93BF93EF93FF939A
:10D68000E091E635F091E735309709F01995FF9173
:10D69000EF91BF91AF919F918F917F916F915F912A
:10D6A0004F913F912F910F900BBE0F900FBE0F9097
:10D6B0001F9018951F920F920FB60F9211240BB660
:10D6C0000F922F933F934F935F936F937F938F931B
:10D6D0009F93AF93BF93EF93FF93E091E435F09165
:10D6E000E535309709F01995FF91EF91BF91AF9112
:10D6F0009F918F917F916F915F914F913F912F916A
:10D700000F900BBE0F900FBE0F901F9018951F9299
:10D710000F920FB60F9211240BB60F922F933F93D7
:10D720004F935F936F937F938F939F93AF93BF9329
:10D73000EF93FF93E091E235F091E335309709F0F4
:10D740001995FF91EF91BF91AF919F918F917F912B
:10D750006F915F914F913F912F910F900BBE0F9062
:10D760000FBE0F901F9018951F920F920FB60F9239
:10D7700011240BB60F922F933F934F935F936F93A8
:10D780007F938F939F93AF93BF93EF93FF93E0911A
:10D79000E035F091E135309709F01995FF91EF915F
:10D7A000BF91AF919F918F917F916F915F914F91B9
:10D7B0003F912F910F900BBE0F900FBE0F901F90B7
:10D7C00018951F920F920FB60F9211240BB60F925D
:10D7D0002F933F934F935F936F937F938F939F9379
:10D7E000AF93BF93EF93FF93E091DE35F091DF3578
:10D7F000309709F01995FF91EF91BF91AF919F91EB
:10D800008F917F916F915F914F913F912F910F90E9
:10D810000BBE0F900FBE0F901F9018951F920F9286
:10D820000FB60F9211240BB60F922F933F934F9385
:10D830005F936F937F938F939F93AF93BF93EF9378
:10D84000FF93E091DC35F091DD35309709F01995C3
:10D85000FF91EF91BF91AF919F918F917F916F91C8
:10D860005F914F913F912F910F900BBE0F900FBE84
:10D870000F901F9018951F920F920FB60F921124C0
:10D880000BB60F922F933F934F935F936F937F93BA
:10D890008F939F93AF93BF93EF93FF93E091DA350C
:10D8A000F091DB35309709F01995FF91EF91BF9119
:10D8B000AF919F918F917F916F915F914F913F9128
:10D8C0002F910F900BBE0F900FBE0F901F901895C9
:10D8D0001F920F920FB60F9211240BB60F922F9337
:10D8E0003F934F935F936F937F938F939F93AF93E8
:10D8F000BF93EF93FF93E091D835F091D9353097EE
:10D9000009F01995FF91EF91BF91AF919F918F9180
:10D910007F916F915F914F913F912F910F900BBE2F
:10D920000F900FBE0F901F9018951F920F920FB679
:10D930000F9211240BB60F922F933F934F935F9347
:10D940006F937F938F939F93AF93BF93EF93FF93C7
:10D95000E091D635F091D735309709F01995FF91C0
:10D96000EF91BF91AF919F918F917F916F915F9157
:10D970004F913F912F910F900BBE0F900FBE0F90C4
:10D980001F9018951F920F920FB60F9211240BB68D
:10D990000F922F933F934F935F936F937F938F9348
:10D9A0009F93AF93BF93EF93FF93E091D435F091A2
:10D9B000D535309709F01995FF91EF91BF91AF914F
:10D9C0009F918F917F916F915F914F913F912F9197
:10D9D0000F900BBE0F900FBE0F901F9018951F92C7
:10D9E0000F920FB60F9211240BB60F922F933F9305
:10D9F0004F935F936F937F938F939F93AF93BF9357
:10DA0000EF93FF93E091D235F091D335309709F041
:10DA10001995FF91EF91BF91AF919F918F917F9158
:10DA20006F915F914F913F912F910F900BBE0F908F
:10DA30000FBE0F901F9018951F920F920FB60F9266
:10DA400011240BB60F922F933F934F935F936F93D5
:10DA50007F938F939F93AF93BF93EF93FF93E09147
:10DA6000D035F091D135309709F01995FF91EF91AC
:10DA7000BF91AF919F918F917F916F915F914F91E6
:10DA80003F912F910F900BBE0F900FBE0F901F90E4
:10DA900018951F920F920FB60F9211240BB60F928A
:10DAA0002F933F934F935F936F937F938F939F93A6
:10DAB000AF93BF93EF93FF93E091CE35F091CF35C5
:10DAC000309709F01995FF91EF91BF91AF919F9118
:10DAD0008F917F916F915F914F913F912F910F9017
:10DAE0000BBE0F900FBE0F901F901895CF93CFB71E
:10DAF000F894282F392F211588E0380749F461E080
:10DB000083E00F94D53364E083E00F94D5334FC0A6
:10DB1000203488E0380749F462E083E00F94D5337D
:10DB200064E083E00F94D53342C0211589E03807C3
:10DB300049F461E084E00F94D53364E084E00F940D
:10DB4000D53335C0203489E0380749F462E084E0F9
:10DB50000F94D53364E084E00F94D53328C02115A9
:10DB60008AE0380749F461E085E00F94D53364E03A
:10DB700085E00F94D5331BC020348AE0380749F480
:10DB800062E085E00F94D53364E085E00F94D533EF
:10DB90000EC021153B4049F461E086E00F94D53377
:10DBA00064E086E00F94D53302C0CFBF01C0CFBF81
:10DBB000CF910895CF93CFB7F894282F392F2115FF
:10DBC00088E0380749F461E083E00F94E13364E0D2
:10DBD00083E00F94E1334FC0203488E0380749F4E4
:10DBE00062E083E00F94E13364E083E00F94E1337B
:10DBF00042C0211589E0380749F461E084E00F94C0
:10DC0000E13364E084E00F94E13335C0203489E0EF
:10DC1000380749F462E084E00F94E13364E084E083
:10DC20000F94E13328C021158AE0380749F461E0F8
:10DC300085E00F94E13364E085E00F94E1331BC08D
:10DC400020348AE0380749F462E085E00F94E1333C
:10DC500064E085E00F94E1330EC021153B4049F4A8
:10DC600061E086E00F94E13364E086E00F94E133F5
:10DC700002C0CFBF01C0CFBFCF910895811528E06A
:10DC8000920729F460931436709315360895803402
:10DC900028E0920729F460930836709309360895B6
:10DCA000811529E0920729F46093003670930136BC
:10DCB0000895803429E0920729F46093F435709335
:10DCC000F535089581152AE0920729F46093EC3523
:10DCD0007093ED35089580342AE0920729F460931B
:10DCE000E0357093E135089581159B4021F46093F0
:10DCF000D8357093D9350895FC01918195FFFDCFFA
:10DD0000608380E090E008954F925F926F927F92DF
:10DD10008F929F92AF92BF92EF92FF920F931F93B9
:10DD2000CF937C014A015B0128013901FC01848108
:10DD300082FF16C0D901C801689412F8B695A7955C
:10DD4000979587951694D1F7B901A801032E36E16E
:10DD500076956795579547953A95D1F7302D15C02B
:10DD6000D901C801689413F8B695A795979587953A
:10DD70001694D1F7B901A801032E37E1769567957E
:10DD8000579547953A95D1F7302D88159905AA05ED
:10DD9000BB0508F4A6C084169506A606B70608F4C7
:10DDA000A2C0F701848182FD04C0880C991CAA1CC2
:10DDB000BB1CC301B201A50194010F944D542F3F28
:10DDC00031054105510508F490C08FEF90E0A0E0C7
:10DDD000B0E0C9EF05C0281739074A075B0758F0BC
:10DDE000880F991FAA1FBB1FCD3F0CF48160CF5F26
:10DDF000C73089F74FC0CC230CF04CC0D501C4010B
:10DE0000880F991FAA1FBB1F880F991FAA1FBB1F2E
:10DE1000880F991FAA1FBB1F481A590A6A0A7B0A52
:10DE2000CE3FF4F48DEF9FEF8C1B9109C7FD9395C6
:10DE300004C0440C551C661C771C8A95D2F7D5018A
:10DE4000C401B695A79597958795BC01CD01640D42
:10DE5000751D861D971DA50194010F944D5437C063
:10DE600083E08C0FA501940104C0220F331F441FCF
:10DE7000551F8A95D2F7DA01C901B695A7959795EE
:10DE80008795BC01CD01640D751D861D971D0F94EE
:10DE90004D541DC083E08C0FA501940104C0220FD6
:10DEA000331F441F551F8A95D2F7DA01C901B69571
:10DEB000A79597958795BC01CD01640D751D861DAD
:10DEC000971D0F944D542150310941095109832F59
:10DED0008F70C295C07FC82BF701C783268381E06E
:10DEE00018C080E016C080E014C0D501C401880FBE
:10DEF000991FAA1FBB1F880F991FAA1FBB1F880F3E
:10DF0000991FAA1FBB1F481A590A6A0A7B0AC9EF40
:10DF100089CFCF911F910F91FF90EF90BF90AF905D
:10DF20009F908F907F906F905F904F9008950F9388
:10DF30001F93CF93DF93EC018B01009709F41EC16F
:10DF4000803C910529F460E180E00F94D53316C13F
:10DF5000C11584E0D80729F464E080E00F94D5333C
:10DF60000DC1C038E1E0DE0729F462E080E00F94E3
:10DF7000D53304C1C115F1E0DF0729F461E080E089
:10DF80000F94D533FBC0C03883E0D80729F461E093
:10DF900081E00F94D533F2C0C039E3E0DE0729F405
:10DFA00061E082E00F94D533E9C0C115F2E0DF07EC
:10DFB00029F462E081E00F94D533E0C0C03482E000
:10DFC000D80729F462E082E00F94D533D7C0C0327D
:10DFD000E3E0DE0729F464E082E00F94D533CEC09D
:10DFE000C115F8E0DF0729F461E083E00F94D53331
:10DFF000C5C0C11589E0D80729F461E084E00F9419
:10E00000D533BCC0C115EAE0DE0729F461E085E044
:10E010000F94D533B3C0C115FBE0DF0729F461E0ED
:10E0200086E00F94D533AAC0C03488E0D80729F41D
:10E0300062E083E00F94D533A1C0C034E9E0DE078D
:10E0400029F462E084E00F94D53398C0C034FAE03C
:10E05000DF0729F462E085E00F94D5338FC0C03923
:10E0600088E0D80729F464E083E00F94D53386C0B4
:10E07000C039E9E0DE0729F464E084E00F94D53389
:10E080007DC0C039FAE0DF0729F464E085E00F9431
:10E09000D53374C0C0398BE0D80729F464E086E03A
:10E0A0000F94D5336BC0C03CE8E0DE0729F468E08C
:10E0B00083E00F94D53362C0C03CF9E0DF0729F458
:10E0C00068E084E00F94D53359C0C03C8AE0D8079B
:10E0D00029F468E085E00F94D53350C0C03AE8E0F9
:10E0E000DE0729F460E183E00F94D53347C0C03ADE
:10E0F000F9E0DF0729F460E184E00F94D5333EC0F6
:10E10000C03A8AE0D80729F460E185E00F94D5335E
:10E1100035C0C03AEBE0DE0729F460E186E00F94F9
:10E12000D5332CC0C03BF8E0DF0729F460E283E080
:10E130000F94D53323C0C03B89E0D80729F460E2AF
:10E1400084E00F94D5331AC0C03BEAE0DE0729F41F
:10E1500060E285E00F94D53311C0C038F4E0DF07EA
:10E1600029F460E483E00F94D53308C0C03A84E01A
:10E17000D80721F460E485E00F94D5338D818F7347
:10E180008D83F80195818481892B9681911198E086
:10E19000892B8D83F801408151816281738100E078
:10E1A00010E62AEE30E0CE01AFDD9C8198609C83C2
:10E1B0009C8190619C83DF91CF911F910F91089575
:10E1C000CF92DF92EF92FF920F931F93CF93DF9343
:10E1D000EC01D901C801B695A79597958795481781
:10E1E00059076A077B0778F46A017B01CC0CDD1CB8
:10E1F000EE1CFF1CC901B801A70196010F944D54F4
:10E200002150310902C020E030E0832F8F708F83CE
:10E210002E83DF91CF911F910F91FF90EF90DF90B0
:10E22000CF900895EF92FF920F931F93CF93DF93B8
:10E23000EC017B01009709F4B9C1803C910529F4F8
:10E2400060E180E00F94D533B1C18115944029F489
:10E2500064E080E00F94D533A9C1C03881E0D807CD
:10E2600029F462E080E00F94D533A0C1C115E1E04C
:10E27000DE0729F461E080E00F94D53397C1C03800
:10E28000F3E0DF0729F461E081E00F94D5338EC11C
:10E29000C03933E0D30729F461E082E00F94D5332D
:10E2A00085C1C11582E0D80729F462E081E00F94AE
:10E2B000D5337CC1C034E2E0DE0729F462E082E0BD
:10E2C0000F94D53373C1C032F3E0DF0729F464E063
:10E2D00082E00F94D5336AC1C11538E0D30729F421
:10E2E00061E083E00F94D53361C1C11589E0D8079F
:10E2F00029F461E084E00F94D53358C1C115EAE0F8
:10E30000DE0729F461E085E00F94D5334FC1C115D4
:10E31000FBE0DF0729F461E086E00F94D53346C1C6
:10E32000C03438E0D30729F462E083E00F94D5339A
:10E330003DC1C03489E0D80729F462E084E00F943D
:10E34000D53334C1C034EAE0DE0729F462E085E069
:10E350000F94D5332BC1C039F8E0DF0729F464E00E
:10E3600083E00F94D53322C1C03939E0D30729F4B3
:10E3700064E084E00F94D53319C1C0398AE0D8072E
:10E3800029F464E085E00F94D53310C1C039EBE087
:10E39000DE0729F464E086E00F94D53307C1C03C62
:10E3A000F8E0DF0729F468E083E00F94D533FEC07E
:10E3B000C03C39E0D30729F468E084E00F94D533FA
:10E3C000F5C0C03C8AE0D80729F468E085E00F94E6
:10E3D000D533ECC0C03AE8E0DE0769F460E183E0E1
:10E3E0000F94D533E0EAF8E084818F7E8483F701CF
:10E3F0002481225053C0C03AF9E0DF0729F460E1DC
:10E4000084E00F94D533D2C0C03A3AE0D30729F460
:10E4100060E185E00F94D533C9C0C03A8BE0D807DE
:10E4200029F460E186E00F94D533C0C0C03BE8E03A
:10E43000DE0729F460E283E00F94D533B7C0C03B18
:10E44000F9E0DF0729F460E284E00F94D533AEC031
:10E45000C03B3AE0D30729F460E285E00F94D5335E
:10E46000A5C0C03884E0D80729F460E483E00F94A5
:10E47000D5339CC0C03AE4E0DE0729F460E485E0CF
:10E480000F94D53393C08C818F7E8C83FB012481C4
:10E490002250CE01C03AF8E0DF0731F480914E06F9
:10E4A00084FD8CC011E18BC0803B38E0930779F08C
:10E4B000803AE9E09E0731F430916E0634FD82C067
:10E4C00019E110C0803BF9E09F0789F001C015E118
:10E4D000803A3AE0930731F480918E0684FD74C04F
:10E4E00011E212C0803BEAE09E0759F001C01DE135
:10E4F000803A9B4049F48091AE0684FD04C019E245
:10E5000003C015E201C01DE2E12FE695E695E69510
:10E5100030E2E39FF0011124FA5F177081E090E090
:10E52000012E02C0880F991F0A94E2F781832230DE
:10E5300010F040E001C040E4DF015096A10FB11D92
:10E540003FB7F8942C9127702C939C91942B9C931B
:10E550003FBF85838D81806C8D83F70184818D7FA2
:10E56000813021F48D8182608D8303C08D818D7F08
:10E570008D83F7018581882321F08D8184608D83CF
:10E5800003C08D818B7F8D83F70140815181628132
:10E59000738100E010E62AEE30E0CE0111DE8C81BE
:10E5A00088608C838C8180618C8310C08C818F7E8D
:10E5B0008C83F70124812250CE0176CF15E180EAC9
:10E5C00098E080CF1DE18ECF15E29ECFDF91CF91F5
:10E5D0001F910F91FF90EF9008950F93E8ECF4E0F6
:10E5E00080818F7D808380818F7D8083E4E1F7E36C
:10E5F00002E00593109216371092173700E2069347
:10E6000000E40693ECE0F7E300E2069300E40693EF
:10E61000E9E5F0E4148615861686178612861386B9
:10E620001092FF360F9108950F9385E08093FF3687
:10E63000E5E1F7E304E00593EDE0F7E304E005939B
:10E640000F9108950F9383E08093FF361092163751
:10E6500010921737E4E1F7E302E006930F91089573
:10E66000E0916540F0916640309709F01995089562
:10E670000F93CF93DF938091FF36833019F4F0DF4F
:10E68000ACDF5EC08091FB369091FC36C091634058
:10E69000D0916440C81BD90B71F52091FD363091A3
:10E6A000FE36820F931F8093FD369093FE362091A5
:10E6B0005F40309160408217930721F080911636B9
:10E6C000882341F084E08093FF36ECE0F7E302E03A
:10E6D000069336C0E0916740F0916840309799F01A
:10E6E0001995882381F01092FB361092FC36C09168
:10E6F0006340D0916440C034D10528F010921636A2
:10E70000C0E4D0E003C081E080931636E0E0F7E398
:10E71000C68BD78B8091FB369091FC36209161405F
:10E7200030916240280F391F208F318FC80FD91FB9
:10E73000C093FB36D093FC36E4E1F7E302E00693A6
:10E74000DF91CF910F910895FC018181E82FE7704F
:10E750008E2F90E0FC013197E730F105D8F488273F
:10E76000EE52FE4F8F4F0D948B5480E190E0089550
:10E7700080E290E0089580E490E0089580E890E0E1
:10E78000089580E091E0089580E092E008958FEF91
:10E7900093E0089588E090E00895282F2F7030E0EE
:10E7A000220F331F082E000C990B8827990F881F02
:10E7B0009927820F931F02979C01220F331F220F6C
:10E7C000331F220F331F820F931F8956994C0895D0
:10E7D0000F93CF938091CC0480FF63C081E080933E
:10E7E000CC04ECE0F7E300E80693E4E1F7E300E8AB
:10E7F00006938093CA04ECE0F7E300E1069380916E
:10E80000FF36882329F08350823008F429DFE5DEC3
:10E8100080910E3790910F37089709F044C088E037
:10E82000EBEBF6E3A9E5B0E401900D928A95E1F7F0
:10E83000E8ECF4E080818062808380818062808364
:10E840000E941862C82F811103C0EEDEC1E02CC007
:10E850008091594088236CF41092FD361092FE3658
:10E860001092FB361092FC3682E08093FF3600DF78
:10E870001BC080915F4090916040892B11F4E2DED3
:10E8800013C01092FD361092FE361092FB36109295
:10E89000FC3681E08093FF36ECE0F7E302E006937C
:10E8A00003C0C0E001C0C1E08C2FCF910F9108954B
:10E8B0008F929F92AF92BF92DF92EF92FF920F934F
:10E8C0001F93CF93DF93D82E68DF8C01CD2DCF70AF
:10E8D000D0E0CE01880F991FCD2D0D2C000CDD0B43
:10E8E000CC27DD0FCC1FDD27C80FD91FCE01880F25
:10E8F000991F880F991F880F991F9C01245F384C1E
:10E900007901C90121DF4C01DD200CF07BC0FE0143
:10E91000EE0FFF1FEE0FFF1FEE0FFF1FE050F94C31
:10E9200022893389D80115968D919C911697820F73
:10E93000931F15968D939C93169713962D913C914A
:10E9400014978217930709F447C0281B390B211528
:10E95000B4E03B0740F02FEF33E0C901B4010F945E
:10E960002654281B390BF801808181FF0AC0C90198
:10E97000B4010F94265441E0892B09F040E0842F24
:10E9800001C080E0D8019C9180FB91F99C93FE012D
:10E99000EE0FFF1FEE0FFF1FEE0FFF1FE050F94CB1
:10E9A000128A138A2687378711962D913C911297E8
:10E9B00015968D919C911697820F931FCC0FDD1F9A
:10E9C000CC0FDD1FCC0FDD1FC05FD84C888399832F
:10E9D000F70102E00693E4C0D8018C9181FFCDC01D
:10E9E0008D7F8C93CC0FDD1FCC0FDD1FCC0FDD1F77
:10E9F000C050D94C1A8A1B8A1E861F86F70102E076
:10EA00000693CEC0FE01EE0FFF1FEE0FFF1FEE0FAD
:10EA1000FF1FE050F94CA684B784D8018C9182FF87
:10EA20001BC01196ED91FC91129715962D913C917A
:10EA3000169713968D919C911497B4010F942654B8
:10EA4000B0E4DB9EB001112469527A4CAC01CF01D5
:10EA5000820F931F0F948A56F801258136812A0D63
:10EA60003B1D25833683838194818217930768F445
:10EA700085839683CC0FDD1FCC0FDD1FCC0FDD1FF0
:10EA8000C050D94C8A899B8978C0FE01EE0FFF1FC8
:10EA9000EE0FFF1FEE0FFF1FE050F94C4289538924
:10EAA000A416B50609F069C02817390709F465C02E
:10EAB000AC01421B530B9A01211554E0350748F075
:10EAC0002FEF33E0C901B4010F942654281B390BF2
:10EAD00006C0C901B4010F942654281B390BFE014E
:10EAE000EE0FFF1FEE0FFF1FEE0FFF1FE050F94C60
:10EAF000168617862815390500F5D8018C91846093
:10EB00008C93B0E4DB9EC001112489529A4CFE0123
:10EB1000EE0FFF1FEE0FFF1FEE0FFF1FE05FF84C21
:10EB200080839183CC0FDD1FCC0FDD1FCC0FDD1F49
:10EB3000C050D94C8A8A9B8A1CC0F80141815281FD
:10EB400085819681840F951FFE01EE0FFF1FEE0F4A
:10EB5000FF1FEE0FFF1FE05FF84C80839183CC0F07
:10EB6000DD1FCC0FDD1FCC0FDD1FC050D94C2A8B11
:10EB70003B8BF70102E0069313C0D8018C9180FF14
:10EB80000FC08E7F8C931796ED91FC91189730975C
:10EB900039F015966D917C9116974D2D80E0199561
:10EBA000DF91CF911F910F91FF90EF90DF90BF9079
:10EBB000AF909F908F900895CF93CFB7F894E1ECEA
:10EBC000F4E080818E7F80831092C00410820F94C5
:10EBD000243410924037CFBFCF9108959FB7F89457
:10EBE00081E080934037EAECF4E080E4808380E2C7
:10EBF0008083E1ECF4E0808181608083A9ECB4E063
:10EC00008C9182608C93E8ECF4E080818064808356
:10EC10008C9181608C938081806880839FBF0895F0
:10EC2000CF93DF93C0E6D0E0188280E30F94EC33FB
:10EC3000E0ECF4E080818064808381E08883CFB75A
:10EC4000F894E0E0F7E31586158A158E15A215A64F
:10EC500015AAE7E9F6E380818E7F8083E0EAF6E398
:10EC600080818E7F8083E9EAF6E380818E7F8083D6
:10EC7000E2EBF6E380818E7F80836AE170E082E0E0
:10EC80000F94E6518F3F19F08093FA0403C08FE18F
:10EC90008093FA046BE170E082E00F94E6518F3FBD
:10ECA00019F08093FB0403C08FE18093FB04E0EC38
:10ECB000F4E08081826080838081806880838081AD
:10ECC000806180838CE097E3868397838081806274
:10ECD00080838FEF8093C504E8ECF4E0808181604D
:10ECE0008083109240377ADFCFBFDF91CF910895B4
:10ECF0008093C30408958091C3040895E9E5F0E486
:10ED000080879187628773870895282F2F7030E05E
:10ED1000220F331F082E000C990B8827990F881F8C
:10ED20009927820F931FFC01EE0FFF1FEE0FFF1FAD
:10ED3000EE0FFF1FE050F94C2585207C09F069C0DB
:10ED40006370613011F018F404C060EC03C060E837
:10ED500001C060E440385105E9F050F440325105FB
:10ED6000A9F040345105A1F040315105D9F40CC04F
:10ED7000411522E0520791F04F3F23E0520781F006
:10ED80004115514079F408C021E00DC022E00BC0CC
:10ED900023E009C024E007C025E005C026E003C049
:10EDA00027E001C020E0FC01EE0FFF1FEE0FFF1F68
:10EDB000EE0FFF1FE050F94C158636E03487262B06
:10EDC0002587FC01EE0FFF1FEE0FFF1FEE0FFF1F49
:10EDD000E050F94C2585207C203C69F4FC01EE0FC5
:10EDE000FF1FEE0FFF1FEE0FFF1FE050F94C2585B0
:10EDF0002770273081F0880F991F880F991F880F7F
:10EE0000991FFC01E050F94C85858062858781E07F
:10EE1000089580E0089581E00895E82FEF70F0E014
:10EE2000EE0FFF1F082E000C990B8827990F881FE3
:10EE30009927E80FF91FEE0FFF1FEE0FFF1FEE0FD0
:10EE4000FF1FE050F94C858582FB882780F90895E3
:10EE5000282F2F7030E0A901440F551F282F082EAE
:10EE6000000C330B2227330F221F3327240F351FAB
:10EE7000F901EE0FFF1FEE0FFF1FEE0FFF1FE05017
:10EE8000F94C958592FF17C0220F331F220F331FB5
:10EE9000220F331FF901E050F94C95859B7F958730
:10EEA0007CDCFC01808180FF06C08E7F8083078030
:10EEB000F085E02D199581E008958F929F92AF9291
:10EEC000BF92CF92DF92EF92FF920F931F93CF9357
:10EED000DF93982E862E6A0179015FDC5C01292D73
:10EEE000C92DCF70D0E0CE01880F991FC92D092CF4
:10EEF000000CDD0BCC27DD0FCC1FDD27C80FD91F81
:10EF0000FE01EE0FFF1FEE0FFF1FEE0FFF1FE05081
:10EF1000F94C8585807C09F47EC0FE01EE0FFF1F51
:10EF2000EE0FFF1FEE0FFF1FE050F94C8585807C30
:10EF3000803C61F0FE01EE0FFF1FEE0FFF1FEE0F92
:10EF4000FF1FE050F94C858582FD67C08FB7F894AC
:10EF5000F501908190FF03C08FBF80E05FC0F50195
:10EF60009081916090838FBFC182D282E382F482CC
:10EF70001582168207831087811006C091E0E11484
:10EF8000F10419F090E001C091E0F501808190FB5F
:10EF900081F98B7F808322235CF4CC0FDD1FCC0FA3
:10EFA000DD1FCC0FDD1FC050D94C1A8A1B8A2FC021
:10EFB000FE01EE0FFF1FEE0FFF1FEE0FFF1FE050D1
:10EFC000F94C8585807C803CB1F4CE01880F991F77
:10EFD000880F991F880F991F845F984CB5DBBC017F
:10EFE000C7010F942654892B31F0F50180818E7F63
:10EFF000808380E013C0CC0FDD1FCC0FDD1FCC0F52
:10F00000DD1FC050D94C1E861F861A8A1B8A892D87
:10F010004FDC81E003C080E001C080E0DF91CF9150
:10F020001F910F91FF90EF90DF90CF90BF90AF9026
:10F030009F908F900895FF920F931F93CF93DF932C
:10F04000182FC82FCF70D0E0CE01880F991FC12F85
:10F05000012E000CDD0BCC27DD0FCC1FDD27C80FE8
:10F06000D91F812F9ADBDC01FE01EE0FFF1FEE0F8F
:10F07000FF1FEE0FFF1FE45FF84C02E005938C9139
:10F0800080FF22C08E7F8C931796ED91FC9118978C
:10F090003097D1F011235CF4CC0FDD1FCC0FDD1FB6
:10F0A000CC0FDD1FC050D94C6A897B890AC0CC0FB8
:10F0B000DD1FCC0FDD1FCC0FDD1FC050D94C6E857E
:10F0C0007F85412F81E01995DF91CF911F910F919D
:10F0D000FF900895CF93C82FAEDFEC2FEF70F0E0D4
:10F0E000EE0FFF1F8C2FCC0F990B8827990F881FCD
:10F0F0009927E80FF91FEE0FFF1FEE0FFF1FEE0F0E
:10F10000FF1FE050F94C1586CF9108950F93E82F1B
:10F11000EF70F0E0EE0FFF1F282F082E000C330BCE
:10F120002227330F221F3327E20FF31FEE0FFF1F9B
:10F13000EE0FFF1FEE0FFF1FDF01A050B94C1D9611
:10F140009C911D9794601D969C93E45FF84C01E0A0
:10F15000069371DF81E00F9108950F931F93CF9372
:10F16000DF938B01C82FCF70D0E0CC0FDD1F282F8D
:10F17000082E000C330B2227330F221F3327C20F18
:10F18000D31F0BDBCC0FDD1FCC0FDD1FCC0FDD1F22
:10F19000C050D94C2D8522FF0AC0FC01208120FDE2
:10F1A0000AC0216020830783108781E005C0F80131
:10F1B000199581E001C080E0DF91CF911F910F91FF
:10F1C00008951F920F920FB60F9211240BB60F9253
:10F1D0000F932F933F934F935F936F937F938F93EF
:10F1E0009F93AF93BF93EF93FF938091CB048823BA
:10F1F00044F480E88093CA040E94E8610E941E598A
:10F2000087C08091CB0482FF20C084E08093CA0431
:10F210008091143786FF7CC08091CC0481FD78C03A
:10F22000D7DA811175C08091FF36813011F40ADA86
:10F230006FC0843009F06CC0E5E1F7E304E00593AA
:10F24000EDE0F7E304E0059363C08091CB0481FF18
:10F250005AC082E08093CA0480910C3786FF58C060
:10F260008091CC0481FD54C0B3DA811151C08091EA
:10F27000FF36823041F484E08093FF36ECE0F7E320
:10F2800002E0069345C0833009F042C0E5E1F7E3B0
:10F2900004E00593EDE0F7E304E0059339C080E175
:10F2A0008093CA0481E0C7DE81E8C5DE0E94BD61AB
:10F2B0001092C304E0E0F7E3158696E0948783E4B8
:10F2C0008587158A948B858B8BEB96E3808B918B4E
:10F2D00084D91EC08091CB0486FF08C080E480934F
:10F2E000CA04109240370E94215912C08091CB0469
:10F2F00085FF0EC080E28093CA0481E0809340378E
:10F300000E94225905C08091CB0484FFE3CFC7CF70
:10F31000FF91EF91BF91AF919F918F917F916F91ED
:10F320005F914F913F912F910F910F900BBE0F90D6
:10F330000FBE0F901F9018951F920F920FB60F924D
:10F3400011240BB60F920F931F932F933F934F935C
:10F350005F936F937F938F939F93AF93BF93CF935D
:10F36000DF93EF93FF938091CC0481FD03C030DAEB
:10F370008111C2C082E08093CC048091C504819544
:10F38000880FECE0F7E3E81BF109208131812C5074
:10F390003743369527953695279536952795822FAD
:10F3A000869520FD02C090E001C090E8890FE82F0B
:10F3B000EF70F0E0EE0FFF1F282F082E000C330B2C
:10F3C0002227330F221F3327E20FF31FDF01AA0F7B
:10F3D000BB1FAA0FBB1FAA0FBB1FA050B94C1C9686
:10F3E0009C9195FF89C0EE0FFF1FEE0FFF1FEE0FE0
:10F3F000FF1FE45FF84C00E20693811178C0809112
:10F40000FF36843019F42CD9E8D876C000910E3735
:10F4100010910F378091634090916440C091FB360A
:10F42000D091FC3698012C0F3D1F8217930718F4DA
:10F430008C010C1B1D0B8091614090916240A801D2
:10F440006BEB76E38C0F9D1F0F948A56C00FD11F74
:10F45000C093FB36D093FC360034110569F48091DB
:10F46000FD369091FE368C0F9D1F20915F403091AC
:10F4700060408217930780F0E9E5F0E4C287D38704
:10F480000684F785E02D309729F01995811102C087
:10F49000CBD832C0D7D830C08091634090916440BF
:10F4A000C817D907F9F4E0916740F09168403097A8
:10F4B00011F4BAD821C01995811102C0B5D81CC069
:10F4C0002091FD363091FE368091FB369091FC36CE
:10F4D000820F931F8093FD369093FE361092FB3679
:10F4E0001092FC36ECE0F7E302E0069305C08038AA
:10F4F00011F4BED801C0DCD9FF91EF91DF91CF911B
:10F50000BF91AF919F918F917F916F915F914F913B
:10F510003F912F911F910F910F900BBE0F900FBE37
:10F520000F901F9018959091800024E0829FB00169
:10F5300011246C7392709160692B80E890E00F94B5
:10F540008751E0E8F0E0828180FDFDCF0895609171
:10F5500080006C73636080E890E00F948751E0E86E
:10F56000F0E0828180FDFDCF0895CF92DF92EF928F
:10F57000FF92CF93DF93EC016B01E12CF12C60E063
:10F5800070E68AEE90E0A70196010F944D54CA01EF
:10F59000B9012FEF3FEF40E050E00F944D5421159B
:10F5A000310529F481E08C8321E030E02DC0223048
:10F5B000310528F482E08C8322E030E025C024303D
:10F5C000310528F483E08C8324E030E01DC028302E
:10F5D000310528F484E08C8328E030E015C0203425
:10F5E000310528F485E08C8320E430E00DC02F3F06
:10F5F000310509F028F486E08C8320E031E004C076
:10F6000087E08C8320E034E040E050E060E070E68A
:10F610008AEE90E00F944D54CA01B901A7019601FA
:10F620000F944D542D833E832436310518F41C82EB
:10F630001D821E82DF91CF91FF90EF90DF90CF90DF
:10F6400008950F931F93CF93DF93EC018901862FC9
:10F6500090E08730910508F08BC0FC018827E752C5
:10F66000FE4F8F4F0D948B5480E098E088839983F0
:10F67000E0E4F6E0308181E090E02FEF240F02C05B
:10F68000880F991F2A95E2F7832B808371C080E44D
:10F6900098E088839983E0E4F6E0308181E090E0AF
:10F6A00023E0240F02C0880F991F2A95E2F7832BCD
:10F6B00080835EC080E099E088839983E0E6F6E08D
:10F6C000308181E090E02FEF240F02C0880F991F56
:10F6D0002A95E2F7832B80834BC080E499E08883EE
:10F6E0009983E0E6F6E0308181E090E023E0240FAA
:10F6F00002C0880F991F2A95E2F7832B808338C0B8
:10F7000080E09AE088839983E0E8F6E0308181E048
:10F7100090E02FEF240F02C0880F991F2A95E2F77F
:10F72000832B808325C080E49AE088839983E0E876
:10F73000F6E0308181E090E023E0240F02C0880FE2
:10F74000991F2A95E2F7832B808312C080E09BE00B
:10F7500088839983E0EAF6E0308181E090E02FEF42
:10F76000240F02C0880F991F2A95E2F7832B80830C
:10F770004A83423061F018F4413031F010C0433018
:10F7800049F0443051F00BC080E18B8308C080E227
:10F790008B8305C080E48B8302C080E88B838881E3
:10F7A00099810E94766DE881F9818181887F8360EB
:10F7B00081831D821E821C82E881F9818081807F85
:10F7C0008083B801CE01D1DEDF91CF911F910F91DF
:10F7D0000895CF93DF93EC012D813E81A62FB0E0F9
:10F7E0000F94935424E630E040E050E00F944D54E1
:10F7F0008A81E881F981E6FD17C0823061F018F452
:10F80000813031F01BC0833049F0843051F016C094
:10F8100020AF31AF13C022AF33AF10C024AF35AF2C
:10F820000DC026AF37AF0AC0813019F0823021F009
:10F8300005C020AF31AF02C022AF33AF8D819E81B2
:10F84000E881F98186A397A38B81E881F981E6FDA0
:10F8500004C09181892B818304C091818073892B9D
:10F860008183E881F9818081807F9C81892B8083DD
:10F87000DF91CF910895CF93DF93EC0141155105AE
:10F8800009F443C0A6ECB2E420E030E0922FF90185
:10F89000E159FB4EE491ED932F5F3F4F2730310547
:10F8A000A9F7FA01DE01C6ECD2E480818B83818165
:10F8B0008C83F901EA53FD4B8CE28083E2E0E90F8F
:10F8C000F0E0EA53FD4B6083C4E0C90F9D5FE92F70
:10F8D000F0E0EA53FD4B8DE78083D0E0FE01EA5370
:10F8E000FD4B108221E0AE0166EC72E4CD010F9475
:10F8F0006A210E94A82A811108C021E0AE0166ECAD
:10F9000072E48EE399E30F946A21DF91CF91089519
:10F910004F925F926F927F928F929F92AF92BF921F
:10F92000DF92EF92FF920F931F93CF93DF931F927B
:10F93000CDB7DEB77C014115510509F466C188E0F9
:10F940008983A6ECB2E420E030E0922FF901E1597E
:10F95000FB4EE491ED932F5F3F4F27303105A9F720
:10F96000FA01162FA6ECB2E4808113968C931397BC
:10F97000818114968C9302E0090FF901EA53FD4B43
:10F980008CE28083623088F5862F0F945908882393
:10F99000B1F0812F0F941E089F938F931F921F9396
:10F9A0008BE599E29F938F93E02FF0E0EA53FD4BB4
:10F9B000FF93EF930F94B856CDBFDEBF08C1812FE0
:10F9C0000E9406C29F938F931F921F938BE599E22B
:10F9D0009F938F93E02FF0E0EA53FD4BFF93EF935B
:10F9E0000F94B856CDBFDEBFF2C0663109F078C0C3
:10F9F00086E10F9462072B013C010E94ECFE4B0153
:10FA00005C01672B682B692BF1F4C301B20120E183
:10FA10003EE040E050E00F946F545F934F933F936C
:10FA20002F931F9286E18F9382E699E29F938F93A3
:10FA3000E02FF0E0EA53FD4BFF93EF930F94B8569D
:10FA4000CDBFDEBFC4C0802F0E94A1C1992334F571
:10FA5000C301B20120E13EE040E050E00F946F545A
:10FA6000CA01B9010F94E726BF92AF929F928F927D
:10FA70009F938F937F936F931F9286E18F938AE674
:10FA800099E29F938F93E02FF0E0EA53FD4BFF93B1
:10FA9000EF930F94B856CDBFDEBF99C0BF92AF921F
:10FAA0009F928F92C301B20120E13EE040E050E01E
:10FAB0000F946F545F934F933F932F931F9286E160
:10FAC0008F9387E799E29F938F93E02FF0E0EA53BB
:10FAD000FD4BFF93EF930F94B856CDBFDEBF77C0B9
:10FAE000663071F5E02FF0E0EA53FD4B86E380834A
:10FAF0006894DD24D2F8D90E9D5FE92FF0E0EA5337
:10FB0000FD4B8CE2808386E00F9462078B019C01A1
:10FB10008D2D90E04BE0BE016F5F7F4F8A539D4B70
:10FB20000F944027E981ED0DAE2FB0E0AA53BD4BF5
:10FB30008DE78C93EF5FF0E0EA53FD4B108247C0F6
:10FB4000653071F5E02FF0E0EA53FD4B85E38083EB
:10FB50006894DD24D2F8D90E9D5FE92FF0E0EA53D6
:10FB6000FD4B8CE2808385E00F9462078B019C0142
:10FB70008D2D90E04BE0BE016F5F7F4F8A539D4B10
:10FB80000F948C28E981ED0DAE2FB0E0AA53BD4B48
:10FB90008DE78C93EF5FF0E0EA53FD4B108217C0C6
:10FBA000862F0F9462079F938F937F936F931F927B
:10FBB0001F9382E699E29F938F93802F90E08A5360
:10FBC0009D4B9F938F930F94B856CDBFDEBFE6EC4D
:10FBD000F2E401900020E9F73197E65CF244E98312
:10FBE000AF01552721E066EC72E4C7010F946A214A
:10FBF0000E94A82A811109C0498150E021E066ECE9
:10FC000072E48EE399E30F946A210F90DF91CF9114
:10FC10001F910F91FF90EF90DF90BF90AF909F905A
:10FC20008F907F906F905F904F900895AC01611519
:10FC3000710571F1E8E7F4E1A6ECB2E42EEC32E4F0
:10FC400094919D933196A217B307D1F7FB01CA0196
:10FC5000A6ECB2E4208113962C931397218114967D
:10FC60002C93149718961C92189721E048E050E0C6
:10FC7000BD010F946A210E94A82A811109C021E0C8
:10FC800048E050E066EC72E48EE399E30D946A215B
:10FC90000895EF92FF920F931F93CF93DF938C0100
:10FCA0006115710509F47FC04115510509F47BC048
:10FCB000E6E6F4E1A6ECB2E4CEECD2E494919D93B6
:10FCC0003196AC17BD07D1F7FA017B01C6ECD2E43F
:10FCD00080818B8381818C831F922F9383E899E2AB
:10FCE0009F938F938EEC92E49F938F930F94B856CB
:10FCF00009900020E9F72197C65CD244F701818181
:10FD00000F900F900F900F900F900F90811115C0D2
:10FD100080811F928F9386E791E29F938F93DD27D7
:10FD2000CA53DD4BDF93CF930F94B8560F900F90CB
:10FD30000F900F900F900F9016C01F928F93F701A6
:10FD400080811F928F9383E791E29F938F93DD27AA
:10FD5000CA53DD4BDF93CF930F94B856EDB7FEB780
:10FD60003896EDBFFEBFE6ECF2E401900020E9F723
:10FD70003197E65CF244EF01DD2721E0AE0166EC4D
:10FD800072E4C8010F946A210E94A82A81110BC055
:10FD90000E53194341F021E0AE0166EC72E48EE3AC
:10FDA00099E30F946A21DF91CF911F910F91FF90FA
:10FDB000EF900895CF93DF93EC014115510509F4BD
:10FDC0003FC0662361F0E8E7F4E1A6ECB2E490E01E
:10FDD00024912D939F5F31969730D1F70BC0EFE6BA
:10FDE000F4E1A6ECB2E490E024912D939F5F31966C
:10FDF0009730D1F7DA01CE01E6ECF2E42C912383BF
:10FE000011962C9124832CE227833CE430872187B0
:10FE100020E322872DE72387148621E04CE050E081
:10FE2000BF010F946A210E94A82A811109C021E014
:10FE30004CE050E066EC72E48EE399E30F946A21A3
:10FE4000DF91CF910895EF92FF920F931F93CF937D
:10FE5000DF9300D01F92CDB7DEB70097C9F16630AF
:10FE60007105C0F1FC0120812035B1F521812C32D2
:10FE7000A9F524812C32A1F57A018C010B5F1F4F6B
:10FE8000AB01455051099E012F5F3F4FB8018CE2F5
:10FE90000F941727882349F149815A814B5F5F4F9F
:10FEA00049835A8346305105E8F045509E012D5F45
:10FEB0003F4F60E0C8010F949F258823B1F08B81EC
:10FEC0009C818C31910580F4F701808381E00DC025
:10FED00080E00BC080E009C080E007C080E005C082
:10FEE00080E003C080E001C080E02496CDBFDEBF8B
:10FEF000DF91CF911F910F91FF90EF900895CF92D6
:10FF0000DF92EF92FF920F931F93CF93DF93CDB7C2
:10FF1000DEB72C97CDBFDEBF009709F431C1663044
:10FF2000710508F42FC1FC012081203509F02CC196
:10FF300021812C3209F02AC124812C3209F028C1F8
:10FF40007B018C016C01F5E0CF0ED11CAB0145505B
:10FF500051099E012F5F3F4FB6018CE20F94172786
:10FF6000982F882309F423C149815A814B5F5F4F41
:10FF700049835A834630510508F40CC145509E010F
:10FF80002D5F3F4F60E0C6010F949F25982F882377
:10FF900009F40DC12B813C812C31310508F0FCC0E6
:10FFA00049815A81DA011196AE15BF0508F0F6C0F5
:10FFB0002C31310508F0F4C0F9018827E052FE4FDA
:10FFC0008F4F0D948B54C8018A0F9B1FFC016081D9
:10FFD0006D3241F4FA013296EE15FF0508F0E2C0E9
:10FFE00040E002C0FD0141E02631310559F46E2D9B
:10FFF0006E1B9E01275F3F4FC8018E0F9F1F0E94FF
:020000021000EC
:1000000058F512C02630310541F46E2D6A1BAE0141
:10001000475F5F4F0E9425F807C06E2D6A1BAE0137
:10002000475F5F4F0E9441F9882309F4BDC04985AD
:100030005A856B857C858B810E94F5C6982F882315
:1000400009F4B5C049855A856B857C858B810F94F1
:10005000750791E0ACC04E2D4A1B9E012B5F3F4FB0
:1000600060E0C8018A0F9B1F0F942A26982F8823CF
:1000700009F49DC04D815E816F81788549875A87DB
:100080006B877C878B810E94F5C6982F882309F4A3
:100090008EC089859A85AB85BC858B309105A1057D
:1000A000B10549F48BE89CE30E94392F982F8823EF
:1000B00009F47DC00CC00C97A105B10544F08BE894
:1000C0009CE30E94392F982F882309F470C049853A
:1000D0005A856B857C858B810F94750791E067C08D
:1000E0004E2D4A1B9E012B5F3F4F60E0C8018A0FD7
:1000F0009B1F0F942A26982F882309F458C04D81FE
:100100005E816F81788549875A876B877C878B8171
:100110000E94F5C6982F882349F049855A856B853A
:100120007C858B810F94750791E041C02B813C81C8
:10013000A9014C50510946305105C8F549855A85E9
:100140006B857C85452B462B472B89F540E050E09D
:10015000BA01822F0F94750791E029C0C7018A1B4D
:100160009B0B899718F56E2D6A1B422FC8018A0FC9
:100170009B1F0F94E00791E0811119C090E017C018
:1001800090E015C090E013C090E011C090E00FC067
:1001900090E00DC090E00BC090E009C090E007C077
:1001A00090E005C090E003C090E001C090E0892F8E
:1001B0002C96CDBFDEBFDF91CF911F910F91FF90A5
:1001C000EF90DF90CF9008950F931F93CF93DF931D
:1001D0001F921F92CDB7DEB7009741F166307105CF
:1001E00038F1FC012081203529F521812C3221F5BF
:1001F00024812C3219F58C01AB0145505109BC0109
:100200006B5F7F4F9E012F5F3F4F8CE20F9417274C
:100210008823B9F089819A810596069788F081E054
:10022000F8019581963469F080E00BC080E009C048
:1002300080E007C080E005C080E003C080E001C02E
:1002400080E00F900F90DF91CF911F910F91089553
:10025000EF92FF920F931F93CF93DF9300D000D0C4
:10026000CDB7DEB7009709F453C06630710508F4C6
:1002700051C0FC012081203509F04EC021812C3273
:1002800009F04CC024812C3209F04AC07B018C015A
:10029000AB0145505109BC016B5F7F4F9E012F5F41
:1002A0003F4F8CE20F941727882309F442C08981BD
:1002B0009A819C012B5F3F4F29833A832630310579
:1002C00088F1F8012581263479F506968E159F056B
:1002D00068F54E2D481B9E012D5F3F4F60E0800F5B
:1002E000911F0F942A26882321F16B817C818D81B7
:1002F0009E818B019C010150110921093109073EA2
:10030000134021053105A0F40E948AC281E011C08A
:1003100080E00FC080E00DC080E00BC080E009C02D
:1003200080E007C080E005C080E003C080E001C03D
:1003300080E02696CDBFDEBFDF91CF911F910F9158
:10034000FF90EF9008950F931F93CF93DF93EC01ED
:100350006115710509F444C0A6ECB2E420E030E078
:10036000922FF901E159FB4EE491ED932F5F3F4F3E
:1003700027303105A9F7FB01A6ECB2E48081139682
:100380008C931397818114968C931497F901EA53F7
:10039000FD4B8CE280839E5FE92FF0E0EA53FD4B3A
:1003A00086E49DE7808391831282FD010190002005
:1003B000E9F73197E65CF2448F01112721E0A801AB
:1003C000BD01CE010F946A210E94A82A811108C0A4
:1003D00021E0A80166EC72E48EE399E30F946A21B0
:1003E000DF91CF911F910F910895FC01892B61F04E
:1003F0006530710558F08081803551F481E091813C
:100400009C3239F080E0089580E0089580E00895FE
:1004100080E00895009799F06330710590F0FC0139
:100420002081203581F421812C3279F424812C32F1
:1004300071F485818354823060F080E0089580E01B
:10044000089580E0089580E0089580E0089580E0B8
:10045000089581E00895009791F06330710588F068
:10046000FC012081203579F421812C3271F4248122
:100470002C3269F485818F3461F080E0089580E04A
:10048000089580E0089580E0089580E0089580E078
:10049000089581E00895009791F06330710588F028
:1004A000FC012081203579F421812C3271F42481E2
:1004B0002C3269F48581873561F080E0089580E011
:1004C000089580E0089580E0089580E0089580E038
:1004D000089581E00895CF92DF92EF92FF920F93FB
:1004E0001F93CF93DF934115510509F4AFC00097D7
:1004F00009F4AEC06630710508F4ACC0FC0120817F
:10050000203509F0A9C021812C3209F0A7C024812F
:100510002C3209F0A5C08581873509F0A3C0EA0116
:100520008BE89CE30E944F14883009F49DC08BE84F
:100530009CE30E944F14863009F498C00F9462190E
:100540000E94F35361E081E99CE30E9467560F9497
:100550009D080E94371D813079F582E00E94AFC16D
:100560006B017C01DD24EE24FF24B701A60182E0AB
:100570000F947507B701A60182E00E9497C10E94FF
:10058000A82A811119C084E1E7E8F9E2A1E2B4E404
:1005900001900D928A95E1F7E1E2F4E401900020E8
:1005A000E9F73197AF014152544420E061E274E42D
:1005B0008EE399E30F946A21CE010E94861C80E0AD
:1005C0000E947DC19B01AC016894EE24E2F801ED2C
:1005D00012E2BE01685E7F4FCE0106960E94C157AF
:1005E0008D8340E050E0BA01CE010E94E92E8D815A
:1005F000882351F182E00E94A1C1062F8BE00E9466
:10060000A1C121E0611120E040E350E4BE016C5C37
:100610007F4FCE01C6960E94C450CE010E945C1C42
:100620009E01265A3D4FAE01475A5D4FBE016C5A9E
:100630007D4FCE018D5A9D4F0E94702D0E94E83350
:1006400068E0CE010E943C148D8111C080E00FC093
:1006500080E00DC080E00BC080E009C080E007C0F2
:1006600080E005C080E003C080E001C080E0DF9151
:10067000CF911F910F91FF90EF90DF90CF90089551
:10068000CF92DF92EF92FF920F93CF93DF934115BA
:10069000510509F4B0C0009709F4AFC06630710588
:1006A00008F4ADC0FC012081203509F0AAC02181E9
:1006B0002C3209F0A8C024812C3209F0A6C0EA012E
:1006C0008581833409F493C0843409F0A0C00E946A
:1006D0003FC20F943B088BE89CE30E944F14883084
:1006E00009F497C08BE89CE30E944F14863009F40C
:1006F00092C00F9462190E94F35361E081E99CE378
:100700000E9467560F949D080E94371D813079F52D
:1007100082E00E94AFC16B017C01DD24EE24FF2446
:10072000B701A60182E00F947507B701A60182E028
:100730000E9497C10E94A82A811119C084E1E7E8AC
:10074000F9E2A1E2B4E401900D928A95E1F7E1E2C9
:10075000F4E401900020E9F73197AF01415254448D
:1007600020E061E274E48EE399E30F946A2180E073
:100770000E947DC19B01AC01BE01685E7F4FCE012E
:1007800006960E94FB538D8340E050E0BA01CE01F3
:100790000E94E92E8D81882341F182E00E94A1C14F
:1007A000062F8BE00E94A1C121E0611120E040E30F
:1007B00050E4BE016C5C7F4FCE01C6960E94C450CF
:1007C000CE010E945C1C9E01265A3D4FAE01475A45
:1007D0005D4FBE016C5A7D4FCE018D5A9D4F0E94D8
:1007E000702D68E0CE010E943C148D8115C00F94DD
:1007F0003B0881E011C080E00FC080E00DC080E0C8
:100800000BC080E009C080E007C080E005C080E048
:1008100003C080E001C080E0DF91CF910F91FF9095
:10082000EF90DF90CF900895BF92CF92DF92EF923A
:10083000FF920F931F93CF93DF931F92CDB7DEB735
:100840006115710509F464C0DB017C01E6ECF2E49A
:100850008BE7808380E781838CE282839C91938302
:1008600011969C91948385839FE49683878380E08F
:100870000E94FCC88B019C0148E0BE016F5F7F4F66
:100880008EEC92E40F94EE28E981E85FD12C0F2ED4
:10089000FCE2BF2EF02DCC24C394CE0EF0E0EA5340
:1008A000FD4BB082D3948D2D0E94FCC88B019C011E
:1008B0008C2D90E048E0BE016F5F7F4F8A539D4BC7
:1008C0000F94EE28E981EC0D83E0D812E4CF81E0AB
:1008D0008E0FF0E0EA53FD4B9DE79083482F50E0E8
:1008E000FA01EA53FD4B1082898321E066EC72E441
:1008F000C7010F946A210E94A82A811109C0498169
:1009000050E021E066EC72E48EE399E30F946A21F3
:100910000F90DF91CF911F910F91FF90EF90DF909B
:10092000CF90BF900895CF93DF9341155105A9F162
:100930000097A9F165307105A0F1FC0120812035F7
:1009400091F521812C3289F52281263481F5EA0145
:1009500084818235E9F0833531F0843451F50E9489
:1009600069C281E027C00F946219BE016C5C7F4FA1
:10097000CE01C6960E94C94E8BE89CE30E94F322EA
:1009800081110F948419CE010E94402A8D8112C0DA
:10099000CA01C6960E9446FE0DC080E00BC080E0F2
:1009A00009C080E007C080E005C080E003C080E0AF
:1009B00001C080E0DF91CF910895FC01892B79F08F
:1009C0006630710570F08081833569F481818C32E5
:1009D00061F481E094819C3249F080E0089580E0E8
:1009E000089580E0089580E0089580E008950F93D1
:1009F000CF93DF93009709F476C06630710508F451
:100A000074C0FC016081633509F071C061816C3292
:100A100009F06FC064816C3209F06DC04115510559
:100A200009F46BC02115310509F469C08581813352
:100A300009F067C0B901EA01F9011082CA010E94F8
:100A4000DA20882309F45FC0CE010E94BB20811107
:100A50002BC0CE010E94402A61E0CE010E946B278C
:100A600064E0CE010E943C1461E0CE010E94AC2003
:100A700019820E94D0A2E2E0F3E4808190E0DC01E0
:100A8000AE5FBC4B25853685880F991FFC01EE5F54
:100A9000FC4B418152811F960C9161E08BE89CE3F5
:100AA0000E945A2581E032C00E94A82A81112DC0DF
:100AB00083E1EBE9F9E2A6ECB2E401900D928A95AC
:100AC000E1F7E6ECF2E401900020E9F73197AF019D
:100AD000465C524421E066EC72E48EE399E30F94A5
:100AE0006A2181E013C080E011C080E00FC080E087
:100AF0000DC080E00BC080E009C080E007C080E04E
:100B000005C080E003C081E001C081E0DF91CF91AA
:100B10000F9108950F93CF93DF93009709F45EC16F
:100B20006630710508F45CC1DC012C91233509F0B5
:100B300059C111962C9111972C3209F055C1149678
:100B40002C9114972C3209F051C14115510509F42B
:100B50004FC11596EC918E2F90E0FC01F097E53493
:100B6000F10508F047C1EA018827E450FE4F8F4F96
:100B70000D948B54CA010E944F14843031F0CE0181
:100B80000E944F14893009F037C1CE010E943820ED
:100B9000CE010F94540BCE010E94402A0F9462198B
:100BA00060E08BE89CE30E946B2763E0CE010E942B
:100BB0003C1419820E94BDA2E2E0F3E4808190E03F
:100BC000DC01AE5FBC4B25853685880F991FFC0183
:100BD000EE5FFC4B418152811F960C9161E08BE8E6
:100BE0009CE30E945A2591E016C1CA010E94BB20D5
:100BF000882309F403C181E0898360E0CE010E946B
:100C00003E1560E0CE010E942C150E94A82A811199
:100C1000F7C080E1EEEAF9E2A6ECB2E401900D92B1
:100C20008A95E1F7E6ECF2E401900020E9F73197CC
:100C3000AF01465C524421E066EC72E48EE399E336
:100C40000F946A2191E0E7C0CA010E94BB2088236B
:100C500009F4D8C060E0CE010E943E1560E0CE01EC
:100C60000E942C15FE01ED5AFD4FDE01A75ABD4F23
:100C70008C918083319611968C91808319820E9489
:100C8000A82A8111C1C080E1EEEBF9E2A6ECB2E442
:100C900001900D928A95E1F7E6ECF2E401900020D4
:100CA000E9F73197AF01465C524421E066EC72E40B
:100CB0008EE399E30F946A2191E0ADC0CA010E94CE
:100CC000BB20982F882309F4A6C0CE010E940828D3
:100CD00091E08111A0C090E09EC0CA010E94BB209B
:100CE000882329F0CE010E949227982F94C00E9459
:100CF0004EC991E090C0CA010E94BB20982F882362
:100D000009F489C00F94621960E08BE89CE30E94AB
:100D10006B2769E0CE010E943C141982CE010F942A
:100D2000640BCE010E94F01CCE010F94FE0F0F94B5
:100D3000661C61E0CE010E94AC2091E06CC0CA014B
:100D40000E944F14893009F061C060E370E4CE0165
:100D50000F949B0FCE010F945B0B843109F058C0A8
:100D6000CE010F94640BCE010F94FE0F0F94661CFE
:100D700091E051C0CA010E944F14893009F04AC065
:100D8000CE010F94540BCE010E94402A61E0CE01A7
:100D90000E946B2764E0CE010E943C1461E0CE010A
:100DA0000E94AC2019820E94D0A2E2E0F3E480818C
:100DB00090E0DC01AE5FBC4B25853685880F991F1E
:100DC000FC01EE5FFC4B418152811F960C9161E06A
:100DD0008BE89CE30E945A2591E01DC090E01BC067
:100DE00090E019C090E017C090E015C090E013C0EB
:100DF00090E011C090E00FC091E00DC091E00BC0F9
:100E000091E009C091E007C091E005C090E003C007
:100E100091E001C090E0892FDF91CF910F9108956B
:100E2000FC01892B61F06630710558F080818D34AA
:100E300051F481E091819C3239F080E0089580E0A6
:100E4000089580E0089580E00895FC01892B61F009
:100E50006630710558F08081823551F481E09181CE
:100E60009C3239F080E0089580E0089580E0089594
:100E700080E00895FC01892B61F06530710558F020
:100E800080818A3551F481E091819C3239F080E093
:100E9000089580E0089580E0089580E00895CF925D
:100EA000DF92EF92FF920F931F93CF93DF93CDB713
:100EB000DEB72897CDBFDEBF009709F457C0653075
:100EC000710508F455C0FC0120812A3509F052C093
:100ED00021812C3209F050C07B018C016C01F2E0C1
:100EE000CF0ED11CAB01425051099E012F5F3F4FE5
:100EF000B6018CE20F941727882309F446C0498174
:100F00005A814E5F5F4F49835A8343305105B0F198
:100F100042509E012D5F3F4F60E0C6010F949F2518
:100F2000882399F18B819C81039750F589819A815F
:100F300001968E159F0530F54E2D481B9E012B5FA7
:100F40003F4F60E0800F911F0F942A268823E9F01D
:100F50006D817E818F819885623071058105910553
:100F600098F48B810E9447DE81E00FC080E00DC0C5
:100F700080E00BC080E009C080E007C080E005C0D1
:100F800080E003C080E001C080E02896CDBFDEBFD6
:100F9000DF91CF911F910F91FF90EF90DF90CF9055
:100FA00008952F923F924F925F926F927F928F920D
:100FB0009F92AF92BF92CF92DF92EF92FF920F93E8
:100FC0001F93CF93DF93CDB7DEB76397CDBFDEBF5F
:100FD0008C01F62E81E08D830115110509F423C3E0
:100FE0008093CE2089E10E94A1C1672B682B692BD9
:100FF00009F025C30F947B01B82E811103C0F110B5
:1010000020C385C38BE89CE30E942D21B82E882342
:1010100009F47DC38BE89CE30E944F148F87F11085
:1010200004C08150823008F400C32F85243031F48D
:101030008BE89CE30E94862A33E03F870F943E09A9
:101040000F9427098BE89CE30E94F32281110F94EF
:1010500084198BE89CE30E94402A82E00E94A1C18F
:10106000E62E8FEF8E0D8A3008F0E1C2AE014A5FA6
:101070005F4FBE016B5F7F4F8E2D0E9468228E8175
:101080000E94B2DD8E8184700E9426DE8D810F94D5
:1010900099030F2EF6ECCF2EF2E4DF2EF02D8BE726
:1010A000D6018C938DE611968C9311978CE2129653
:1010B0008C93129787E713968C9320E044E050E0DE
:1010C000B601C8010F946A211F92EF928EEC99E24B
:1010D0009F938F93DF92CF920F94B856F6010190B1
:1010E0000020E9F73197AF01465C524420E0B60199
:1010F000C8010F946A21E8E7F3E587858F93868519
:101100008F9385858F9384858F930F2EF2EDAF2E6D
:10111000F9E2BF2EF02DBF92AF92DF92CF920F94E3
:10112000B856F60101900020E9F73197AF01465C0F
:10113000524420E0B601C8010F946A218AE00E945F
:10114000A1C19F938F937F936F93BF92AF92DF92D2
:10115000CF920F94B856F60101900020E9F731972D
:10116000AF01465C524420E0B601C8010F946A21E9
:101170008BE00E94A1C19F938F937F936F93BF9247
:10118000AF92DF92CF920F94B856F60101900020F3
:10119000E9F73197AF01465C524420E0B601C8013F
:1011A0000F946A210F2EF2E9CF2EF3E5DF2EF02DFA
:1011B000CDBFDEBF412C512C320145010F2EF6EC84
:1011C000AF2EF2E4BF2EF02D2BC0D6018C911196DC
:1011D0009C91119712962C91129713963C91B4E022
:1011E000CB0ED11C3F932F939F938F939F928F92FF
:1011F000BF92AF920F94B856F50101900020E9F725
:101200003197AF01465C524420E0B501C8010F940C
:101210006A21EFEF4E1A5E0A6E0A7E0ACDBFDEBF6C
:101220000F94631C90E0A0E0B0E0481659066A06EF
:101230007B0658F28DE78093C64221E041E050E002
:1012400066EC72E4C8010F946A2165E08BE89CE3C8
:101250000E943C140F9462198BE89CE30E94452580
:101260000E94A05960E072E080E090E00E94925AF3
:101270001092694010926A4087E193E40E9461A84D
:101280000E94335C8111FCCFB82EF11004C00E9483
:1012900020208823E1F389E00E94A1C16F3171050C
:1012A0008105910508F59B01AC01012E1CE0220F80
:1012B000331F441F551F1A95D1F7102D2B873C87DC
:1012C0004D875E87CA01B9010F94E0080F942C1A6C
:1012D00081E00F947C1C80E090E1A0E0B0E08F837F
:1012E0009887A987BA873FC09B01AC01012E19E0FE
:1012F000220F331F441F551F1A95D1F7102D2B872E
:101300003C874D875E87CA01B9010F94E0080F94AE
:101310002C1A0F94AC1C80E092E0A0E0B0E08F8328
:101320009887A987BA871FC0412C512C32019F2C66
:10133000CB84DC84ED84FE840F94E91C8823E1F0E7
:101340008D810F94561867E173E40E94C4A8A82EFB
:101350000F94D81C9FEF491A590A690A790AA110FB
:101360000BC0F92C0FC02B853C854D855E85232B4A
:10137000242B252BC9F606C04C145D046E047F0493
:10138000D8F2F92C0F94D31C87E193E40E9428A98A
:10139000E82E0E941F5B0F942716EE2031F06F8518
:1013A0008BE89CE30E943C14B2C180E495E40E9467
:1013B0003ECF882351F0F11008C060913F4670E0A5
:1013C00080E495E40E9488A909C0E6ECF2E410826A
:1013D000118262E070E0CF010E9488A960E072E0B3
:1013E00080E090E00E94A8590E94335C8111FCCFFC
:1013F0008B859C85AD85BE85892B8A2B8B2B09F42B
:10140000F3C0C12CD12C76010F2EF6EC2F2EF2E476
:101410003F2EF02D4F80588469847A8491E0491AD8
:101420005108610871080E9477A9809369409093E0
:101430006A40AE014F5F5F4FBC018D810E94501525
:10144000882309F463C1C701B6012F813885498516
:101450005A850F944D544B015C01672B682B692B07
:10146000A1F5C701B6012F81388549855A850F94AA
:101470004D54288B398B4A8B5B8B89E00E94A1C12C
:10148000AB89AF93BA89BF93E989EF93F889FF934A
:101490009F938F937F936F9327ED39E23F932F9321
:1014A0003F922F920F94B856F10101900020E9F776
:1014B0003197AF01465C524420E0B101C8010F945E
:1014C0006A211092CE20CDBFDEBF2F81388549859D
:1014D0005A85211582E038074105510509F4BAC043
:1014E000211530414105510509F4DDC0D701C60180
:1014F00087709927AA27BB27892B8A2B8B2B09F06A
:1015000043C08C818F938B818F938A818F93898144
:101510008F93A2EEBAE2BF93AF933F922F920F94B4
:10152000B856F10101900020E9F73197AF01465C10
:10153000524420E0B101C8010F946A21C701B601ED
:101540002F81388549855A850F944D542F5F3F4F21
:101550004F4F5F4F6F81788589859A850F940B5423
:10156000CDBFDEBFA7019601285F3F4F4F4F5F4FB2
:10157000621773078407950719F41092CE20C0C034
:1015800031E03093CE20BCC01092CE20841495045C
:10159000A604B70479F4EDE7D101EC9321E041E032
:1015A00050E0B101C8010F946A210FC0ECE2D101F3
:1015B000EC9304C08091CE20882339F020E041E0F4
:1015C00050E0B101C8010F946A21FFEFCF1ADF0A82
:1015D000EF0AFF0A2B853C854D855E85C216D30632
:1015E000E406F50609F01FCF0E94735A0F942716E0
:1015F0000F94972A80E390E40F945D4C6F858BE8FD
:101600009CE30E943C140F94B5098BE89CE30E9474
:10161000F32281110F9484198BE89CE30E94402AE5
:10162000BB24B39474C0B12C72C0B12C70C0B12C67
:101630006EC08BE89CE30E944F148F87F6CCFF248A
:10164000F3948BE89CE30E942D21B82E882309F4A3
:101650005EC0EFCF8C818F938B818F938A818F9324
:1016600089818F9342EE5AE25F934F933F922F927C
:101670000F94B856F10101900020E9F73197AF01BE
:10168000465C524420E0B101C8010F946A2191E008
:101690009093CE20CDBFDEBF481459046A047B046A
:1016A00009F084CF78CF8C818F938B818F938A813F
:1016B0008F9389818F93E2EEFAE2FF93EF933F924B
:1016C0002F920F94B856F10101900020E9F731975D
:1016D000AF01465C524420E0B101C8010F946A2179
:1016E00031E03093CE20CDBFDEBF481459046A04E8
:1016F0007B0409F05BCF4FCFECE2D101EC935ACFE2
:1017000084149504A604B704B9F745CFB82E8B2DE1
:101710006396CDBFDEBFDF91CF911F910F91FF90F8
:10172000EF90DF90CF90BF90AF909F908F907F9081
:101730006F905F904F903F902F900895CF92DF92DF
:10174000EF92FF921F93CF93DF936115710509F418
:1017500074C04630510508F472C0DB01EC91ED34E1
:1017600009F06FC01196EC91EC3209F06CC02115B4
:10177000310509F46AC0009709F469C069017A016A
:10178000EB012D81203341F440E060E00ADC11E000
:10179000811160C010E05EC0233541F5C6010E9492
:1017A0003A21182F882309F455C0C70106970297DC
:1017B00018F40E9449AA0CC08E818C3219F00E9444
:1017C00049AA06C069EF6E0DCE0107960E9414AAC1
:1017D000A601485E5F4FB6016A5C7F4F80E00E94C1
:1017E0005C4A11E0811136C010E034C00E94A82A82
:1017F000182F81112EC08D811F928F9383EE99E255
:101800009F938F93C6ECD2E4DF93CF930F94B85697
:1018100009900020E9F72197AE01465C524421E08F
:1018200066EC72E48EE399E30F946A210F900F90B7
:101830000F900F900F900F900DC010E00BC010E0B4
:1018400009C010E007C010E005C010E003C010E0C0
:1018500001C010E0812FDF91CF911F91FF90EF9099
:10186000DF90CF900895FC01892BA9F068307105B5
:10187000A0F08081813599F481818C3291F484814A
:101880008C3289F486818C3281F481E095819033A9
:1018900069F080E0089580E0089580E0089580E098
:1018A000089580E0089580E0089580E00895EF9223
:1018B000FF920F931F93CF93DF9300D0CDB7DEB786
:1018C0009CE29B8321153105A9F161157105A1F1F8
:1018D000FA013197F39790F5823390F5803391F5C3
:1018E000C9017A018B010E944F14843069F59E0171
:1018F0002F5F3F4F41E050E0BE016D5F7F4F80E3BF
:1019000090E40F94AF4A9E012F5F3F4FA701B801AB
:1019100080E390E40F94AF4A80E390E40F945D4C31
:101920000F941B1C8BE690E40E9448A00F94F11AC0
:1019300081E00BC080E009C080E007C080E005C006
:1019400080E003C081E001C080E02396CDBFDEBF10
:10195000DF91CF911F910F91FF90EF900895FC01BF
:10196000892B61F06330710558F080818C3451F41B
:1019700081E091819C3239F080E0089580E0089503
:1019800080E0089580E00895452BB1F00097B1F014
:10199000672BB1F0FC0185818136A1F480EB91E4E5
:1019A0000E947BA0811110C060E070E080EB91E4A8
:1019B0000E9486A081E0089580E0089580E0089567
:1019C00080E0089580E0089580E00895CF93DF934C
:1019D000452BC9F10097C9F165317105C0F1FC01D2
:1019E00025812037B1F52781203319F41092BE41AB
:1019F00009C0213321F421E02093BE4103C022E03D
:101A00002093BE41EC0180EB91E40E947BA0811108
:101A100022C00E943A34811109C0BE01675F7F4F26
:101A200080EB91E40E9486A081E018C08091BE41C5
:101A3000811113C0BE01675F7F4F89EE9EE30E9454
:101A4000E9A181E00BC080E009C080E007C080E030
:101A500005C080E003C080E001C081E0DF91CF914C
:101A60000895CF93DF93452B61F1009761F16531C4
:101A7000710558F1FC0125812E3649F52781203367
:101A800019F41092BE4109C0213321F421E02093C2
:101A9000BE4103C022E02093BE41EC0180EB91E403
:101AA0000E947BA0811115C08091BE41882399F0CE
:101AB000BE01675F7F4F80EB91E40E94A7A081E0A9
:101AC0000BC080E009C080E007C080E005C080E076
:101AD00003C080E001C081E0DF91CF9108950097BD
:101AE00099F06630710590F0FC018581833681F4B0
:101AF00080EB91E40E947BA0882361F00E94FC9E11
:101B00001092B04181E0089580E0089580E008954A
:101B100080E0089581E00895FC01892B49F066304A
:101B2000710540F081E09581933729F080E00895B8
:101B300080E0089580E00895FC01892B49F066302B
:101B4000710540F081E09581953629F080E0089597
:101B500080E0089580E00895BF92CF92DF92EF92E7
:101B6000FF920F931F93CF93DF9300D0CDB7DEB7D3
:101B70009CE29B83882359F000919E41002311F041
:101B800010E009C000916B4010916C4004C00091BE
:101B90009F411091A0410D3291E0190710F00CE225
:101BA00011E00115110509F44CC0B82E9E012F5FFC
:101BB0003F4F41E050E0BE016D5F7F4F80E390E416
:101BC0000F94AF4A10926D4010926E4020E030E0CA
:101BD000C12CD12C0F2EFBE6EF2EF0E4FF2EF02DC2
:101BE000F901E559FF4B95819B839E012F5F3F4F84
:101BF00041E050E0BE016D5F7F4F80E390E40F94C1
:101C0000AF4A29813A81232B19F4EFEFCE1ADE0A6D
